:100000000C94241E0C94511E0C94511E0C94511EE1
:100010000C94511E0C94511E0C94511E0C94511EA4
:100020000C94511E0C94511E0C94511E0C94511E94
:100030000C94511E0C94ADFD0C94511E0C94511E49
:100040000C94511E0C94926D0C94511E0C94511EE4
:100050000C94511E0C94511E0C94DB5E0C9404FA0B
:100060000C94511E0C9413240C94511E0C94511E8C
:100070000C94511E0C94511E0C94511E0C94511E44
:100080000C94511E0C94511E0C94511E0C94511E34
:100090000C94511E0C94511E0C94511E0C945AF247
:1000A0000C94511E0C94511E0C94511E0C94511E14
:1000B0000C94511E0C94511E0C94511E0C94511E04
:1000C0000C94511E0C94511E0C94511E0C94511EF4
:1000D0000C94511E0C94511E0C94511E0C94511EE4
:1000E0000C94511E084AD73B3BCE016E84BCBFFD29
:1000F000C12F3D6C74319ABD56833DDA3D00C77FF8
:1001000011BED9E4BB4C3E916BAAAABE0000008090
:100110003F05A84CCDB2D44EB93836A9020C50B91F
:10012000918688083CA6AAAA2ABE000000803F4DFE
:10013000383420582059205A2045006563686F3AAA
:100140000043616E6E6F7420656E74657220737506
:10015000626469723A20004D3234004D32332025FA
:1001600073006175746F25692E67004572726F7236
:100170003A006572726F722077726974696E6720D7
:10018000746F2066696C65004E6F74205344207054
:1001900072696E74696E67002F0053442070726933
:1001A0006E74696E67206279746520002E00446564
:1001B0006C6574696F6E206661696C65642C20469D
:1001C000696C653A200046696C652064656C6574ED
:1001D00065643A002E006F70656E206661696C651B
:1001E000642C2046696C653A200057726974696E08
:1001F0006720746F2066696C653A20002E006F706E
:10020000656E206661696C65642C2046696C653A90
:1002100020002E006F70656E206661696C65642C2D
:100220002046696C653A200046696C652073656CF0
:100230006563746564002053697A653A20004669F5
:100240006C65206F70656E65643A20002E006F70DB
:10025000656E206661696C65642C2046696C653A40
:1002600020004E6F772066726573682066696C6542
:100270003A20004E6F7720646F696E672066696C64
:10028000653A20002220706F730022207061726531
:100290006E743A2200535542524F5554494E4520F0
:1002A00043414C4C207461726765743A2200747249
:1002B00079696E6720746F2063616C6C207375625E
:1002C0002D67636F64652066696C65732077697458
:1002D0006820746F6F206D616E79206C6576656C37
:1002E000732E204D4158206C6576656C2069733AF9
:1002F0000053442063617264206F6B006F70656E01
:10030000526F6F74206661696C656400766F6C75FE
:100310006D652E696E6974206661696C6564005351
:100320004420696E6974206661696C006563686F5A
:100330003A004572726F723A0053544F5050454420
:100340002E20005072696E7465722073746F707025
:1003500065642064756520746F206572726F7273B6
:100360002E2046697820746865206572726F72204D
:10037000616E6420757365204D39393920746F20A2
:10038000726573746172742E202854656D70657285
:1003900061747572652069732072657365742E20AF
:1003A0005365742069742061667465722072657388
:1003B00074617274696E6729004B494C4C45442E38
:1003C00020005072696E7465722068616C74656497
:1003D0002E206B696C6C28292063616C6C6564212C
:1003E000006F6B00526573656E643A200022005501
:1003F0006E6B6E6F776E20636F6D6D616E643A2009
:1004000022004368616E67652066696C616D656E88
:1004100074006C636420636F6E7472617374207611
:10042000616C75653A2000486F74656E64206F6674
:1004300066736574733A007A5F6D696E3A2000796D
:100440005F6D696E3A2000785F6D696E3A20005AE0
:100450003A00593A0020436F756E7420583A2000D4
:10046000453A005A3A00593A00583A004649524D26
:10047000574152455F4E414D453A4D61726C696E30
:100480002056313B20537072696E7465722F67720B
:10049000626C206D617368757020666F722067658D
:1004A0006E36204649524D574152455F55524C3A9F
:1004B000687474703A2F2F7777772E6D656E646548
:1004C0006C2D70617274732E636F6D2050524F5497
:1004D0004F434F4C5F56455253494F4E3A312E30A1
:1004E000204D414348494E455F545950453A447563
:1004F000616C4D6574616C54415A20455854525595
:100500004445525F434F554E543A32205555494465
:100510003A30303030303030302D303030302D30D7
:100520003030302D303030302D30303030303030D1
:1005300030303030300A004475616C4D6574616C48
:1005400054415A204F66662E004475616C4D6574A7
:10055000616C54415A2052656164792E0042656491
:1005600020646F6E652E0020423A0020453A005408
:100570003A004265642048656174696E672E0048E0
:10058000656174696E6720646F6E652E0020573A4E
:100590000020453A00543A0048656174696E672E40
:1005A0002E2E002042403A0020403A00202F003AF0
:1005B00000205400202F0020423A00202F006F6BB3
:1005C00020543A002569206D696E2C20256920731E
:1005D000656300456E642066696C65206C697374A0
:1005E00000426567696E2066696C65206C6973748A
:1005F000004E6F206D6F76652E00526573756D69C4
:100600006E67207072696E74005761697420666F3E
:100610007220757365722E2E2E00536C6565702ED8
:100620002E2E00000095430080A24300007A43FF75
:10063000FFFF0000000000000000000000000000BC
:100640000000000000000000000000009543008052
:10065000A24300007A430000A0400000A040000038
:100660008040256920686F757273202569206D6947
:100670006E7574657300446F6E65207072696E7478
:10068000696E672066696C650053544F505045444D
:100690002E20005072696E7465722073746F7070D2
:1006A00065642064756520746F206572726F727363
:1006B0002E2046697820746865206572726F7220FA
:1006C000616E6420757365204D39393920746F204F
:1006D000726573746172742E202854656D70657232
:1006E00061747572652069732072657365742E205C
:1006F0005365742069742061667465722072657335
:1007000074617274696E6729006F6B004E6F204CC4
:10071000696E65204E756D62657220776974682018
:10072000636865636B73756D2C204C617374204C2A
:10073000696E653A20004E6F20436865636B737580
:100740006D2077697468206C696E65206E756D62C6
:1007500065722C204C617374204C696E653A2000E0
:10076000636865636B73756D206D69736D61746328
:10077000682C204C617374204C696E653A20004CE3
:10078000696E65204E756D626572206973206E6FAB
:1007900074204C617374204C696E65204E756D62D7
:1007A00065722B312C204C617374204C696E653A54
:1007B00020004D31313000446F6E652073617669E1
:1007C0006E672066696C652E006F6B004D323900D4
:1007D0002020506C616E6E6572427566666572426D
:1007E000797465733A20002046726565204D656D09
:1007F0006F72793A20004A756C20323820323031DD
:100800003500436F6D70696C65643A200028416C57
:10081000657068204F626A656374732C20496E634B
:100820002C2054415A2020636F6E6669672900208E
:100830007C20417574686F723A20004A756C2032D2
:100840003820323031352031323A35353A343900BA
:10085000204C61737420557064617465643A2000A3
:10086000312E302E30004D61726C696E20002053A5
:100870006F667477617265205265736574002057E6
:1008800061746368646F6720526573657400204209
:10089000726F776E206F75742052657365740020D7
:1008A00045787465726E616C205265736574005092
:1008B0006F77657255700073746172740022006501
:1008C0006E717565696E672022002200656E717514
:1008D00065696E672022004572726F723A00457238
:1008E000723A204D415854454D50204245440054E1
:1008F000656D706572617475726520686561746597
:100900006420626564207377697463686564206F2E
:1009100066662E204D415854454D502074726967CB
:100920006765726564202121004572723A204D4945
:100930004E54454D50003A20457874727564657286
:10094000207377697463686564206F66662E204D36
:10095000494E54454D5020747269676765726564ED
:100960002021004572723A204D415854454D5000A7
:100970003A20457874727564657220737769746380
:10098000686564206F66662E204D415854454D5071
:1009900020747269676765726564202100202D20CC
:1009A000496E76616C6964206578747275646572ED
:1009B000206E756D6265722021001000AD0330015C
:1009C0006A0150022B0170030A019004F500B00582
:1009D000E500D006D800F007CE001009C500300AA7
:1009E000BE00500BB700700CB100900DAB00B00E04
:1009F000A600D00FA200F0109D0010129900301335
:100A000095005014920070158E0090168B00B01750
:100A10008700D0188400F0198100101B7E00301C64
:100A20007B00501D7900701E7600901F7300B0206F
:100A30007000D0216E00F0226B0010246900302578
:100A40006600502663007027610090285E00B02980
:100A50005C00D02A5900F02B5600102D5400302E87
:100A60005100502F4E0070304B0090314800B03292
:100A70004500D0334200F0343E0010363B003037A2
:100A800037005038330070392E00903A2900B03BBF
:100A90002300D03C1B00F03D1100103F0100F03F4F
:100AA0000000504944204175746F74756E6520666E
:100AB000696E697368656421205075742074686577
:100AC000204B702C204B6920616E64204B642063A6
:100AD0006F6E7374616E747320696E746F20436FF0
:100AE0006E66696775726174696F6E2E6800504931
:100AF00044204175746F74756E65206661696C651C
:100B000064212074696D656F75740020403A006F30
:100B10006B20543A006F6B20423A00504944204108
:100B200075746F74756E65206661696C65642120EB
:100B300054656D706572617475726520746F6F2095
:100B40006869676800204B643A2000204B693A20AE
:100B500000204B703A200020436C61736963205081
:100B6000494420002054753A2000204B753A20005B
:100B7000206D61783A2000206D696E3A2000206473
:100B80003A200020626961733A20001000C9021007
:100B9000012C014001220170011801B0010E01F089
:100BA0000104015002FA00B002F0003003E600D068
:100BB00003DC009004D2007005C800A006BE00004F
:100BC00008B400B009AA00D00BA000600E96006027
:100BD000118C000015820020197800C01D6E00A045
:100BE000226400B0275A00902C500000314600E0EB
:100BF000343C0010383200903A2800603C1E00A0BF
:100C00003D1400803E0A00203F000045313A20009C
:100C100045303A20005A3A2000593A2000583A20EC
:100C2000004D53312C4D53322050696E730A00240D
:100C3000F404D9201BC40C5C0E9804C4095F02653F
:100C4000077101F405F900FB04B30048048700C1F3
:100C50000369005803550003034500BE023A0084AF
:100C600002310053022A002902250004022000E478
:100C7000011C00C8011900AF01170098011400847D
:100C8000011300710110006101100051010E0043B9
:100C9000010D0036010B002B010B0020010B00158C
:100CA0000109000C01090003010800FB000800F322
:100CB000000800EB000700E4000600DE000600D894
:100CC000000600D2000600CC000500C7000500C2E7
:100CD000000500BD000400B9000400B5000400B127
:100CE000000400AD000400A9000400A5000300A258
:100CF0000003009F0004009B000300980003009580
:100D000000020093000300900003008D0002008B9E
:100D100000030088000200860002008400030081B6
:100D20000002007F0002007D0002007B00020079CB
:100D300000020077000100760002007400020072D9
:100D4000000100710002006F0002006D0001006CE4
:100D50000002006A000100690002006700010066ED
:100D600000010065000100640002006200010061F2
:100D7000000100600001005F0002005D0001005CF6
:100D80000001005B0001005A0001005900010058F9
:100D900000010057000100560001005500010054F9
:100DA00000010053000000530001005200010051F7
:100DB000000100500001004F0001004E0000004EF5
:100DC0000001004D0001004C0001004B0000004BF1
:100DD0000001004A000100490001004800000048ED
:100DE00000010047000100460000004600010045E8
:100DF00000000045000100440001004300000043E2
:100E000000010042000000420001004100000041DA
:100E1000000100400001003F0000003F0001003ED3
:100E20000000003E0001003D0000003D0001003CCC
:100E30000000003C0000003C0001003B0000003BC3
:100E40000001003A0000003A0001003900000039BA
:100E500000010038000000380000003800010037B1
:100E600000000037000100360000003600000036A8
:100E7000000100350000003500000035000100349D
:100E80000000003400000034000100330000003393
:100E90000000003300010032000000320000003288
:100EA000000100310000003100000031000100307D
:100EB00000000030000000300001002F0000002F73
:100EC0000000002F0000002F0001002E0000002E67
:100ED0000000002E0001002D0000002D0000002D5C
:100EE0000000002D0001002C0000002C0000002C50
:100EF0000000002C0001002B0000002B0000002B44
:100F00000000002B0001002A0000002A0000002A37
:100F10000000002A0001002900000029000000292B
:100F2000000000290000002900010028000000281E
:100F30000000002800000028000000280001002711
:100F40000000002700000027000000270000002705
:100F500000010026000000260000002600000026F8
:100F600000000026000100250000002500000025EB
:100F700000000025000000250000002500010024DD
:100F800000000024000000240000002400000024D1
:100F900000010023000000230000002300000023C4
:100FA00000000023000000230000002300010022B5
:100FB00000000022000000220000002200000022A9
:100FC000000000220001002100000021000000219B
:100FD000000000210000002100000021000000218D
:100FE0000001002000000020000000200000002080
:100FF0000000002000000020000000200000002071
:101000000001001F0000001F0000001F0000001F63
:101010000000001F0000001F0000001F0001001E54
:101020000000001E0000001E0000001E0000002442
:10103000F4D43050C38E20C2A24017828B7011129C
:101040007A910D816CD90AA861E108C758660761D9
:101050005143061E4B5D05C145A7041A4111040901
:101060003D9803713931034036DB0265339102D478
:10107000305402802E1D02632CEE01752AC501B08A
:1010800028A001102781018F2564012B244B01E04A
:10109000223401AC211F018D200D01801FFC008432
:1010A0001EED00971DDF00B81CD200E61BC6002015
:1010B0001BBC00641AB200B219A8000A19A0006A89
:1010C000189900D117910040178B00B51684003194
:1010D000167E00B31579003A157300C7146F0058D7
:1010E000146A00EE1366008813630025135E00C7C0
:1010F000125B006C12570015125400C111510070A0
:10110000114F0021114B00D61049008D10470046A9
:1011100010440002104200C00F4000800F3E004209
:101120000F3C00060F3B00CB0E3800930E37005CDF
:101130000E3500270E3400F30D3200C10D31009042
:101140000D3000600D2E00320D2D00050D2C00D944
:101150000C2B00AE0C2900850C29005C0C270035F7
:101160000C27000E0C2600E80B2400C40B2400A062
:101170000B23007D0B23005A0B2100390B21001893
:101180000B2000F80A1F00D90A1E00BB0A1E009D92
:101190000A1D00800A1D00630A1C00470A1B002C60
:1011A0000A1B00110A1A00F7091A00DD091900C408
:1011B000091900AB091900920917007B091800638F
:1011C0000917004C09160036091600200916000AF6
:1011D000091500F5081500E0081400CC081400B843
:1011E000081400A4081400900813007D0812006B76
:1011F0000813005808120046081200340811002392
:101200000811001208110001081100F0071000E099
:10121000071000D0071000C0071000B0070F00A192
:1012200007100091070E0083070F0074070F006579
:10123000070E0057070E0049070E003B070D002E52
:10124000070E0020070D0013070D0006070D00F91B
:10125000060C00ED060D00E0060C00D4060C00C8DC
:10126000060C00BC060C00B0060C00A4060B00998E
:10127000060C008D060B0082060B0077060B006C37
:10128000060B0061060A0057060B004C060A0042D6
:10129000060A0038060A002E060A0024060A001A6A
:1012A000060A001006090007060A00FD050900F4F9
:1012B000050900EB050900E2050900D9050900D080
:1012C000050900C7050900BE050900B5050800AD00
:1012D000050800A50509009C050800940508008C78
:1012E000050800840508007C050800740508006CEA
:1012F000050700650508005D050700560508004E56
:1013000005070047050700400508003805070031BC
:101310000507002A050700230507001C050600161F
:101320000507000F0507000805060002050700FB7A
:10133000040600F5040700EE040600E8040600E2D7
:10134000040700DB040600D5040600CF040600C92C
:10135000040600C3040600BD040600B7040600B17D
:10136000040500AC040600A6040600A00405009BCA
:1013700004060095040500900406008A0405008513
:10138000040500800406007A040500750405007059
:101390000405006B04050066040500610405005C9B
:1013A00004050057040500520405004D04050048DB
:1013B000040500430405003E0404003A040500351A
:1013C000040500300404002C040500270404002355
:1013D0000405001E0404001A04040016040500118C
:1013E0000404000D040400090405000404040000C2
:1013F000040400FC030400F8030400F4030400F0F8
:10140000030400EC030400E8030400E4030400E028
:10141000030400DC030400D8030400D4030400D058
:10142000030400CC030400C8030300C503030065E4
:1014300063686F3A00656E6473746F7073206869D7
:10144000743A205A00205A3A00656E6473746F70C3
:1014500073206869743A20590020593A00656E6417
:1014600073746F7073206869743A20580020583A7A
:1014700000656E6473746F7073206869743A20003D
:101480007C3C3E5E2B3D3F2F5B5D3B2C2A225C006B
:101490006563686F3A0020746F6F206C6F6E672011
:1014A000657874727573696F6E2070726576656E9B
:1014B0007465640020636F6C642065787472757362
:1014C000696F6E2070726576656E746564000006E3
:1014D0000900FE06018902FE20FFFE07FE06FE004F
:1014E00000000600070106060602008080808000DA
:1014F00080030303060103A0A0A00507070600FF61
:101500005050F850F850500509090600FE2070A808
:10151000A07028A870200608080600FF40A8481000
:10152000204854080507070600FF609090609890D7
:10153000680103030602038080800207070602FF9A
:10154000408080808080400207070602FF80404084
:10155000404040800505050600008850F850880589
:1015600005050600002020F820200204040602FEE3
:10157000C0404080050101060002F8020202060296
:1015800000C0C00406060601001010204080800440
:101590000606060100609090909060030606060122
:1015A0000040C0404040E004060606010060901084
:1015B0002040F0040606060100F020601010E0054F
:1015C000060606000010305090F8100406060601CA
:1015D00000F080E01010E00406060601006080E0E4
:1015E000909060040606060100F0101020404004B0
:1015F00006060601006090609090600406060601F1
:1016000000609090701060020505060200C0C000E6
:10161000C0C00207070602FEC0C000C040408005EF
:101620000505060000186080601805030306000128
:10163000F800F8050505060000C0300830C00407B2
:101640000706010060901060400040050606060095
:10165000007090A8B0807005060606000020508833
:10166000F88888050606060000F088F08888F004EF
:101670000606060100609080809060040606060160
:1016800000E090909090E0040606060100F080E0F3
:101690008080F0040606060100F080E0808080046F
:1016A0000606060100609080B09060040606060100
:1016B000009090F0909090030606060100E04040F4
:1016C0004040E00506060600003810101090600447
:1016D000060606010090A0C0A09090040606060130
:1016E000008080808080F005060606000088D8A86B
:1016F000A8888804060606010090D0B09090900556
:1017000006060600007088888888700406060601B0
:1017100000E09090E080800407070601FF60909051
:10172000D0B06010040606060100E09090E09090B2
:10173000040606060100609040209060050606063B
:101740000000F820202020200406060601009090CA
:1017500090909060040606060100909090F0606002
:101760000506060600008888A8A8D888050606068B
:101770000000885020205088050606060000888852
:1017800050202020040606060100F010204080F0C2
:10179000030606060100E080808080E0040606065D
:1017A0000100808040201010030606060100E020A2
:1017B000202020E0050303060003205088050101D6
:1017C0000600FEF802020206020480400404040639
:1017D0000100709090700406060601008080E09081
:1017E00090E0040404060100708080700406060680
:1017F000010010107090907004040406010060B0A5
:10180000C070040606060100205040E04040040677
:10181000060601FE60909070106004060606010046
:101820008080E09090900306060601004000C040D2
:1018300040E00308080601FE200060202020A040B0
:101840000406060601008080A0C0A09003060606DC
:101850000100C040404040E0050404060000D0A85C
:10186000A888040404060100E09090900404040693
:101870000100609090600406060601FEE09090E092
:1018800080800406060601FE70909070101004041B
:1018900004060100A0D0808004040406010070C08A
:1018A00030E00406060601004040E04050200404F9
:1018B00004060100909090700404040601009090CA
:1018C000606005040406000088A8A850040404060B
:1018D0000100906060900406060601FE90909070F2
:1018E0009060040404060100F02040F0030707069E
:1018F0000100204040804040200107070602FF8091
:10190000808080808080030707060100804040209F
:1019100040408004020206010350A0FFFFFFFFFFCA
:10192000FFFFFFFFFFFFFFFFFFFFFFFFFFFFFFFFC7
:10193000FFFFFFFFFFFFFFFFFFFFFFFF00000006AD
:1019400000070106060602008000808080800406F1
:10195000060601FF2070A0A070200507070600FF03
:10196000304840F04040F8050505060000A85088C2
:1019700050A80506060600008850F820F820010748
:10198000070602FF80808000808080040707060130
:10199000FF708060906010E0030101060105A00661
:1019A0000707060000788494A4948478030505064C
:1019B000010160A06000E00505050600002850A0B8
:1019C0005028040303060100F01010040101060171
:1019D00002F00607070600007884B4A4A484780403
:1019E0000101060105F00403030601026090600591
:1019F00007070600FF2020F8202000F80305050651
:101A0000010140A02040E0030505060101C020407F
:101A100020C002020206020440800405050601FF00
:101A20009090B0D08005060606000078E8E86828A7
:101A300028010101060202800202020602FE408025
:101A400003050506010140C04040E003050506010D
:101A50000140A04000E0050505060000A050285008
:101A6000A00508080600FF40C040507030781005FF
:101A700008080600FF40C0405068081038050808F4
:101A80000600FFC0204030F0307810040707060140
:101A900000200020608090600507070600004020BD
:101AA000205070888805070706000010202050701D
:101AB0008888050707060000205020507088880598
:101AC0000707060000285020507088880507070681
:101AD000000050002050708888050707060000208D
:101AE00050205070888805060606000078A0F0A0F7
:101AF000A0B80408080601FE609080809060204035
:101B00000407070601004020F080E080F00407078A
:101B10000601002040F080E080F004070706010085
:101B20002050F080E080F00407070601005000F02C
:101B300080E080F00307070601008040E04040405D
:101B4000E00307070601002040E0404040E00307B3
:101B50000706010040A0E0404040E00307070601FF
:101B600000A000E0404040E0050606060000704886
:101B7000E848487004070706010050A090D0B090D4
:101B800090040707060100402060909090600407D1
:101B9000070601002040609090906004070706014E
:101BA000002050609090906004070706010050A04C
:101BB00060909090600407070601005000609090CC
:101BC000906005050506000088502050880408082C
:101BD0000601FF1070B0B0D0D0E080040707060106
:101BE000004020909090906004070706010020407C
:101BF000909090906004070706010020509090900C
:101C000090600407070601005000909090906005D6
:101C10000707060000102088502020200406060632
:101C2000010080E09090E0800406060601006090CC
:101C3000A0A090A00407070601004020007090902B
:101C400070040707060100204000709090700407A0
:101C500007060100205000709090700407070601ED
:101C60000050A0007090907004060606010050001D
:101C7000709090700407070601002050207090902B
:101C80007005040406000070A8B07804060606017A
:101C9000FE7080807020400407070601004020008D
:101CA00060B0C07004070706010020400060B0C0AB
:101CB0007004070706010020500060B0C0700406E1
:101CC00006060100500060B0C0700307070601005F
:101CD000804000C04040E0030707060100204000AC
:101CE000C04040E003070706010040A000C040409C
:101CF000E0030606060100A000C04040E00407071C
:101D00000601003060107090906004070706010023
:101D100050A000E0909090040707060100402000CA
:101D200060909060040707060100204000609090DA
:101D300060040707060100205000609090600407CF
:101D40000706010050A0006090906004060606019E
:101D5000005000609090600505050600002000F826
:101D6000002004040406010070B0D0E00407070658
:101D700001004020009090907004070706010020A9
:101D800040009090907004070706010020500090DA
:101D90009090700406060601005000909090700428
:101DA00009090601FE2040009090907090600408A0
:101DB000080601FE8080E09090E08080040808061C
:101DC00001FE500090909070906000060900FE07A0
:101DD0000199032B20FFFE08FE07FE00000006000D
:101DE00000010707060200808080808000800303D6
:101DF00003060104A0A0A00507070600005050F844
:101E000050F850500507070600002070A070287099
:101E10002005070706000048A8502050A890050795
:101E20000706000040A0A040A89068010303060236
:101E300004808080030707060100204080808040E6
:101E40002003070706010080402020204080050570
:101E5000050600018850F850880505050600012098
:101E600020F820200303030601FF604080050101E4
:101E7000060003F80303030601FF40E040050707DF
:101E800006000008081020408080050707060000B3
:101E9000205088888850200507070600002060A091
:101EA000202020F8050707060000708808304080D1
:101EB000F8050707060000F80810300888700507C5
:101EC0000706000010305090F810100507070600B4
:101ED00000F880B0C8088870050707060000304089
:101EE00080B0C88870050707060000F808101020A9
:101EF00040400507070600007088887088887005D4
:101F00000707060000708898680810600307070636
:101F100001FF40E0400040E0400307070601FF40AA
:101F2000E040006040800407070601001020408068
:101F3000402010050303060002F800F80407070616
:101F40000100804020102040800507070600007037
:101F5000881020200020050707060000708898A838
:101F6000B0807005070706000020508888F8888830
:101F7000050707060000F04848704848F0050707C5
:101F800006000070888080808870050707060000C2
:101F9000F04848484848F0050707060000F88080E8
:101FA000F08080F8050707060000F88080F0808048
:101FB00080050707060000708880809888700507F4
:101FC00007060000888888F88888880307070601C4
:101FD00000E04040404040E00507070600003810A0
:101FE00010101090600507070600008890A0C0A0A0
:101FF0009088050707060000808080808080F805B3
:1020000007070600008888D8A8888888050707067B
:1020100000008888C8A8988888050707060000700F
:10202000888888888870050707060000F08888F08F
:102030008080800508080600FF7088888888A8705E
:1020400008050707060000F08888F0A090880507BB
:102050000706000070888070088870050707060072
:1020600000F820202020202005070706000088888F
:10207000888888887005070706000088888850507F
:102080005020050707060000888888A8A8D888057A
:102090000707060000888850205088880507070633
:1020A000000088885020202020050707060000F83F
:1020B0000810204080F8030707060100E0808080B8
:1020C0008080E00507070600008080402010080897
:1020D000030707060100E02020202020E00503037D
:1020E0000600042050880501010600FFF8020202E4
:1020F000060206804005050506000070087888780D
:102100000507070600008080B0C888C8B00505052F
:102110000600007088808870050707060000080820
:1021200068988898680505050600007088F8807032
:10213000050707060000304840F04040400507070B
:102140000600FE7888887808887005070706000072
:102150008080B0C88888880307070601004000C057
:10216000404040E00409090601FE10003010101044
:1021700090906005070706000080808890E09088B6
:10218000030707060100C04040404040E005050548
:10219000060000D0A8A8A888050505060000B0C85C
:1021A00088888805050506000070888888700507FE
:1021B000070600FEB0C888C8B08080050707060083
:1021C000FE68988898680808050505060000B0C8EC
:1021D00080808005050506000070807008F0050706
:1021E000070600004040F040404830050505060065
:1021F0000088888898680505050600008888505082
:10220000200505050600008888A8A85005050506D4
:10221000000088502050880507070600FE8888982F
:1022200068088870050505060000F8102040F804CD
:102230000707060100304020C02040300107070694
:10224000020080808080808080040707060100C033
:102250002040304020C005030306000448A8900039
:10226000000001000000000001000000000001006B
:10227000000000000100000000000100000000005C
:10228000010000000000010000000000010000004B
:10229000000001000000000001000000000001003B
:1022A000000000000100000000000100000000002C
:1022B000010000000000010000000000010000001B
:1022C000000001000000000001000000000001000B
:1022D00000000000010000000000010000000000FC
:1022E00001000000000001000000000001000000EB
:1022F00000000100000000000100000000000100DB
:1023000000000000010000000000010000000000CB
:1023100001000000000001000000000001000000BA
:10232000000001000000000006000001070706028F
:1023300000800080808080800507070600FF2078ED
:10234000A0A0A07820050707060000304840E04024
:1023500048B005050506000088705070880508081B
:102360000600FF88885020F8202020010707060279
:1023700000808080008080800508080600FF708053
:10238000E09048380870030101060107A00507071F
:102390000600007088A8C8A8887004060606010117
:1023A0007090B05000F006050506000024489048E3
:1023B00024040202060102F010040101060103F0E8
:1023C0000507070600007088E8C8C8887005010185
:1023D000060007F803030306010440A040050606B3
:1023E0000600002020F82020F804050506010360FF
:1023F000902040F0040505060103E0106010E002A3
:10240000020206020640800506060600FF8888884C
:10241000C8B08005070706000078E8E86828282883
:10242000010101060203800202020602FE4080034F
:10243000050506010340C04040E004060606010110
:102440006090906000F00605050600009048244862
:10245000900609090600FF40C04040E40C143C040B
:102460000609090600FF40C04040E81404081C05A6
:1024700009090600FFC0204020C818287808050771
:10248000070600002000202040887005080806008C
:10249000004020708888F888880508080600001029
:1024A00020708888F8888805080806000020507089
:1024B0008888F8888805080806000048B070888871
:1024C000F888880508080600005000708888F88899
:1024D000880508080600002050708888F88888065B
:1024E00007070600003C50909CF0909C05090906E7
:1024F00000FE7088808080887020400508080600F3
:102500000040F88080F08080F80508080600001080
:10251000F88080F08080F805080806000020F88028
:1025200080F08080F805080806000050F88080F0F0
:102530008080F80308080601008040E040404040E9
:10254000E00308080601002040E040404040E0036E
:10255000080806010040A0E040404040E0030808B1
:10256000060100A000E040404040E00507070600EB
:1025700000F04848E84848F00508080600002850E0
:1025800088C8A89888880508080600004020708838
:1025900088888870050808060000102070888888E0
:1025A00088700508080600002050708888888870A8
:1025B000050808060000285070888888887005087B
:1025C0000806000050007088888888700505050698
:1025D0000000885020508805070706000070989872
:1025E000A8C8C870050808060000402088888888A8
:1025F0008870050808060000102088888888887080
:1026000005080806000020500088888888700508A2
:102610000806000050008888888888700508080629
:1026200000001020888850202020050707060000A1
:1026300080F088F080808005070706000070889091
:10264000A09088B0050808060000402000700878B7
:10265000887805080806000010200070087888783F
:1026600005080806000020500070087888780508E2
:1026700008060000285000700878887805070706CB
:1026800000005000700878887805080806000020CF
:102690005020700878887806050506000078147CBC
:1026A000907C0507070600FE708880887020400532
:1026B00008080600004020007088F88070050808AF
:1026C0000600001020007088F880700508080600D9
:1026D000002050007088F880700507070600005041
:1026E000007088F88070030808060100804000C070
:1026F000404040E0030808060100408000C0404020
:1027000040E003080806010040A000C0404040E04F
:10271000060A0A0600FEA4A800FC8480808084FCCF
:10272000060A0A0600FE549400FC8404040484FC97
:10273000050808060000285000B0C88888880508E9
:10274000080600004020007088888870040A0A0685
:1027500002FE30408090909090909090040A0A067B
:1027600000FEC02010909090909090900607070671
:102770000001448C8C8480403C06070706000188D9
:10278000C4C4840408F00505050600012000F80013
:102790002005080806000040F0C8888898781005D1
:1027A0000808060000E0F88888888888F80505058C
:1027B0000600012030F830200508080600002070CF
:1027C000F820202020E00509090600FF2070A8A8B5
:1027D000B8888850200509090600FFE080C0B0A82D
:1027E000A83028280509090600FFF8A888888888E5
:1027F00088A8F8050A0A0600FE205050505088A804
:10280000A888700000000000000000000000007FA9
:10281000FFE0000000000000000000000000700069
:10282000E0000000000000000000000000630C60F9
:10283000000000000000000000000000470E200023
:1028400000000000000000000000004F0F2000000A
:10285000000000000000000000005F0FA00000006A
:102860000000000000000000005E07A07F80003F25
:10287000C0003FC000410400406020FBC00079E080
:102880000079E00020820040F020F3C00076E000F4
:1028900076E00020820040F020EBC0007EE0007E69
:1028A000E0004104004060207B80003DC00039C052
:1028B000008208005E07A07B80003BC0003EC00194
:1028C0000410005F0FA0FBC00077E00076E0010479
:1028D00010004F0F20FBC00070E00079E00082087C
:1028E00000470E20FFC0007FE0007FE000410400B1
:1028F000630C603F00001F80001F8000000000701C
:1029000000E01E00000F00000F0001FFFF807FFFAE
:10291000E00C0000060000060001FFFF8000000040
:102920000000000000000000000000007FFFE00049
:1029300000000000000000000000007000E0000047
:102940000000000000000000000061F860000000CE
:1029500000000000000000000041F820000000001E
:10296000000000000000000040F020000000000017
:102970000000000000000040602000000000000097
:102980000000000000005801A07F80003FC0003F11
:10299000C0004104005C63A0FBC00079E00079E066
:1029A000002082005EF7A0F3C00076E00076E00031
:1029B0002082005EF7A0EBC0007EE0007EE00041D8
:1029C00004005C63A07B80003DC00039C000820829
:1029D000005801A07B80003BC0003EC001041000F5
:1029E000406020FBC00077E00076E001041000406A
:1029F000F020FBC00070E00079E00082080041F8A0
:102A000020FFC0007FE0007FE00041040061F8602B
:102A10003F00001F80001F80000000007000E01ECB
:102A200000000F00000F0001FFFF807FFFE00C009F
:102A300000060000060001FFFF800000005900B002
:102A40002000B02000B02000B02000B02000B02056
:102A5000002D2D3A2D2D004E6F20436172640050E1
:102A600072696E742066726F6D2053440053746FE8
:102A700070205072696E7400526573756D652050D8
:102A800072696E74005061757365205072696E745E
:102A900000436F6E66696775726174696F6E00548A
:102AA000656D7065726174757265004D6F76656DE8
:102AB000656E740054756E6500496E666F207363B1
:102AC0007265656E00F92E2E004D61696E004D3203
:102AD00034004D3233202573004D383420582059AE
:102AE000205A204500526573746F726520466169F3
:102AF0006C73616665004C6F6164206D656D6F720B
:102B0000790053746F7265206D656D6F7279004145
:102B10006476616E6365642053657474696E67736F
:102B2000004D61696E004531737470732F6D6D00D7
:102B30004531737470732F6D6D00457374657073D8
:102B40002F6D6D004573746570732F6D6D005A7332
:102B5000746570732F6D6D005A73746570732F6D8B
:102B60006D005973746570732F6D6D0059737465C2
:102B700070732F6D6D005873746570732F6D6D00D9
:102B80005873746570732F6D6D00412D726574728A
:102B900061637400412D7265747261637400416DEC
:102BA0006178206500416D6178206500416D617834
:102BB000207A00416D6178207A00416D617820793A
:102BC00000416D6178207900416D61782078004185
:102BD0006D61782078005654726176206D696E00C0
:102BE0005654726176206D696E00566D696E00569E
:102BF0006D696E00566D6178206500566D617820B4
:102C00006500566D6178207A00566D6178207A00F3
:102C1000566D6178207900566D6178207900566D87
:102C20006178207800566D617820780056652D6AAD
:102C300065726B0056652D6A65726B00567A2D6A57
:102C400065726B00567A2D6A65726B005678792D25
:102C50006A65726B005678792D6A65726B00416304
:102C600063656C00416363656C005A204F66667350
:102C70006574005A204F666673657400436F6E6614
:102C8000696775726174696F6E00436F6F6C646F12
:102C9000776E005056412F504C4100504C412F5000
:102CA0004C4100484950532F48495053004142532A
:102CB0002F48495053004142532F4142530043751E
:102CC00073746F6D2054656D70004D61696E0050B6
:102CD000564120436F6E660041425320436F6E663B
:102CE000004849505320436F6E6600504C412043CA
:102CF0006F6E66005049442D43005049442D4300F7
:102D00005049442D44005049442D44005049442D1D
:102D100049005049442D49005049442D5000504924
:102D2000442D50002002204661637400200220469A
:102D3000616374002002204D6178002002204D6103
:102D400078002002204D696E002002204D696E003F
:102D50004F6666004F6E20004F6666004F6E200083
:102D60004175746F74656D700046616E2073706597
:102D700065640046616E2073706565640042656439
:102D800000426564004E6F7A7A6C6532004E6F7A4D
:102D90007A6C6532004E6F7A7A6C65004E6F7A7A83
:102DA0006C650054656D7065726174757265005371
:102DB000746F7265206D656D6F7279004265640095
:102DC000426564004E6F7A7A6C65004E6F7A7A6C59
:102DD000650046616E2073706565640046616E2013
:102DE000737065656400437573746F6D2054656D11
:102DF000700053746F7265206D656D6F727900425B
:102E0000656400426564004E6F7A7A6C65004E6FAF
:102E10007A7A6C650046616E207370656564004661
:102E2000616E20737065656400437573746F6D2007
:102E300054656D700053746F7265206D656D6F72AF
:102E4000790042656400426564004E6F7A7A6C6571
:102E5000004E6F7A7A6C650046616E20737065650E
:102E6000640046616E207370656564004375737419
:102E70006F6D2054656D700053746F7265206D65C1
:102E80006D6F72790042656400426564004E6F7A2E
:102E90007A6C65004E6F7A7A6C650046616E2073BD
:102EA000706565640046616E2073706565640043FB
:102EB0007573746F6D2054656D70004D6F7665206D
:102EC0004178697300473238004175746F20486F4C
:102ED0006D65004D38340044697361626C65205340
:102EE00074657070657273004D61696E004D6F7628
:102EF0006520302E316D6D004D6F766520316D6D22
:102F0000004D6F76652031306D6D004D6F76656DCB
:102F1000656E74004578747275646572004D6F76E5
:102F200065205A004D6F76652059004D6F766520FB
:102F300058004D6F7665204178697300457874724A
:102F400075646572005A00590058004D36303000E3
:102F50004368616E67652066696C616D656E7400BB
:102F6000466C6F7700466C6F770046616E20737019
:102F70006565640046616E20737065656400426536
:102F80006400426564004E6F7A7A6C6532004E6F61
:102F90007A7A6C6532004E6F7A7A6C65004E6F7A81
:102FA0007A6C6500537065656400537065656400F4
:102FB0004D61696E00436172642072656D6F766564
:102FC00064004361726420696E73657274656400A5
:102FD00000000000000000000000000000000000F1
:102FE00000000000000000000000000000000000E1
:102FF0000000000C000000000000000C00000000B9
:10300000000000120000000000000023000000008B
:1030100000000021000000000000004C80000000C3
:103020000000005E800000000000009240000000F0
:10303000000000A14000000000000121200000006D
:103040000000027F9000000000000200100000005D
:10305000000007FFF8000000000004000800000066
:103060000000080004000000000008000600000046
:1030700000001000020000000000301E01000000EF
:103080000000207F81000000000041FFE080000080
:10309000000043FCF08000000000873B7840000007
:1030A00000018EDBFC60000000010FEBCC20000073
:1030B00000021FEDB610000000021FDEB610000077
:1030C000000439CD7F080000000436E0FF0800004E
:1030D00000087EC0BB84000000187F005D860000F1
:1030E00000107FC0ED82000000203CC07301000092
:1030F00000203B337F01000000701BE77E0380004F
:1031000000C81DEEDE04C00000880FDEDC044000B5
:1031100001240FDF3C092000012607DBF8192000FD
:10312000027203E7F0139000025101FFE0229000C9
:103130000489007F802448000904801E0048240080
:103140000BFE400000DFF400100040000080020091
:103150001FFFFFFFFFFFFE00000000000000000057
:10316000000000000000000000000000000000005F
:103170001022103C3C0E1F001022100422110400EB
:103180001022100822110400102210083C11040023
:10319000102210102211040010221020221104000D
:1031A0001E1C1E3C3C0E040000000000000000003D
:1031B000000000000000000000000000000000000F
:1031C00000000000000000000000000000000000FF
:1031D00000000000000000000000000000000000EF
:1031E00000000000000000000000000000000000DF
:1031F00000000000000000000000000000000000CF
:1032000000000000000000000000000000006563F6
:10321000686F3A0048617264636F64656420446556
:103220006661756C742053657474696E6773204CA5
:103230006F616465640053746F72656420736574B4
:1032400074696E677320726574726965766564006F
:103250002044002049002020204D333031205000F0
:103260005049442073657474696E67733A00205A3C
:103270000020590020204D323036205800486F6D14
:1032800065206F666673657420286D6D293A00208D
:103290004500205A002058002042002054002020E1
:1032A0004D323035205300416476616E6365642091
:1032B0007661726961626C65733A20533D4D696E47
:1032C00020666565647261746520286D6D2F7329B1
:1032D0002C20543D4D696E2074726176656C2066B9
:1032E0006565647261746520286D6D2F73292C20CB
:1032F000423D6D696E696D756D207365676D656EB4
:10330000742074696D6520286D73292C20583D6DDB
:103310006178696D756D205859206A65726B202837
:103320006D6D2F73292C20205A3D6D6178696D7564
:103330006D205A206A65726B20286D6D2F73292CC1
:103340002020453D6D6178696D756D2045206A6569
:10335000726B20286D6D2F73290020540020204DA2
:10336000323034205300416363656C657261746967
:103370006F6E3A20533D616363656C657261746979
:103380006F6E2C20543D72657472616374206163AA
:1033900063656C65726174696F6E00204500205A28
:1033A0000020590020204D3230312058004D6178E6
:1033B000696D756D20416363656C65726174696FD9
:1033C0006E20286D6D2F7332293A00204500205A57
:1033D0000020590020204D3230332058004D6178B4
:1033E000696D756D2066656564726174657320280A
:1033F0006D6D2F73293A0020453100204500205A79
:103400000020590020204D39322058005374657037
:10341000732070657220756E69743A005365747418
:10342000696E67732053746F72656400010508004C
:10343000FF060121023520FFFF07FF06FF090050AC
:10344000221656808080800080153353A0A0A002F1
:1034500057575050F850F850500257572070A070EE
:1034600028702013355580A040A02002475740A067
:10347000A040A0A050251353808080122656408083
:103480008080804012265680404040408002455552
:103490009060F060900255552020F82020113353A1
:1034A000604080044151F011335340E040024656E1
:1034B00010102040808012365640A0A0A0A04012DC
:1034C000365640C0404040E0024656609010608052
:1034D000F0024656F020601090600246562060A030
:1034E000F02020024656F080E010906002465660C0
:1034F00080E0909060024656F01020204040024646
:103500005660906090906002465660909070106097
:10351000122555C0C000C0C0113656606000604022
:1035200080123656204080804020034353F000F044
:1035300012365680402020408012365640A020404F
:103540000040015858304898A8A89040300246568C
:10355000609090F09090024656E090E09090E002EB
:103560004656609080809060024656E09090909021
:10357000E0024656F080E08080F0024656F080E09F
:10358000808080024656609080B0906002465690DF
:1035900090F0909090123656E040404040E0024655
:1035A0005670202020A04002465690A0C0A0A090B7
:1035B0000246568080808080F002465690F0F0905F
:1035C000909002465690D0F0B0B09002465660906F
:1035D00090909060024656E09090E08080014757BE
:1035E000609090D0B06010024656E09090E09090CD
:1035F000024656609040209060123656E0404040AF
:1036000040400246569090909090600246569090AE
:1036100090906060024656909090F0F0900246566E
:10362000909060609090025656888850202020022A
:103630004656F010204080F0123656E080808080A0
:10364000E0024656808040201010123656E02020BE
:103650002020E016325240A0014151F01622528043
:1036600040024454709090700246568080E09090E2
:10367000E0123454608080600246561010709090C2
:103680007002445460B0C060024656205040E04092
:103690004001455560907010600246568080E09071
:1036A00090901236564000C04040E011375720003D
:1036B000202020A040024656808090E09090123654
:1036C00056C040404040E0025454D0A8A8A802444C
:1036D00054E090909002445460909060014555E011
:1036E00090E080800145557090701010024454A005
:1036F000D0808012345460C020C00246564040E062
:1037000040502002445490909070123454A0A0A0D5
:103710004002545488A8A85002445490606090011C
:1037200045559090709060024454F02040F002475C
:1037300057304020C0204030221656808080808044
:1037400080024757C02040304020C006425250A05F
:10375000FFFFFFFFFFFFFFFFFFFFFFFFFFFFFFFF79
:10376000FFFFFFFFFFFFFFFFFFFFFFFFFFFFFFFF69
:10377000FF09005022165680008080808001465646
:103780002070A0A070200246562050E04050A002B9
:10379000555588705070880256568850F820F82089
:1037A000221757808080008080800247577080E019
:1037B000907010E0173151A002565670A8C8C8A8E2
:1037C0007014355560A06000E003435350A05012C0
:1037D0003353E02020143151E002565670E8D8E807
:1037E000D870173151E015335340A0401235554081
:1037F000E04000E014355540A02040E0143555C0AD
:1038000020C020C01622524080014555909090E083
:103810008002565678E8E868282824115180112241
:1038200052408014355540C04040E014355540A00A
:103830004000E0034353A050A0024757808080A07F
:1038400060F0200247578080A0D0102070024757B8
:1038500080408060A0F02012365640004080A0409A
:1038600002475740206090F09090024757204060F8
:1038700090F0909002475760906090F090900247CF
:103880005750A06090F0909002475790006090F0E1
:10389000909002475760906090F09090024656706A
:1038A000A0A0F0A0B00147576090808090604002D7
:1038B00047574020F080E080F00247572040F080DA
:1038C000E080F00247576090F080E080F0024757B8
:1038D0009000F080E080F01237578040E040404098
:1038E000E01237572040E0404040E012375740A0F8
:1038F000E0404040E0123757A000E0404040E00286
:1039000056567048E848487002475750A090D0B0CB
:103910009090024757402060909090600247572057
:1039200040609090906002475760906090909060E7
:1039300002475750A06090909060024757900060F7
:1039400090909060123353A040A002465670B0B0E1
:10395000D0D0E002475740209090909060024757A7
:103960002040909090906002475760909090909087
:103970006002475790009090909060025757102037
:10398000885020202002465680E09090E080024639
:10399000566090A0A090A0024757402000709090E1
:1039A0007002475720400070909070024757205097
:1039B000007090907002475750A000709090700275
:1039C000465650007090907002475760906070901B
:1039D0009070025454F068B0781135556080806062
:1039E0004002475740200060B0C060024757204067
:1039F0000060B0C06002475760900060B0C06002D5
:103A00004656500060B0C060123757804000C0403A
:103A100040E0123757204000C04040E01237574086
:103A2000A000C04040E0123656A000C04040E00276
:103A30004757A040A01070906002475750A000E088
:103A40009090900247574020006090906002475746
:103A50002040006090906002475760900060909016
:103A60006002475750A00060909060024656900058
:103A7000609090601235554000E000400244547060
:103A8000B0D0E00247574020009090907002475716
:103A90002040009090907002475760900090909066
:103AA0007002465690009090907001485820400057
:103AB00090907090600147578080E090E080800196
:103AC00047579000909070906000002100240027DC
:103AD000002A002D0030003300010100000401071E
:103AE000010A0100002200250028002B002E0031D1
:103AF00000340002010000050108010B0100002054
:103B0000002300260029002C002F003200000100B5
:103B10000003010601090105050505070508080858
:103B200008020202020A0A0808040404040101014E
:103B30000101010101030303030303030304070756
:103B4000070C0C0C0C0C0C0C0C02020202060606F4
:103B500006060606060B0B0B0B0B0B0B0B07070AD7
:103B60000A0A0A0A0A0505050401021020200808AD
:103B700010204010204080020102010804020101CF
:103B800002040810204080804020100804020180B8
:103B9000040201804020100804020108040201010F
:103BA0000204081020408001020408102040801008
:103BB00008040880102040044080100000090A0218
:103BC000080B0C0D070603040100000000000000B4
:103BD00000000000000000000000000000000000E5
:103BE0000000000000000011100F000000000000A5
:103BF00000000000000000000000000000000000C5
:103C00000002494E46494E4954594E414ECDCCCC06
:103C10003D0AD7233C17B7D13877CC2B329595E6A0
:103C2000241FB14F0A000020410000C84200401C80
:103C30004620BCBE4CCA1B0E5AAEC59D7400A724BC
:103C4000FF34EDDFC9F1FA3411241FBECFEFD1E20A
:103C5000DEBFCDBF00E00CBF14E0A0E0B2E0EAECB4
:103C6000FCE002E00BBF02C007900D92A03DB1073F
:103C7000D9F71BBE16E1A0EDB4E001C01D92AB3236
:103C8000B107E1F71CE3C6E4DCE304C02297FE01C0
:103C90000F940B06CE33D107C9F70E9457FD0D9440
:103CA00059060C940000A0E0B0E0E9E5FEE10D94B7
:103CB0002806EC015B016115710519F0FB01918388
:103CC0008083F9908F2D90E00F940F06892BC9F710
:103CD000FDE2FF1621F4F990EE24E39405C02BE2F7
:103CE000F21609F4F990EE248E0101501040C8013B
:103CF00062E07CE343E050E072D2892BF9F48E015C
:103D00000E5F1F4FC80165E07CE345E050E067D2DD
:103D1000892B19F48E01095F1F4FA114B10419F00A
:103D2000F50111830083E0FC04C070E090E080E8BE
:103D300013C070E090E080E86FEF07C1C8016AE04F
:103D40007CE343E050E04BD2892B69F4A114B10429
:103D500029F470E090E080EC6FE7F7C02296F5015F
:103D6000D183C083F6CF8824992440E050E060E0FE
:103D700070E0EF2DE053EA30A0F5F2E0EF2A8E2D4F
:103D800090E09C0128703070E2FE06C0232B79F58C
:103D90000894811C911C2BC0232B19F008948108D6
:103DA0009108DB01CA0112E0880F991FAA1FBB1FEF
:103DB0001A95D1F7480F591F6A1F7B1F440F551FD3
:103DC000661F771F4E0F511D611D711D483929E96E
:103DD000520729E9620729E1720748F084E0E82ADE
:103DE00006C0EE3F31F4E3FC39C098E0E92AF990CF
:103DF000C0CFE53311F0E53189F529912D3219F461
:103E0000E0E1EE2A05C02B3219F081E090E003C01A
:103E1000299182E090E0E22FE053EA3018F0C81BCD
:103E2000D90B1CC020E030E0FCE020383F075CF4F8
:103E3000C901880F991F880F991F280F391F220F5A
:103E4000331F2E0F311DE991E053EA3068F3E4FE91
:103E500003C0309521953F4F820E931ECE2CDD245A
:103E6000E1FE07C0A114B10421F02197F501D1832F
:103E7000C083CB01BA010F9474027B018C01F3E083
:103E8000CF22DD2423E0C216D10421F417FB1095C4
:103E900017F9109557016801C801B70120E030E01B
:103EA00040E050E00F94D401882309F44AC097FE03
:103EB0000DC021E2E22E2CE3F22E90948194910821
:103EC0009394C0E2D0E000E010E012C099E3E92E44
:103ED0009CE3F92EF6CFF701259135914591549148
:103EE000C601B5010F94B4045B016C018C1A9D0AE4
:103EF0008C169D0684F7D595C7950F5F1F4F06302A
:103F0000110529F08CEF9FEFE80EF91EF1CFC501E6
:103F1000D6017C018D018C2D880F8D2D881F8F3F40
:103F200051F0C601B50120E030E040E050E00F94D0
:103F3000D401882331F482E290E090932A16809392
:103F400029167E2D9F2D802F612F272F392F482F47
:103F5000562FB901CA01CDB7DEB7ECE00D94440687
:103F60002F923F925F926F927F928F929F92AF9229
:103F7000BF92CF92DF92EF92FF920F931F93CF9356
:103F8000DF938C011B01EA016115710519F0FB013A
:103F900091838083209749F0CE010297839728F080
:103FA00020E030E040E050E0F6C0F801A1908F0141
:103FB0008A2D90E00F940F06892BB9F7FDE2AF161A
:103FC00031F4F801A1908F015524539407C0FBE20E
:103FD000AF1619F4F801A1908F015524209719F01C
:103FE000C031D105C1F4F0E3AF1679F4F801808156
:103FF000883711F0883549F4F801A1800E5F1F4F12
:10400000F2E05F2AC0E1D0E006C0209721F480E30F
:10401000A816E9F427C0C830D10531F1C930D1055F
:1040200024F4C230D10531F50CC0CA30D10589F075
:10403000C031D105F9F4C12CD12CE12CB8E0FB2E14
:1040400028C0C12CD12CE12CA0E4FA2E22C0CAE059
:10405000D0E0FCECCF2EFCECDF2EFCECEF2EFCE0F5
:10406000FF2E17C0C8E0D0E0C12CD12CE12CE0E13C
:10407000FE2E0FC09E01442737FD4095542F60E06F
:1040800070E080E090E80F94CC05C901DA016C0182
:104090007D0120E030E040E050E060E03E01882417
:1040A00077FC8094982C70EDB72EBA0CE9E0EB15F4
:1040B00070F48A2D81548A3118F499ECB92E06C017
:1040C0008A2D81568A3150F589EAB82EBA0C8B2D8B
:1040D00090E08C179D0714F56F3FE1F0C216D306F0
:1040E000E406F506B0F0CA01B901A40193010F94EA
:1040F00086059B01AC012B0D311D411D511D213049
:10410000F0E03F07F0E04F07F0E85F0710F461E0F0
:1041100001C06FEFF801A1908F01C5CF21143104C8
:1041200081F0662331F001501040F10111830083CA
:1041300008C051FE1AC002501040F10111830083E3
:1041400014C067FF12C050FC05C02FEF3FEF4FEFC8
:104150005FE704C020E030E040E050E882E290E019
:1041600090932A168093291616C050FE08C05095C9
:104170004095309521953F4F4F4F5F4F0CC057FFF3
:104180000AC082E290E090932A16809329162FEFBE
:104190003FEF4FEF5FE7B901CA01DF91CF911F9168
:1041A0000F91FF90EF90DF90CF90BF90AF909F90D6
:1041B0008F907F906F905F903F902F900895FB01BC
:1041C000DC0105900D920020E1F70895FC010590B7
:1041D0000020E9F7809590958E0F9F1F0895FB01B1
:1041E000DC014150504088F08D9181341CF08B35BA
:1041F0000CF4805E659161341CF06B350CF4605EEC
:10420000861B611171F3990B0895881BFCCFFB018C
:10421000DC014150504048F005900D920020C9F754
:1042200001C01D9241505040E0F70895FB015591A7
:104230005523A9F0BF01DC014D9145174111E1F76C
:1042400059F4CD010590002049F04D9140154111E0
:10425000C9F3FB014111EFCF81E090E00197089590
:10426000FB01DC0104C08D910190801921F44150C3
:104270005040C8F7881B990B0895FB01DC0102C070
:1042800001900D9241505040D8F70895FB01DC0198
:104290000D900020E9F7119701900D920020E1F7B1
:1042A0000895FC018191861721F08823D9F7992779
:1042B00008953197CF010895FB01DC0101900D9223
:1042C0000020E1F70895FB01DC014150504030F03F
:1042D0008D910190801919F40020B9F7881B990B72
:1042E0000895FB01DC014150504048F001900D92CF
:1042F0000020C9F701C01D9241505040E0F70895D9
:10430000AEE0B0E0E6E8F1E20D9430060E891F89D8
:104310008EE08C831A8309838FEF9FE79E838D83C2
:104320009E01265E3F4FCE010196688D798DA901D1
:104330000AD02F813885020F131FF80110822E96A4
:10434000E4E00D944C06ABE0B0E0E9EAF1E20D9454
:1043500022063C012B015A01FC011782168283813F
:1043600081FD03C06FEF7FEFB9C19AE0892E1E0176
:104370000894211C311CF3012381F20123FD859156
:1043800023FF81912F01882309F4A5C1853239F4D7
:1043900023FD859123FF81912F01853221F490E047
:1043A000B301B7D1E8CF982FFF24EE249924FFE181
:1043B000FF15D0F09B3269F09C3228F4903259F00E
:1043C000933291F40EC09D3249F0903369F441E08C
:1043D00024C052E0F52A84E0F82A28C098E0F92A9F
:1043E00025C0E0E1FE2A22C0F7FC29C0892F8053B6
:1043F0008A3070F4F6FE05C0989C902C1124980E1B
:1044000015C0E89CE02C1124E80EF0E2FF2A0EC053
:104410009E3229F4F6FC5FC140E4F42A07C09C36C2
:1044200019F450E8F52A02C0983649F4F20123FD48
:10443000959123FF91912F01992309F0B8CF892FEE
:104440008554833018F08052833038F444E050E0D3
:10445000A40EB51E5FE359830FC0933631F0933736
:1044600079F0933509F052C01FC0F501808189832E
:1044700042E050E0A40EB51E610101E010E011C061
:10448000F501C080D180F6FC03C06FEF7FEF02C062
:10449000692D70E042E050E0A40EB51EC6012ED199
:1044A0008C015FE7F52213C0F501C080D180F6FCD6
:1044B00003C06FEF7FEF02C0692D70E042E050E073
:1044C000A40EB51EC6010FD18C0150E8F52AF3FEEB
:1044D00006C018C080E290E0B3011BD1EA948E2D93
:1044E00090E008171907B0F30DC0F601F7FC8591AD
:1044F000F7FE81916F0190E0B3010BD1E110EA94D6
:10450000015010400115110581F7E2C0943611F0F9
:10451000993661F5F7FE08C0F501208131814281AD
:10452000538184E090E00AC0F501808191819C0173
:10453000442737FD4095542F82E090E0A80EB91E25
:104540009FE6F92257FF09C0509540953095219577
:104550003F4F4F4F5F4FE0E8FE2ACA01B901A1016A
:104560002AE030E002D1D82ED2183FC0953729F486
:104570001F2D1F7E2AE030E01DC01F2D197F9F36A2
:1045800061F0903720F4983509F0A5C00FC090373E
:1045900039F0983709F09FC004C028E030E00AC025
:1045A000106114FD146020E130E004C014FD1660B9
:1045B00020E132E017FF08C0F5016081718182813E
:1045C000938144E050E008C0F50180819181BC01F5
:1045D00080E090E042E050E0A40EB51EA101C5D0FD
:1045E000D82ED2188FE7F82EF122F6FE0BC05EEF20
:1045F000F522D91438F4F4FE07C0F2FC05C08FEEA2
:10460000F82202C01D2D01C0192DF4FE0DC0FE01BF
:10461000ED0DF11D8081803319F499EEF92208C067
:104620001F5FF2FE05C003C08F2D867809F01F5F63
:104630000F2DF3FC13C0F0FE0EC01E1510F09D2CC4
:104640000AC09D2C9E0C911A1E2D05C080E290E0A0
:10465000B3015FD01F5F1E15C8F304C01E1510F410
:10466000E11A01C0EE2404FF0EC080E390E0B30124
:1046700050D002FF1BC001FD03C088E790E00EC0D0
:1046800088E590E00BC0802F867881F001FF02C0A2
:104690008BE201C080E2F7FC8DE290E0B30139D0FB
:1046A00005C080E390E0B30134D09A94D914C8F3E4
:1046B000DA94F101ED0DF11D808190E0B30129D074
:1046C000DD20B1F705C080E290E0B30122D0EA948A
:1046D000EE20C9F750CEF30166817781CB012B968E
:1046E000E2E10D943E06FC0105906150704001101E
:1046F000D8F7809590958E0F9F1F0895FC0161500B
:10470000704001900110D8F7809590958E0F9F1FF3
:1047100008950F931F93CF93DF938C01EB018B814F
:1047200081FF1BC082FF0DC02E813F818C819D8146
:104730002817390764F4E881F9810193F983E88344
:1047400006C0E885F985802F1995892B31F48E8173
:104750009F8101969F838E8302C00FEF1FEFC801D8
:10476000DF91CF911F910F910895FA01AA27283068
:1047700051F1203181F1E8946F936E7F6E5F7F4F2E
:104780008F4F9F4FAF4FB1E03ED0B4E03CD0670FAA
:10479000781F891F9A1FA11D680F791F8A1F911DFD
:1047A000A11D6A0F711D811D911DA11D20D009F44D
:1047B00068943F912AE0269F11243019305D31938F
:1047C000DEF6CF010895462F4770405D4193B3E078
:1047D0000FD0C9F7F6CF462F4F70405D4A3318F01F
:1047E000495D31FD4052419302D0A9F7EACFB4E0D0
:1047F000A6959795879577956795BA95C9F7009788
:104800006105710508959B01AC010A2E0694579528
:10481000479537952795BA95C9F7620F731F841F7F
:10482000951FA01D08951F920F920FB60F920BB601
:104830000F9211242F933F934F938F939F93EF9356
:10484000FF934091C600E0915005F09151053196DB
:104850009F012F77307031978091520590915305C9
:104860002817390739F0E053FB4F40833093510547
:1048700020935005FF91EF919F918F914F913F9120
:104880002F910F900BBE0F900FBE0F901F90189599
:104890009A01AB01203081EE380780E0480780E0C4
:1048A000580749F182E08093C00060E079E08DE331
:1048B00090E00F94EE052150304040405040CA0136
:1048C000B90122E030E040E050E00F94EE05309373
:1048D000C5002093C4008091C10080618093C10015
:1048E0008091C10088608093C1008091C100806880
:1048F0008093C10008951092C00020E130E0E7CF1E
:1049000020915205309153058091500590915105A9
:104910008217930719F42FEF3FEF0EC0F901E05310
:10492000FB4F80812F5F3F4F2F77307030935305BF
:1049300020935205282F30E0C90108958091520537
:1049400090915305909351058093500508950895D3
:104950002F923F924F925F926F927F928F929F928F
:10496000AF92BF92CF92DF92EF92FF920F931F937D
:10497000DF93CF93CDB7DEB7A0970FB6F894DEBF25
:104980000FBECDBF1C016A017B01411551056105B8
:10499000710541F440E350E060E070E020E030E079
:1049A0008BD055C0882499245401422E5524662466
:1049B000772401E010E00C0F1D1F080D191DC70121
:1049C000B601A30192010F94CC05F801608308940D
:1049D000811C911CA11CB11CC701B601A30192014D
:1049E0000F94CC05C901DA016C017D01C114D10419
:1049F000E104F104F1F681E0E82EF12CEC0EFD1E4D
:104A0000E80CF91C3E010894611C711CD501C4011D
:104A10000197A109B1096C01C818D90815C0F601A0
:104A2000EE0DFF1D40814A3010F4405D01C0495C2D
:104A3000552747FD5095652F752FC10120E030E0C7
:104A40003BD00894E108F1086E147F0441F7A0966A
:104A50000FB6F894DEBF0FBECDBFCF91DF911F918F
:104A60000F91FF90EF90DF90CF90BF90AF909F900D
:104A70008F907F906F905F904F903F902F90089510
:104A80002115310539F48091C00085FFFCCF40939A
:104A9000C60008955DCFEF92FF920F931F939A0186
:104AA000E62EFF2400E010E0B801A701E9DF1F9126
:104AB0000F91FF90EF900895EF92FF920F931F9345
:104AC000CF93DF93EC017A018B012115310539F485
:104AD0008091C00085FFFCCFE092C60019C02A304B
:104AE0003105A9F477FF0FC04DE250E060E070E0BF
:104AF00020E030E0E1DF10950095F094E094E11CB7
:104B0000F11C011D111DCE01B801A7012AE020DF13
:104B1000DF91CF911F910F91FF90EF900895EF9249
:104B2000FF920F931F937B019A010027F7FC0095DA
:104B3000102FB801A701C0DF1F910F91FF90EF90D8
:104B400008950F931F938C014DE050E060E070E0FA
:104B500020E030E0B1DFC8014AE050E060E070E002
:104B600020E030E0A9DF1F910F910895CF92DF92EE
:104B7000EF92FF920F931F938C019A016B01EE2429
:104B8000FF24B701A6017CDFC801DBDF1F910F9175
:104B9000FF90EF90DF90CF9008959F92AF92BF92D9
:104BA000CF92DF92EF92FF920F931F93CF93DF93F9
:104BB000EC017A018B01922ECB01BA0120E030E0AA
:104BC00040E050E00F94D401882364F4CE014DE21C
:104BD00050E060E070E020E030E06EDF17FB109501
:104BE00017F9109520E030E040E05FE3AA240BC005
:104BF000CA01B90120E030E040E251E40F94DB014A
:104C00009B01AC01A394A91498F3C801B7010F94B8
:104C1000FB007B018C010F9448025B016C010F9437
:104C200074029B01AC01C801B7010F94FA007B012B
:104C30008C01CE01B601A5012AE030E021DF9920E8
:104C400099F1E0E0F2E007C08091C00085FFFCCF61
:104C500031969093C60090819923B1F725C0C80181
:104C6000B70120E030E040E251E40F94B4047B014E
:104C70008C010F9443025B016C01CC24B7FCC094FF
:104C8000DC2CCE01B601A5012AE030E015DFC6011B
:104C9000B5010F9476029B01AC01C801B7010F94D6
:104CA000FA007B018C019A949920C9F6DF91CF918B
:104CB0001F910F91FF90EF90DF90CF90BF90AF903A
:104CC0009F9008956ACF0895FC011282138208957F
:104CD000FC018381882311F081E082830895FC0127
:104CE0008281811112820895CF93DF93DC01FC0150
:104CF000EB55FE4F808191810097C9F10197918317
:104D00008083ED01CC5ADF4FFD01ED58FF4F8BE161
:104D1000019009928150E1F7FD01EE5AFF4FAF5823
:104D2000BF4F8D919C911197A157B0409183808383
:104D3000FD01ED58FF4F20E030E0AD014B555E4FD7
:104D400010C02F5F3F4FEF01DF015F968BE10D90A9
:104D500009928150E1F7858D968D329791838083FA
:104D6000B196DA018D919C912817390750F3DF91A4
:104D7000CF910895FC018BE794E091838083878134
:104D8000882321F0CF0104960C9425810895CF92B9
:104D9000DF92EF92FF920F931F93DF93CF93CDB7E4
:104DA000DEB76F970FB6F894DEBF0FBECDBF8C0194
:104DB0006B01095A1F4FD8018C9107551040882369
:104DC00021F42FE2E22EF12C03C090E5E92EF12C24
:104DD000E00EF11E8BE794E09A8389831C821B828C
:104DE00018861D82B7016C5F7F4FCE010596A60124
:104DF00021E00E941288882391F5EBE3F1E0949181
:104E000008C08091C00085FFFCCF9093C60031960A
:104E100094919923B1F7E1E4F1E0949108C0809175
:104E2000C00085FFFCCF9093C600319694919923E2
:104E3000B1F709C08091C00085FFFCCF0894C11C68
:104E4000D11C9093C600F6019081992399F7809127
:104E5000C00085FFFCCF8AE08093C6005AC0F801ED
:104E6000EB55FE4F208131812A30310508F040C0DA
:104E70002F5F3F4F3183208321503040F90185E07F
:104E8000EE0FFF1F8A95E1F7E21BF30BED58FF4F82
:104E9000E00FF11F13C0AF01415E5F4FBF018BE117
:104EA000DB010D90BD01DA010D92AD018150C1F71A
:104EB000929182913296968F858F7F9721503040C4
:104EC000BFEF2E3F3B0739F7D801AD58BF4FF70171
:104ED00034968BE101900D928150E1F70F581F4FEE
:104EE000F70182819381D8018D939C9301571040E3
:104EF000D801AC5ABF4FFE0135968BE101900D925F
:104F00008150E1F70E5A1F4F8B819C81F8019183EC
:104F10008083CE0101962EDF6F960FB6F894DEBF28
:104F20000FBECDBFCF91DF911F910F91FF90EF90FA
:104F3000DF90CF900895EF92FF920F931F938C0113
:104F40003EECE32E31E0F32EE80EF91EC7010E947D
:104F5000D980C7010E942581F801108211821F911A
:104F60000F91FF90EF900895CF92DF92EF92FF9212
:104F70000F931F93CF93DF937C016B01DB010D90A7
:104F80000020E9F78D0101501040061B170BEEECD5
:104F9000F1E0EE0EFF1ED7011C92E2E3FEEFEE0EF3
:104FA000FF1ECB016EE470E07CD9EC01009731F478
:104FB000F8013197EC0DFD1D86010CC060E270E038
:104FC00070D98C010F5F1F4FCE016AE270E069D982
:104FD000FC0131978DE081838AE082831382C701CF
:104FE00086539E4FB8010E94877F8EEC91E0E80EB9
:104FF000F91ED7018C91882319F1EBE6F1E0949129
:1050000008C08091C00085FFFCCF9093C600319608
:1050100094919923B1F7E2E7F1E0949108C080916F
:10502000C00085FFFCCF9093C600319694919923E0
:10503000B1F78091C00085FFFCCF8AE08093C60065
:10504000DF91CF911F910F91FF90EF90DF90CF9064
:105050000895CF93DF93EC018B81882309F439C045
:10506000EAE9F1E0949108C08091C00085FFFCCF8F
:105070009093C600319694919923B1F7CD57DD4FA7
:10508000488159816A817B81C358D24084E595E08B
:105090002AE030E0F5DCE8E9F1E0949108C0809185
:1050A000C00085FFFCCF9093C60031969491992360
:1050B000B1F7C558DD4F488159816A817B8184E50C
:1050C00095E02AE030E0DCDC8091C00085FFFCCF79
:1050D00012C0E8E8F1E0949108C08091C00085FF1B
:1050E000FCCF9093C600319694919923B1F78091AB
:1050F000C00085FFFCCF8AE08093C600DF91CF918E
:1051000008952F923F924F925F926F927F928F926B
:105110009F92AF92BF92CF92DF92EF92FF920F9346
:105120001F93DF93CF93CDB7DEB7AC970FB6F8944C
:10513000DEBF0FBECDBF5C014B01FC018381882324
:1051400009F434C1C50182539E4F0E942581F501A7
:1051500012821A8A1D8A198A188A8BE794E09F871F
:105160008E875EE4C52ED12CCA0CDB1C2FE230E00A
:10517000A20EB31EF601B182A08221ED3FEFA20E76
:10518000B31EF40180818F3209F08DC0C4016FE23B
:1051900070E087D87C010894E11CF11C3E01089462
:1051A000611C711C260142E1242E312C2C0E3D1E67
:1051B00075C0C7016FE270E074D86C01009709F404
:1051C00080C0E816F90608F07CC08C010E191F0992
:1051D000C301B701A80185D8060D171DF80110827B
:1051E000F30107C08091C00085FFFCCF31969093FA
:1051F000C60090819923B1F78091C00085FFFCCF54
:10520000FAE0F093C600F2016081718161157105C9
:1052100019F460E070E002C06C5F7F4FC101A30130
:1052200021E00E941288882371F5E6EDF1E0949167
:1052300008C08091C00085FFFCCF9093C6003196D6
:1052400094919923B1F7FE01319607C08091C00077
:1052500085FFFCCF31969093C60090819923B1F7DA
:10526000E4EDF1E0949108C08091C00085FFFCCF8F
:105270009093C600319694919923B1F78091C00024
:1052800085FFFCCF8DC02EE030E02C0F3D1FF201DA
:105290003183208376010894E11CF11CE114F104B0
:1052A00009F087CF0BC080E590E0A80EB91EF6018B
:1052B000B182A08220EB3FEFA20EB31ED82C092DA5
:1052C00002C0DE2C0F2D8EE490E0A80EB91EF50171
:1052D0008081918122EB3FEFA20EB31E009719F45B
:1052E00080E090E001C004966D2D702F0E94DE8852
:1052F000882339F1E6ECF1E0949108C08091C00078
:1053000085FFFCCF9093C600319694919923B1F715
:105310008D2D902F9C01F90107C08091C00085FF61
:10532000FCCF31969093C60090819923B1F783E822
:1053300092E0A80EB91EF50110821182128213822A
:1053400032C0EEEAF1E0949108C08091C00085FF80
:10535000FCCF9093C600319694919923B1F78D2D8F
:10536000902F9C01F90107C08091C00085FFFCCF00
:1053700031969093C60090819923B1F7ECEAF1E061
:10538000949108C08091C00085FFFCCF9093C60027
:10539000319694919923B1F78091C00085FFFCCF9D
:1053A0008AE08093C600CE010E96E4DCAC960FB680
:1053B000F894DEBF0FBECDBFCF91DF911F910F914B
:1053C000FF90EF90DF90CF90BF90AF909F908F9025
:1053D0007F906F905F904F903F902F900895BF9275
:1053E000CF92DF92EF92FF920F931F93CF93DF93B1
:1053F0008C01EB018FE28993EE24E394FF2475EA9C
:10540000C72E71E0D72EC00ED11E6FE1B62E14C08C
:10541000FB9CC00111248D589F4F800F911FBE012E
:105420000E94358102C02196E3948881882319F077
:105430008CE88E15C0F7F3942F2D30E0F6018081B3
:1054400091812817390720F3E7FC07C0C801825370
:105450009E4FBE010E94358101C01882DF91CF911D
:105460001F910F91FF90EF90DF90CF90BF90089524
:105470002F923F924F925F926F927F928F929F9264
:10548000AF92BF92CF92DF92EF92FF920F931F9352
:10549000DF93CF93CDB7DEB7AD970FB6F894DEBFED
:1054A0000FBECDBF6C014B014DA7DC0113968C9153
:1054B000882309F445C3E1EDF1E0CE0EDF1ED601ED
:1054C0008C91EFE2FEEFCE0EDF1E882309F416C1A9
:1054D000222309F0DEC029EE31E0C20ED31ED60130
:1054E0008C91E7E1FEEFCE0EDF1E882369F1EBE63B
:1054F000F1E0949108C08091C00085FFFCCF9093AB
:10550000C600319694919923B1F7EEEAF2E09491B6
:1055100008C08091C00085FFFCCF9093C6003196F3
:1055200094919923B1F784E595E061E070E04AE059
:1055300050E0F5DA8091C00085FFFCCF8AE08093CF
:10554000C6000E944C35FCC2EBE3F1E0949108C028
:105550008091C00085FFFCCF9093C6003196949156
:105560009923B1F7E5E9F2E0949108C08091C00079
:1055700085FFFCCF9093C600319694919923B1F7A3
:10558000F40107C08091C00085FFFCCF3196909355
:10559000C60090819923B1F7EAE8F2E0949108C03F
:1055A0008091C00085FFFCCF9093C6003196949106
:1055B0009923B1F7C6012EEE31E0C20ED31EB6011B
:1055C0000EDF4BEF5FEFC40ED51ED6019C91E7E1D5
:1055D000FEEFCE0EDF1E8DE8989FF0011124E25100
:1055E000FE4FEC0DFD1D07C08091C00085FFFCCF74
:1055F00031969093C60090819923B1F7E4E8F2E0E8
:10560000949108C08091C00085FFFCCF9093C600A4
:10561000319694919923B1F723E832E0C20ED31E5C
:10562000D6014D915D916D917C91EDE7FDEFCE0E30
:10563000DF1E84E595E02AE030E022DA8091C000A8
:1056400085FFFCCF8AE08093C600A60147515E4FDC
:10565000DA012C91E22FF0E0EE0FFF1FEE0FFF1F9B
:10566000EC0DFD1DE651FE4F83E892E0C80ED91EF9
:10567000D6014D905D906D907C908DE79DEFC80EAA
:10568000D91E40825182628273822F5FDA012C938D
:105690002FC0EBE3F1E0949108C08091C00085FF3A
:1056A000FCCF9093C600319694919923B1F7E3E72C
:1056B000F2E0949108C08091C00085FFFCCF9093E8
:1056C000C600319694919923B1F7F40107C08091F7
:1056D000C00085FFFCCF31969093C600908199233E
:1056E000B1F78091C00085FFFCCF8AE08093C600AF
:1056F000C60182539E4F0E94258139C0E9EEF1E038
:10570000CE0EDF1ED6011C92E7E1FEEFCE0EDF1EAD
:10571000EBE3F1E0949108C08091C00085FFFCCFDD
:105720009093C600319694919923B1F7E2E6F2E0A6
:10573000949108C08091C00085FFFCCF9093C60073
:10574000319694919923B1F7F40107C08091C0007C
:1057500085FFFCCF31969093C60090819923B1F7D5
:105760008091C00085FFFCCF8AE08093C600D601FF
:1057700012961C921A8A1D8A198A188A8BE794E05D
:105780009F878E87FEE4AF2EB12CAC0CBD1CEFE2E0
:10579000F0E0CE0EDF1ED501CD92DC92E1EDFFEF01
:1057A000CE0EDF1ED4018C918F3209F090C0C4015F
:1057B0006FE270E00E9451217C010894E11CF11C11
:1057C0003E010894611C711C2501E2E12E2E312C52
:1057D0002C0E3D1E77C0C7016FE270E00E94512180
:1057E0005C01009709F481C0E816F90608F07DC055
:1057F0008C010E191F09C301B701A8010E94712174
:10580000060D171DF8011082F30107C08091C0003A
:1058100085FFFCCF31969093C60090819923B1F714
:105820008091C00085FFFCCFFAE0F093C600D20162
:105830006D917C916115710519F460E070E002C012
:105840006C5F7F4FC101A30121E00E941288882371
:1058500071F5EEE4F2E0949108C08091C00085FFFC
:10586000FCCF9093C600319694919923B1F7FE0135
:10587000319607C08091C00085FFFCCF3196909390
:10588000C60090819923B1F7ECE4F2E0949108C04E
:105890008091C00085FFFCCF9093C6003196949113
:1058A0009923B1F78091C00085FFFCCF1AC12EE08B
:1058B00030E02C0F3D1FF2013183208375010894E5
:1058C000E11CF11CE114F10409F085CF0BC040E5A7
:1058D00050E0C40ED51ED501CD92DC92E0EBFFEF77
:1058E000CE0EDF1E082DF92C01C00E2DF601E25B55
:1058F000FF4F2DA5222309F4B0C06081718161158D
:10590000710519F460E070E002C06C5F7F4FC60162
:1059100082539E4F402F5F2D21E00E9412888823E2
:1059200009F46BC04FED51E0C40ED51ED6014D9168
:105930005D916D917C91ECE9F0E0CE0EDF1ED60119
:105940004D935D936D937C931397E5E8FDEFCE0E39
:10595000DF1EEEE3F2E0949108C08091C00085FF65
:10596000FCCF9093C600319694919923B1F7802F84
:105970009F2D9C01F90107C08091C00085FFFCCFDD
:1059800031969093C60090819923B1F7E6E3F2E057
:10599000949108C08091C00085FFFCCF9093C60011
:1059A000319694919923B1F784E595E02AE030E0AF
:1059B00067D88091C00085FFFCCF8AE08093C60045
:1059C00023E832E0C20ED31ED6011D921D921D9215
:1059D0001C921397E8E2F2E0949108C08091C00015
:1059E00085FFFCCF9093C600319694919923B1F72F
:1059F0008091C00085FFFCCF99C0E4E1F2E0949172
:105A000008C08091C00085FFFCCF9093C6003196FE
:105A100094919923B1F7802F9F2D9C01F90107C024
:105A20008091C00085FFFCCF31969093C600908195
:105A30009923B1F7E2E1F2E0949108C08091C000AF
:105A400085FFFCCF9093C600319694919923B1F7CE
:105A50008091C00085FFFCCF44C0608171816115D9
:105A6000710519F460E070E002C06C5F7F4FC60101
:105A700082539E4F402F5F2D26E50E941288882377
:105A800009F033C0EEEFF1E0949108C08091C000BE
:105A900085FFFCCF9093C600319694919923B1F77E
:105AA000802F9F2D9C01F90107C08091C00085FFC8
:105AB000FCCF31969093C60090819923B1F7ECEF1B
:105AC000F1E0949108C08091C00085FFFCCF9093D5
:105AD000C600319694919923B1F78091C00085FF5B
:105AE000FCCF8AE08093C60028C081E0F601808365
:105AF000EAEEF1E0949108C08091C00085FFFCCFF0
:105B00009093C600319694919923B1F7F40107C0A0
:105B10008091C00085FFFCCF31969093C6009081A4
:105B20009923B1F78091C00085FFFCCF8AE0809374
:105B3000C600802F9F2D0E947AE0CE010E961AD9C2
:105B4000AD960FB6F894DEBF0FBECDBFCF91DF91FB
:105B50001F910F91FF90EF90DF90CF90BF90AF908B
:105B60009F908F907F906F905F904F903F902F907D
:105B70000895EF92FF920F931F93CF93DF93EC0161
:105B80000E94776D8E0107511E4FD8018C919EECBB
:105B9000E92E91E0F92EEC0EFD1E882399F1C70144
:105BA0000E942581F8016081615060838DE8689FC3
:105BB000B001112462517E4F6C0F7D1FCE0141E078
:105BC00021E056DCD801EC91F0E0EE0FFF1FEE0F64
:105BD000FF1FEC0FFD1FE651FE4F40815181628196
:105BE0007381CD57DD4F488359836A837B83C358C4
:105BF000D240C7010E9411808B81882389F181E006
:105C00008A832EC00E94576BC7010E9425811A8289
:105C10008FE291E00E94065C8091700D882301F173
:105C20001092700D80912808C82FD0E0CC0FDD1F96
:105C3000C55FD54F68817981882777FD8095982F3A
:105C40000F9476022091EB033091EC034091ED0329
:105C50005091EE030F94E203181614F4198218827F
:105C6000DF91CF911F910F91FF90EF900895FC016C
:105C700081E08183CF0140E021E0FACBEF92FF92F7
:105C80000F931F93CF93DF938C01FC01138286A99E
:105C9000882321F0C801C3960E94258127EAE22EBD
:105CA00021E0F22EE00EF11EC70160E045E30E9404
:105CB000177A882309F5EBE3F1E0949108C080910D
:105CC000C00085FFFCCF9093C60031969491992334
:105CD000B1F7EFE1F3E0949108C08091C00085FF37
:105CE000FCCF9093C600319694919923B1F780919F
:105CF000C00085FFFCCF7DC0E801C455DE4FCE015A
:105D0000B70141E00E94557B882341F5CE01B701E0
:105D100040E00E94557B882309F5EBE6F1E0949181
:105D200008C08091C00085FFFCCF9093C6003196DB
:105D300094919923B1F7ECE0F3E0949108C080913D
:105D4000C00085FFFCCF9093C600319694919923B3
:105D5000B1F78091C00085FFFCCF4BC0C801C3964E
:105D6000BE010E941484882309F5EBE6F1E09491CA
:105D700008C08091C00085FFFCCF9093C60031968B
:105D800094919923B1F7ECEFF2E0949108C08091DF
:105D9000C00085FFFCCF9093C60031969491992363
:105DA000B1F78091C00085FFFCCF23C081E0F801EE
:105DB0008383EBE3F1E0949108C08091C00085FFFC
:105DC000FCCF9093C600319694919923B1F7E1EFFF
:105DD000F2E0949108C08091C00085FFFCCF9093C1
:105DE000C600319694919923B1F78091C00085FF48
:105DF000FCCF8AE08093C600D801AC5ABF4FF801AF
:105E0000F3968BE101900D928150E1F7F80181A9A1
:105E100092A90E5A1F4FF8019183808302551040BA
:105E2000C8018F96025B1F4FF80191838083DF9139
:105E3000CF911F910F91FF90EF9008952F923F9275
:105E40004F925F926F927F929F92AF92BF92CF924A
:105E5000DF92EF92FF920F931F93DF93CF93CDB713
:105E6000DEB7CC55D0400FB6F894DEBF0FBECDBF25
:105E70006C01662311F527E832E0C20ED31ED6016D
:105E80008C91E9E7FDEFCE0EDF1E882309F4E3C015
:105E90002FE732E0C20ED31ED601ED90FD900D919A
:105EA0001C91E1E8FDEFCE0EDF1E0E944CFAE616D3
:105EB000F7060807190708F4CEC027E832E0C20E3B
:105EC000D31ED6011C92E9E7FDEFCE0EDF1ED601F0
:105ED00013968C91882339F4C601D0DEF6018381B4
:105EE000882309F4B8C000D000D0EDB7FEB73196D2
:105EF0007E010894E11CF11CADB7BEB71296FC926E
:105F0000EE92119782E691E093838283D6019D966B
:105F10008D919C919E97958384830E948021870117
:105F2000EDB7FEB736960FB6F894FEBF0FBEEDBFC5
:105F300057010AC0D8018C91992787FD90950F943D
:105F40001706F80181938F01F50101900020E9F710
:105F50003197EA19FB09802F8E198E175CF363E3E2
:105F6000A62EB12CAC0CBD1CC50140E050E060E099
:105F700070E00E94118099245DE3E52EF12CEC0E77
:105F8000FD1E2E010894411C511C4FE1642E712C02
:105F90006C0E7D1E3BE5232E31E0332E42C0D8012E
:105FA0008C9190E00F941706F80181938F01D7012F
:105FB0000D900020E9F71197AE19BF09802F8E19B7
:105FC0008A176CF327968FAD27978E3751F1C7014B
:105FD000B20145E050E00E946321009711F500D026
:105FE00000D0EDB7FEB73196ADB7BEB712967C9232
:105FF0006E92119733822282558244820E948021C0
:10600000EDB7FEB736960FB6F894FEBF0FBEEDBFE4
:10601000C3010E947F5C87E591E00E94065C9924A1
:106020009394C501B70140E050E00E9433831816F5
:1060300014F48701BCCF992041F48FEF9FEFD60174
:106040009E969C938E939D9706C0F60185A596A576
:10605000019696A785A7C45ADF4F0FB6F894DEBF06
:106060000FBECDBFCF91DF911F910F91FF90EF90A9
:10607000DF90CF90BF90AF909F907F906F905F9098
:106080004F903F902F9008952F923F924F925F92A2
:106090006F927F928F929F92AF92BF92CF92DF9238
:1060A000EF92FF920F931F93DF93CF93CDB7DEB79D
:1060B000CF58D0400FB6F894DEBF0FBECDBF8C01D5
:1060C0003B016A0184E090E0C80ED91EF801719688
:1060D000C757DF4FF983E883C958D040C8010496F9
:1060E000CA57DF4F99838883C658D040C857DF4FBF
:1060F0001882C858D040B6E6EB2EF12CEC0EFD1EEF
:10610000F7013B96C557DF4FF983E883CB58D04062
:10611000A8E88A2EA2E09A2E800E911EFAE8AF2EF1
:10612000F2E0BF2EA00EB11EEEE02E2E312C2C0E72
:106130003D1E77E4472E512C4C0E5D1EC201049685
:10614000C357DF4F99838883CD58D040EBE3F1E00C
:106150009491C157DF4F9883CF58D0404EC1F7017B
:106160008385482F50E0BA01687170706031710505
:1061700009F051C1F401208131812130310509F448
:106180004AC12230310509F446C1F701DE011196FA
:106190009081903239F08E2F8E19883011F48EE272
:1061A0008D939D933196C557DF4F88819981CB5848
:1061B000D040E817F90761F71C921E86F301808131
:1061C000882329F4C10162E072E00E944621C101E6
:1061D000B3010E944621C101BE016F5F7F4F0E9443
:1061E0004621C10162E072E00E9446211CA61FA662
:1061F0001BA61AA68BE794E099A788A7CE018C96D8
:10620000B601AE014F5F5F4F21E00E9412888823E4
:1062100009F03FC0F40180819181892BD1F5C157EC
:10622000DF4F9881CF58D040EBE3F1E008C0809178
:10623000C00085FFFCCF9093C600319694919923BE
:10624000B1F7E4E0F2E007C08091C00085FFFCCF29
:1062500031969093C60090819923B1F78091C00048
:1062600085FFFCCFFAE0F093C600FE01319607C02F
:106270008091C00085FFFCCF31969093C60090813D
:106280009923B1F78091C00085FFFCCF8AE080930D
:10629000C600C357DF4FA881B981CD58D040FE0159
:1062A000BC968BE101900D928150E1F78AA59BA5E8
:1062B000F201938382838BE794E091838083C8010A
:1062C000B101A201E1DEC2010E94BA26CE01889688
:1062D0000E94BA2692C0953E09F48FC09E3209F4FE
:1062E0008CC09F3509F489C0F8019189992331F058
:1062F0009E3209F482C09F3509F47FC043FD7DC002
:1063000080E06031710509F481E0F80184A78823F9
:1063100049F4F7018085873409F06FC081858E3795
:1063200009F46BC0CA57DF4FA881B981C658D04065
:10633000F7018081803241F08E2F8E19883011F460
:106340008EE28D9380818D933196C557DF4F888182
:106350009981CB58D040E817F90759F71C92F401FE
:1063600080819181009729F5F30107C08091C000D9
:1063700085FFFCCF31969093C60090819923B1F7A9
:10638000CA57DF4FE881F981C658D04007C08091D5
:10639000C00085FFFCCF31969093C6009081992371
:1063A000B1F78091C00085FFFCCFFAE0F093C60002
:1063B00024C08130910539F4F501808191810196E5
:1063C000918380831AC00297C1F4C857DF4FF881C8
:1063D000C858D0402F2F30E0F501808191812817D7
:1063E0003907F1F0C857DF4FF881C858D040FF5F38
:1063F000C857DF4FF883C858D040C601B701C75708
:10640000DF4F48815981C958D0400E943383181604
:106410000CF4A5CE05C0F7019081992309F05BCF5C
:10642000C157DF4F0FB6F894DEBF0FBECDBFCF917F
:10643000DF911F910F91FF90EF90DF90CF90BF9071
:10644000AF909F908F907F906F905F904F903F9014
:106450002F900895EF92FF920F931F93DF93CF93A6
:10646000CDB7DEB76F970FB6F894DEBF0FBECDBFC6
:106470007C018C01025B1F4F805B9F4FF801918371
:10648000808328E832E0E20EF31E21E030E0F701DD
:10649000219331937F011182108226E73DEFE20EB6
:1064A000F31E049640E050E060E070E00E9411802E
:1064B000F80120813181DE011596F90134968BE1D6
:1064C00001900D928150E1F7F901828193819C83C3
:1064D0008B838BE794E09A838983C70167E172E03D
:1064E0008E010F5F1F4FA801CFDDC8010E94BA26A1
:1064F000F701E657FD4F808191816F960FB6F894B2
:10650000DEBF0FBECDBFCF91DF911F910F91FF90E6
:10651000EF900895EF92FF920F931F93DF93CF9325
:10652000CDB7DEB76F970FB6F894DEBF0FBECDBF05
:106530007C018C01025B1F4F805B9F4FF8019183B0
:10654000808328E832E0E20EF31E22E030E0F7011B
:106550003183208328E73DEFE20EF31EF701E65773
:10656000FD4F60831182049640E050E060E070E0EF
:106570000E941180F80120813181DE011596F90118
:1065800034968BE101900D928150E1F7F9018281FF
:1065900093819C838B838BE794E09A838983C701E3
:1065A00067E172E08E010F5F1F4FA8016DDDC8012A
:1065B0000E94BA266F960FB6F894DEBF0FBECDBF0D
:1065C000CF91DF911F910F91FF90EF900895EF927F
:1065D000FF920F931F93DF93CF93CDB7DEB76F97E3
:1065E0000FB6F894DEBF0FBECDBF7C0188E892E005
:1065F000E80EF91EF7011182108288E79DEFE80E80
:10660000F91E87010D5C1F4FC80140E050E060E0BB
:1066100070E00E941180DE011596F8018BE1019077
:106620000D928150E1F7F70181A992A99C838B8398
:106630008BE794E09A838983C70167E172E08E015A
:106640000F5F1F4FA80120DDC8010E94BA266F9678
:106650000FB6F894DEBF0FBECDBFCF91DF911F9173
:106660000F91FF90EF9008950F931F93CF93DF93B7
:10667000DC01D3961C92D397D6961C92D697D296CD
:106680001C921E92D1978BE794E0D0969C938E93A8
:106690009F97AC5ABF4F1C9213961C92A755B040BF
:1066A000FD01E05BFF4FAE5ABF4F11961C921E9248
:1066B000A255B04091838083ED01C159DF4FFE01A7
:1066C00020E030E0482F1482178213821282408328
:1066D0009183215E3F4F7F9681E02633380799F7FB
:1066E000A855BE4F89E18C9313961C9258961C9224
:1066F0001B961C9213961C92A15DB140FD01E653BE
:10670000FE4FA453BE4F11961C921E92408391835C
:10671000A155BF4F1D921D921D921C921397189662
:106720001D921D921D921C921397A358B24012966F
:106730001C92129713961C9213971C9211961C92FE
:1067400011978D0101581D4FF8011082118212829C
:106750001382AB55BE4F11961C921E92AC5BBF4F7D
:106760001C92FE01C90111920197E9F7A256BF4F91
:1067700081E08C93A758B2409E961C921E929D97E2
:106780000E944CFA68577C4E8F4F9F4FF8016083F0
:10679000718382839383DF91CF911F910F9108952D
:1067A000EF92FF920F931F93CF93DF93EC01E09052
:1067B0000508F09006080091070810910808688104
:1067C00079818A819B81A80197010F94D401882344
:1067D00024F4E882F9820A831B83E0900908F09090
:1067E0000A0800910B0810910C086C817D818E8144
:1067F0009F81A80197010F94D401882324F4EC828F
:10680000FD820E831F83E0900D08F0900E0800912A
:106810000F0810911008688579858A859B85A801E5
:1068200097010F94D401882324F4E886F9860A8717
:106830001B87E090A503F090A6030091A703109199
:10684000A803688179818A819B81A80197010F94AF
:10685000E203181624F4E882F9820A831B83E0908D
:10686000A903F090AA030091AB031091AC036C81D3
:106870007D818E819F81A80197010F94E2031816F4
:1068800024F4EC82FD820E831F83E090AD03F09030
:10689000AE030091AF031091B003688579858A85B6
:1068A0009B85A80197010F94E203181624F4E8864B
:1068B000F9860A871B87DF91CF911F910F91FF9077
:1068C000EF90089580913608089567707070E82FF2
:1068D000F0E0E554F44C84918B3028F48830A0F437
:1068E000863090F106C08E30D0F08F50833060F546
:1068F00021C08091B100887F8093B1008091B10068
:10690000862B8093B100089580919100887F8093B9
:10691000910080919100862B809391000895809141
:10692000A100887F8093A1008091A100862B809395
:10693000A100089580912101887F80932101809199
:106940002101862B8093210108950F931F93CF93EC
:10695000DF938130910541F46F5F7F4F09F045C0AF
:1069600085E595E081DE41C0892B09F03EC06F5F6F
:106970007F4FD9F58BE794E09093200780931F0712
:1069800080912607882321F083E297E00E942581E9
:10699000CBEDD6E00BE714E005C06F9785E0C53A74
:1069A000D80751F0198308838F818823B1F3CE0172
:1069B00004960E942581F1CF8BE794E09983888328
:1069C0008F81882321F0CE0104960E9425818BE7D8
:1069D00094E0909385058093840580918B058823AE
:1069E00021F088E895E00E942581DF91CF911F91E9
:1069F0000F91089580E090E06FEF7FEFA6CF81E0E8
:106A000090E06FEF7FEFA1CF0E94ED5D809136089F
:106A1000882309F03AC081E08093360880914108CC
:106A200090914208A0914308B09144088093450892
:106A300090934608A0934708B0934808E2E3F3E038
:106A4000949108C08091C00085FFFCCF9093C60050
:106A5000319694919923B1F7E3E4F3E0949108C05F
:106A60008091C00085FFFCCF9093C6003196949131
:106A70009923B1F78091C00085FFFCCF8AE0809315
:106A8000C60089E393E00C9458E0089580E560E047
:106A90000E94F3FB779A0895F8940E94ED5D179A8F
:106AA00010921108169A10921208159A1092130853
:106AB000149A139A84E060E00E94F3FBE2E3F3E0AF
:106AC000949108C08091C00085FFFCCF9093C600D0
:106AD000319694919923B1F7E2ECF3E0949108C0D8
:106AE0008091C00085FFFCCF9093C60031969491B1
:106AF0009923B1F78091C00085FFFCCF8AE0809395
:106B0000C60089EB93E00E9467E0FFCF0E944CFA39
:106B10006093490870934A0880934B0890934C08FF
:106B2000E0917208F0917308EC58F74F8081882348
:106B3000A9F4E1EEF3E0949108C08091C00085FFD4
:106B4000FCCF9093C600319694919923B1F7809130
:106B5000C00085FFFCCF8AE08093C60008950E94A4
:106B60004CFA20913C0830913D0840913E085091EC
:106B70003F08621B730B840B950B645C794080406B
:106B8000904008F446C00E944CFA60933C08709311
:106B90003D0880933E0890933F08079B06C0069BE4
:106BA00004C0059B02C004990AC00E944CFA60937D
:106BB00038087093390880933A0890933B080E94F4
:106BC0004CFA209138083091390840913A08509198
:106BD0003B08621B730B840B950B60567A4E80400A
:106BE000904028F4211531054105510549F482E012
:106BF00060E00E94A6FC82E060E070E00C9415FB6F
:106C000082E062E80E94A6FC82E062E870E00C94F8
:106C100015FB0895EF92FF920F931F930E944CFA79
:106C2000E0904D08F0904E0800914F0810915008E8
:106C30002091490830914A0840914B0850914C08E6
:106C4000621B730B840B950BE616F70608071907F2
:106C500030F4E114F1040105110509F01DDF809104
:106C6000B3039091B403A091B503B091B60300971C
:106C7000A105B10561F10E944CFA209149083091BB
:106C80004A0840914B0850914C08621B730B840BCF
:106C9000950B2091B3033091B4034091B50350910B
:106CA000B603261737074807590788F490918112D1
:106CB00080918212981759F4179A10921108169A17
:106CC00010921208159A10921308149A139A679941
:106CD00001C0E2DE44DF0E94C58C1F910F91FF903E
:106CE000EF9008956F927F928F929F92AF92BF9292
:106CF000CF92DF92EF92FF920F931F93F82E609145
:106D00005108709152088091530890915408209135
:106D100055083091560840915708509158080F94E3
:106D2000EF033B014C0100D000D00DB71EB70F5F41
:106D30001F4F6091990370919A03882777FD809582
:106D4000982F0F9476022091B7033091B8034091A9
:106D5000B9035091BA030F94B40420E030E040E747
:106D600052E40F94DB0120E030E048EC52E40F9451
:106D7000DB015B016C01F801608271828282938287
:106D8000F48280912808858389EE97E06DE578E0AC
:106D900041E558E020E001E032E0E32E0E94E47497
:106DA00080915D0890915E08A0915F08B0916008A5
:106DB0008093E9079093EA07A093EB07B093EC0761
:106DC0008091610890916208A0916308B091640875
:106DD0008093ED079093EE07A093EF07B093F00731
:106DE0008091650890916608A0916708B091680845
:106DF0008093F1079093F207A093F307B093F40701
:106E00008091690890916A08A0916B08B0916C0814
:106E10008093F5079093F607A093F707B093F807D0
:106E20008DB79EB706960FB6F8949EBF0FBE8DBF66
:106E30000E944CFA6093490870934A0880934B086B
:106E400090934C081F910F91FF90EF90DF90CF909F
:106E5000BF90AF909F908F907F906F900895CF924A
:106E6000DF92EF92FF920F931F938DE598E098DCED
:106E70000E944CFA6093490870934A0880934B082B
:106E800090934C086091E9077091EA078091EB07B5
:106E90009091EC0720915D0830915E0840915F0869
:106EA000509160080F94D401882309F07AC0609152
:106EB000ED077091EE078091EF079091F007209118
:106EC00061083091620840916308509164080F9402
:106ED000D401882309F065C06091B7037091B803AD
:106EE0008091B9039091BA0320E030E040E752E48A
:106EF0000F94DB017B018C018DE598E061E678E081
:106F000045E658E029E638E0E8E2CE2EE8E0DE2E5D
:106F10000E94F38F80915D0890915E08A0915F08B8
:106F2000B09160088093E9079093EA07A093EB077C
:106F3000B093EC078091610890916208A09163087A
:106F4000B09164088093ED079093EE07A093EF074C
:106F5000B093F0078091650890916608A09167084A
:106F6000B09168088093F1079093F207A093F3071C
:106F7000B093F4078091690890916A08A0916B081A
:106F8000B0916C088093F5079093F607A093F707EC
:106F9000B093F8071F910F91FF90EF90DF90CF9083
:106FA00008956091990370919A03882777FD8095E1
:106FB000982F0F9476022091B7033091B803409137
:106FC000B9035091BA030F94B40420E030E040E7D5
:106FD00052E40F94DB0120E030E048EC52E488CF2B
:106FE00084E595E00E949E24E4EEF3E0949108C0CD
:106FF0008091C00085FFFCCF9093C600319694919C
:107000009923B1F74091410850914208609143089B
:10701000709144084F5F5F4F6F4F7F4F84E595E05D
:107020002AE030E00E945C258091C00085FFFCCF03
:107030008AE08093C6006ACD2F923F924F925F9272
:107040006F927F928F929F92AF92BF92CF92DF9278
:10705000EF92FF920F931F93DF93CF93CDB7DEB7DD
:1070600028970FB6F894DEBF0FBECDBF98878F83E9
:107070008330910508F056C1FC01E15DF94FD490D1
:107080003C01660C771C660C771C93012751384F26
:107090003A83298380E090E0A0E0B0E0F9018083AA
:1070A0009183A283B38389EE97E06DEE77E041EFA1
:1070B00057E025EF37E00E94948AF301ED5DF94F28
:1070C000E590F590059114916D2D772767FD7095EA
:1070D000882777FD8095982F0F9476021B012C014D
:1070E0009301235A374F3C832B83C801B70120E01B
:1070F00030E040EC5FE30F94B404A20191010F94DF
:10710000B404AB81BC816D937D938D939C93139755
:10711000F301E757FC4FFE83ED836081718182812B
:1071200093816093B7037093B8038093B9039093EE
:10713000BA0320E030E040E752E40F94DB017B012A
:107140008C018DE598E061E678E045E658E029E6B7
:1071500038E0A8E2CA2EA8E0DA2E0E94F38F0E943F
:10716000776D80E090E0A0E0B0E0E981FA81808373
:107170009183A283B38389EE97E06DEE77E041EFD0
:1071800057E025EF37E00E94948AF301EA5AF94F5D
:1071900085909590A590B490C501B4019058A20136
:1071A00091010F94B404AB81BC816D937D938D9359
:1071B0009C9313976091B7037091B8038091B903C2
:1071C0009091BA0320E030E040E752E40F94DB01F5
:1071D0007B018C018DE598E061E678E045E658E0BA
:1071E00029E638E00E94F38F0E94776DC501B40153
:1071F000A50194010F94FB00A20191010F94B40426
:10720000EB81FC816083718382839383AD81BE8136
:107210006D917D918D919C9120E030E040E05FE3A5
:107220000F94B4046093B7037093B8038093B903C9
:107230009093BA0320E030E040E752E40F94DB0182
:107240007B018C018DE598E061E678E045E658E049
:1072500029E638E00E94F38F0E94776DF301EE5C1F
:10726000F94F6591759185919491F301E750F84F2D
:10727000A080B180C280D380A60195010F94FB004D
:107280007B018C01CB01D801E981FA818083918354
:10729000A283B383F301E25CF94F65917591859107
:1072A0009491F5E08F2EF8E09F2E860C971CA60196
:1072B00095010F94FB00D4016D937D938D939C9366
:1072C0001397F301E65BF94F659175918591949160
:1072D000E5EAF3E06E0E7F1EA60195010F94FB0018
:1072E000D3016D937D938D939C931397C701D80120
:1072F000EB81FC8180839183A283B38380E090E063
:10730000A0E0B0E08093B7039093B803A093B903D3
:10731000B093BA030E94EA6AAF81B885AF5EB74FF7
:1073200081E08C9328960FB6F894DEBF0FBECDBFD8
:10733000CF91DF911F910F91FF90EF90DF90CF9051
:10734000BF90AF909F908F907F906F905F904F9085
:107350003F902F900895409172085091730820E655
:1073600030E0B901469F9001479F300D569F300D88
:107370001124682F772767FD7095C9018258974FB0
:107380000E9451219C0190937D0880937C0880E0AD
:10739000232B09F081E00895FC01949108C08091AD
:1073A000C00085FFFCCF9093C6003196949199233D
:1073B000B1F784E595E022E030E00C946226FC0110
:1073C000949108C08091C00085FFFCCF9093C600C7
:1073D000319694919923B1F784E595E02AE030E065
:1073E0000C94402580917C0890917D08019660E086
:1073F00070E04AE050E00C94B01F80917C089091BE
:107400007D08019660E070E00C94531ECF93DF93EB
:10741000EC01809128088093400884E59CDF882354
:1074200009F46EC0EADF0F944802262F60934008EB
:10743000623008F465C0ECE2F3E0949108C08091FA
:10744000C00085FFFCCF9093C6003196949199239C
:10745000B1F7C936D10599F0CA36D10524F4C8363A
:10746000D105F1F50FC0CD36D10531F0CA3DD105BA
:10747000B9F5E8E1F2E031C0EFE2F2E023C0E6E482
:10748000F2E015C0EDE5F2E007C08091C00085FF95
:10749000FCCF31969093C60090819923B1F720C01C
:1074A0008091C00085FFFCCF31969093C6009081FB
:1074B0009923B1F715C08091C00085FFFCCF3196AC
:1074C0009093C60090819923B1F70AC08091C000C3
:1074D00085FFFCCF31969093C60090819923B1F738
:1074E00084E595E0622F40E050E00E944B258091BA
:1074F000C00085FFFCCF8AE08093C60081E001C018
:1075000080E0DF91CF910895AF92BF92CF92DF924A
:10751000EF92FF920F931F93CF93DF9319EEE12E1B
:1075200017E0F12ECDE5D8E000E010E0F801E25ED2
:10753000FB4F808110DF882331F15FDF5B016C013D
:10754000F801ED51F84F8081882311F061E002C00D
:1075500060916D0870E0882777FD8095982F0F94D3
:107560007602F70120813181428153810F94B40466
:107570009B01AC01C601B5010F94FB0068837983C0
:107580008A839B8309C0F70180819181A281B381A5
:1075900088839983AA83BB830F5F1F4F84E090E0A9
:1075A000E80EF91E24960430110509F0BFCF86E4D9
:1075B000D2DE8823D9F021DF7B018C0160936E0835
:1075C00070936F08809370089093710820E030E00A
:1075D00040E050E00F94E203181644F4E092B70341
:1075E000F092B8030093B9031093BA03DF91CF91DF
:1075F0001F910F91FF90EF90DF90CF90BF90AF90D1
:10760000089582DF89E4A7DE882351F0F6DE6093D7
:1076100051087093520880935308909354080CC0FB
:1076200080E090E0A0E0B0E0809351089093520891
:10763000A0935308B09354088AE48DDE882351F058
:10764000DCDE60935508709356088093570890933A
:107650005808089580E090E0A0E0B0E080935508DD
:1076600090935608A0935708B093580808952F9206
:107670003F924F925F926F927F928F929F92AF92C2
:10768000BF92CF92DF92EF92FF920F931F93DF93FF
:10769000CF93CDB7DEB7EE970FB6F894DEBF0FBE2F
:1076A000CDBF87E458DE882309F4E4C3A6DE0F9437
:1076B00043026430710509F43CC06530710554F42F
:1076C0006230710531F16330710554F57723CCF4E4
:1076D0000C945E556A35710509F47BC36B357105F1
:1076E00034F46C31710511F00C945E5565C06B3546
:1076F000710509F472C36C35710511F00C945E5577
:1077000071C380913608882321F4FEDEA8DB0C9437
:10771000855580913608882319F473DF81E006C00F
:1077200080913608882329F46CDF80E0DBDA0C9442
:1077300085558AE196E00E9458E080E50CDE8823BA
:1077400021F4EE24FF24870105C057DE0F94480280
:107750007B018C0183E5FFDD882359F04EDE20E0BC
:1077600030E04AE754E40F94B4040F9448027B01DC
:107770008C010E94776D0E944CFA5B016C01AE0C8B
:10778000BF1CC01ED11E0E944CFA60934908709322
:107790004A0880934B0890934C0805C00E943763B9
:1077A00039DA0E9435E10E944CFA6A157B058C0596
:1077B0009D05A0F30C945E558091B7039091B8039A
:1077C000A091B903B091BA03809378089093790897
:1077D000A0937A08B0937B088091990390919A03C3
:1077E0009093E8078093E70784E690E090939A03EC
:1077F000809399030E944CFA6093490870934A0859
:1078000080934B0890934C0881E00E94F16A80912C
:10781000E9079091EA07A091EB07B091EC078093FC
:107820005D0890935E08A0935F08B0936008809114
:10783000ED079091EE07A091EF07B091F0078093CC
:10784000610890936208A0936308B09364088091E4
:10785000F1079091F207A091F307B091F40780939C
:10786000650890936608A0936708B09368088091B4
:10787000F5079091F607A091F707B091F80780936C
:10788000690890936A08A0936B08B0936C0880E035
:1078900090E0A0E0B0E08093B7039093B803A0938A
:1078A000B903B093BA0388E556DD882351F489E51E
:1078B00052DD882331F48AE54EDD882311F481E01E
:1078C00001C080E08093BB03882351F488E543DD49
:1078D000882309F4D3C189E53EDD882309F4CEC1AC
:1078E00080E090E0A0E0B0E08093E9079093EA07A1
:1078F000A093EB07B093EC078093ED079093EE070E
:10790000A093EF07B093F007FFE28F2EF6E09F2ED3
:10791000F401E49089EE97E06DEE77E041EF57E0F7
:1079200025EF37E00E94948AE3E2F6E065917591D5
:107930008591949120E030E040EC5FE30F94B40433
:107940005B016C01FF24E7FCF0940027F7FC009535
:10795000102FC801B7010F9476029B01AC01C6013C
:10796000B5010F94B40460935D0870935E08809332
:107970005F0890936008E7E2F6E065917591859164
:1079800094910894811C911CF401D49020E030E083
:1079900040EC5FE30F94B4047B018C016D2D7727DD
:1079A00067FD7095872F972F0F9476029B01AC018E
:1079B000C801B7010F94B404609361087093620822
:1079C00080936308909364082091890330918A031F
:1079D00040918B0350918C032093B7033093B803ED
:1079E0004093B9035093BA03E0908D03F0908E0357
:1079F00000918F0310919003C801B7010F94D40137
:107A0000882344F4E092B703F092B8030093B903DB
:107A10001093BA036091B7037091B8038091B903D2
:107A20009091BA0320E030E040E752E40F94DB018C
:107A30007B018C018DE598E061E678E045E658E051
:107A400029E638E0E8E2CE2EE8E0DE2E0E94F38F51
:107A50000E94776DE2E3F6E06591759185919491CE
:107A60002091F9073091FA074091FB075091FC07EC
:107A70000F94FB006093E9077093EA078093EB078C
:107A80009093EC07EEE3F6E0659175918591949102
:107A90002091F9073091FA074091FB075091FC07BC
:107AA0000F94FB0060930508709306088093070805
:107AB00090930808EAE4F6E06591759185919491B8
:107AC0002091F9073091FA074091FB075091FC078C
:107AD0000F94FB006093A5037093A6038093A70304
:107AE0009093A803E6E3F6E06591759185919491F2
:107AF0002091FD073091FE074091FF07509100084B
:107B00000F94FB006093ED077093EE078093EF07EF
:107B10009093F007E2E4F6E0659175918591949178
:107B20002091FD073091FE074091FF07509100081A
:107B30000F94FB006093090870930A0880930B0868
:107B400090930C08EEE4F6E065917591859194911F
:107B50002091FD073091FE074091FF0750910008EA
:107B60000F94FB006093A9037093AA038093AB0367
:107B70009093AC0389EE97E06DEE77E041EF57E02C
:107B800025EF37E00E94948A8091E9079091EA07F7
:107B9000A091EB07B091EC0780935D0890935E088D
:107BA000A0935F08B09360088091ED079091EE0775
:107BB000A091EF07B091F00780936108909362085D
:107BC000A0936308B09364086091B7037091B80301
:107BD0008091B9039091BA0320E030E040E752E48D
:107BE0000F94DB017B018C018DE598E061E678E084
:107BF00045E658E029E638E00E94F38F80E090E007
:107C0000A0E0B0E08093B7039093B803A093B903CA
:107C1000B093BA030E94776D0E94EA6A80915D0872
:107C200090915E08A0915F08B09160088093E90789
:107C30009093EA07A093EB07B093EC07809161085B
:107C400090916208A0916308B09164088093ED0759
:107C50009093EE07A093EF07B093F007809165082B
:107C600090916608A0916708B09168088093F10729
:107C70009093F207A093F307B093F4078091BB03AE
:107C8000882321F488E567DB882319F080E090E001
:107C9000D3D98091BB03882321F489E55CDB882359
:107CA00019F081E090E0C8D988E555DB8823C9F058
:107CB00099DB611571058105910599F09EDB209195
:107CC000F9073091FA074091FB075091FC070F9498
:107CD000FB006093E9077093EA078093EB079093AA
:107CE000EC0789E538DB8823C9F07CDB6115710579
:107CF0008105910599F081DB2091FD073091FE0708
:107D00004091FF07509100080F94FB006093ED072E
:107D10007093EE078093EF079093F0078091BB0379
:107D2000882321F48AE517DB882319F082E090E0AC
:107D300083D98AE510DB8823C9F054DB611571050E
:107D40008105910599F059DB2091010830910208D5
:107D500040910308509104080F94FB006093F107D1
:107D60007093F2078093F3079093F40789EE97E0FE
:107D70006DEE77E041EF57E025EF37E00E94948AFF
:107D800080E00E94F16A8091780890917908A09132
:107D90007A08B0917B088093B7039093B803A093BF
:107DA000B903B093BA038091E7079091E8079093E5
:107DB0009A03809399030E944CFA60934908709348
:107DC0004A0880934B0890934C080E94EA6A0C94EE
:107DD0005E5510926D080C945E5581E080936D089D
:107DE0000C945E5585E4B7DA882311F40E94776D10
:107DF00059EEE52E57E0F52E49EFC42E47E0D42E7C
:107E000000E010E0F801E25EFB4F8081A4DA8823F5
:107E100021F1033059F4F1DAF70160837183828331
:107E2000938385EF97E00E94648A17C0E6DAF60133
:107E300020813181428153810F94FB00F7016083DF
:107E400071838283938389EE97E06DEE77E041EF53
:107E500057E025EF37E00E94948A0F5F1F4F24E020
:107E600030E0E20EF31EC20ED31E0430110551F6AF
:107E70000C945E558DE46FDA882311F40C9402544F
:107E8000BCDA0F9443026737710509F48AC1683779
:107E900071050CF0B3C06032710509F401C36132A1
:107EA00071050CF049C06731710509F420C26831D1
:107EB000710524F56231710511F40C943349633175
:107EC000710574F477FF02C00C945E556230710541
:107ED0000CF46BC16131710511F00C945E55C0C199
:107EE0006531710509F4F7C1663171050CF0F9C10E
:107EF0006431710511F00C945E55BDC16B31710593
:107F000009F445C26C3171054CF46931710509F40D
:107F10001AC26A3171050CF01CC205C26E317105BE
:107F200009F478C26F3171050CF065C36C317105CD
:107F300011F00C945E5531C26C35710511F40C943E
:107F4000A5496D3571054CF56235710511F40C9438
:107F50002A496335710584F46035710511F40C9478
:107F6000FF486135710514F00C940C496A327105B3
:107F700011F00C945E55EEC36435710511F40C9448
:107F800033496435710514F40C942E496535710537
:107F900011F00C945E550C948E496B36710511F4FA
:107FA0000C94F3486C3671057CF46936710509F45C
:107FB0004CC46A36710514F00C9464486836710537
:107FC00011F00C945E5510C46237710511F40C94D5
:107FD000524A6337710534F46D36710511F00C9413
:107FE0005E5570C56337710511F40C942B4A6537E3
:107FF000710511F00C945E550C943B4A31E06C32E3
:10800000730711F40C946C4E41E06D3274070CF060
:108010005AC06C3C710511F40C94A64C6D3C710572
:1080200044F56E3B710509F43CC76F3B710584F460
:108030006937710511F40C944C4B6937710514F4D0
:108040000C94474B6C38710511F00C945E55ECC3E1
:10805000693C710511F40C94644C6B3C710511F48E
:108060000C94874C683C710511F00C945E550C948F
:10807000D94B6C3D710511F40C94F64D6D3D7105B5
:108080008CF46E3C710511F40C94284D6E3C710516
:1080900014F40C94C84C6A3D710511F00C945E55B3
:1080A0000C94474D623E710511F40C94144E6A3FD6
:1080B000710511F40C9429506D3D710511F00C946B
:1080C0005E550C94054E51E0643F750711F40C9415
:1080D000B65081E0653F780754F591E06033790749
:1080E00011F40C947B4FE1E061337E076CF4F1E016
:1080F0006E327F0711F40C9464506F52714014F08B
:108100000C9473500C94A34E31E06F35730711F447
:108110000C94835341E06039740711F40C94B3500C
:108120006E55714011F00C945E550C94435382E0EF
:108130006835780711F40C94C25092E069357907DC
:108140009CF4E1E0663F7E0711F40C94BC50F1E032
:10815000663F7F0714F40C94B950675F714011F0CB
:108160000C945E550C94BF5033E06C38730711F4D7
:108170000C942A5343E06D3874073CF46B587340F9
:1081800011F00C945E550C94ED5283E0603A780740
:1081900009F4F6C1675E734011F00C945E550C94BF
:1081A000EB53E4E7F2E00C94584B89E096E00E9430
:1081B00058E080E5D0D8882321F4EE24FF248701FD
:1081C00005C01BD90F9448027B018C0183E5C3D8FD
:1081D000882359F012D920E030E04AE754E40F94A4
:1081E000B4040F9448027B018C010E94776D0E94B9
:1081F0004CFA6093490870934A0880934B08909317
:108200004C08E114F1040105110501F10E944CFA3A
:108210005B016C01AE0CBF1CC01ED11E0E944CFA4B
:108220006A157B058C059D05A8F40E94959C882302
:1082300089F40E9437630E940A360E9435E1EECF2E
:108240000E9437630E940A360E9435E10E94959C85
:108250008823B1F38AEF95E00E9458E00C945E55B4
:1082600081EF95E00E9458E0179816981598149899
:1082700013980C945E55E1EEF5E0949108C080915E
:10828000C00085FFFCCF9093C6003196949199234E
:10829000B1F78091C00085FFFCCF8AE08093C600D3
:1082A00085E595E00E94E732E3EDF5E0949108C0A2
:1082B0008091C00085FFFCCF9093C60031969491C9
:1082C0009923B1F78091C00085FFFCCF8AE08093AD
:1082D000C6000C945E5585E595E00E943E2E0C94F8
:1082E0005E5585E595E00E9464260C945E5580916C
:1082F0007C0890917D0804966AE270E00E9451210A
:10830000FC01009711F03197108260917C08709108
:108310007D086C5F7F4F85E595E041E021E00E949C
:10832000382A0C945E5585E595E00E9468260E94E7
:108330004CFA60932E0870932F0880933008909326
:1083400031080C945E5585E595E00E946F260C94EB
:108350005E5580915805882311F40C945E5583E591
:108360000E94AB39882311F40C945E553BD8AB01C5
:10837000BC014093D8075093D9078093DA077093D4
:10838000DB0783E297E00E9411800C945E5585E53F
:1083900095E00E9429280C945E5580917C0890916C
:1083A0007D0804966AE270E00E9451218C010097DA
:1083B00019F1209172083091730880E690E0FC0179
:1083C0002E9FC0012F9F900D3E9F900D112482582B
:1083D000974F6EE470E00E94512160E270E00E94CD
:1083E00051219C012F5F3F4F30937D0820937C08E3
:1083F00001501040F801108260917C0870917D0856
:108400006C5F7F4F85E595E040E021E00E94382ACF
:108410000C945E5580915805882311F40C945E5598
:1084200085E595E060E00E949B2780917C08909113
:108430007D0804966AE270E00E9451218C01009749
:1084400019F1209172083091730880E690E0AC0138
:10845000249FC001259F900D349F900D11248258B8
:10846000974F6EE470E00E94512160E270E00E943C
:1084700051219C012F5F3F4F30937D0820937C0852
:1084800001501040F801108260917C0870917D08C5
:108490006C5F7F4F85E595E00E9481280C945E55C6
:1084A00080915705882311F00E94776DE0907C0839
:1084B000F0907D0824E030E0E20EF31EC7016AE28E
:1084C00070E00E9451218C01C70161E270E00E94BE
:1084D0005121009721F07C010894E11CF11C011549
:1084E000110521F001501040F801108280E50E9432
:1084F000AB39182F80917C0890917D08E816F90619
:1085000008F410E080915805882311F40C945E550E
:1085100021E0212785E595E0B70141E00E94382A56
:1085200083E50E94AB398823B9F080917C08909153
:108530007D088E159F0580F40E94F239AB01BC01C5
:108540004093D8075093D9078093DA077093DB07DD
:1085500083E297E00E94118085E595E00E946826FD
:10856000112311F00C945E550E944CFA60932E0872
:1085700070932F0880933008909331080C945E55C7
:1085800080917C0890917D0805966AE270E00E94D7
:1085900051218C01009719F12091720830917308D4
:1085A00080E690E0AC01249FC001259F900D349F90
:1085B000900D11248258974F6EE470E00E94512173
:1085C00060E270E00E9451219C012F5F3F4F309389
:1085D0007D0820937C0801501040F80110826091C2
:1085E0007C0870917D086B5F7F4F85E595E00E9468
:1085F000372E0C945E550E944CFA609332087093AB
:108600003308809334089093350820912E083091D8
:108610002F084091300850913108621B730B840B76
:10862000950B28EE33E040E050E00F94CC05F22E9D
:10863000E32ED42EC52E2DB73EB7285030400FB6AE
:10864000F8943EBF0FBE2DBF0DB71EB70F5F1F4F73
:10865000CE018196EDB7FEB79283818384EC95E0DD
:10866000F801938382836F2D7E2D842F952F2CE329
:1086700030E040E050E00F94CC05F80135832483CE
:108680006F2D7E2D8D2D9C2D2CE330E040E050E0B1
:108690000F94CC05F801778366830E948021ECE279
:1086A000F3E094912DB73EB7285F3F4F0FB6F89493
:1086B0003EBF0FBE2DBF08C08091C00085FFFCCF1C
:1086C0009093C600319694919923B1F7FE01B1962B
:1086D00007C08091C00085FFFCCF31969093C60003
:1086E00090819923B1F78091C00085FFFCCF8AE08B
:1086F0008093C600CE0181960E947AE08091700D31
:10870000882311F40C945E551092700D8091280806
:10871000082F10E0000F111F055F154FF801608151
:108720007181882777FD8095982F0F94760220918C
:10873000EB033091EC034091ED035091EE030F9465
:10874000E203181614F00C945E55F80111821082A1
:108750000C945E5583E50E94AB39882311F40C9488
:108760005E550E94FD390F9443027B018C016B0121
:1087700080E50E94AB39882369F0F7FC0BC0FFEF5E
:10878000EF16F10409F034F40E94FD390F9443020E
:108790008B0102C00DE010E0E2E2F4E08081918103
:1087A0008017910711F40C945E55329624E0E23A5A
:1087B000F207A1F70630110529F4D0922B08C092D8
:1087C0002A0804C017FF02C00C945E55802F61E098
:1087D0000E94F3FB802F6C2D0E94A6FC802FB60117
:1087E0000E9415FB0C945E5588E690E00E94063AC4
:1087F000882311F00C945E5583E50E94AB398823E1
:1088000079F00E94FD3920914008022F10E0000FFE
:10881000111F055F154F0F944302F80171836083A8
:108820000E94EC5D0C945E5583E50E94AB39882371
:1088300011F40C945E550E94FD390F94430270931D
:10884000100A60930F0A0C945E5589E690E00E942E
:10885000063A882311F00C945E55EEEBF5E0949106
:1088600008C08091C00085FFFCCF9093C600319670
:1088700094919923B1F7E0914008F0E0EE0FFF1FCB
:10888000EE0FFF1FEB5EF54F4081518162817381D6
:1088900084E595E021E030E00E946226EBEBF5E014
:1088A000949108C08091C00085FFFCCF9093C600D2
:1088B000319694919923B1F7E0914008F0E0EE0FE2
:1088C000FF1FE55FF54F60817181882777FD8095F7
:1088D000982F0F947602AB01BC0184E595E021E06E
:1088E00030E00E946226E7EBF5E0949108C08091A9
:1088F000C00085FFFCCF9093C600319694919923D8
:10890000B1F740911F0A5091200A6091210A70919D
:10891000220A84E595E021E030E00E946226E4EB43
:10892000F5E0949108C08091C00085FFFCCF909342
:10893000C600319694919923B1F760910F0A709116
:10894000100A882777FD8095982F0F947602AB0147
:10895000BC0184E595E021E030E00E9462260BE056
:10896000C02E0AE0D02E15E1E12E1AE0F12E00E033
:1089700010E0E1EBF5E09490EFEAF5E0A490ECEA8A
:10898000F5E0B490992DE1EBF5E008C08091C000CE
:1089900085FFFCCF9093C600319694919923B1F74F
:1089A00084E595E0B8014AE050E00E948F259A2DB9
:1089B000EFEAF5E008C08091C00085FFFCCF9093FE
:1089C000C600319694919923B1F7F7014081518106
:1089D0006281738184E595E021E030E00E946226A7
:1089E0009B2DECEAF5E008C08091C00085FFFCCF2C
:1089F0009093C600319694919923B1F7F601619155
:108A000071916F01882777FD8095982F0F947602DA
:108A1000AB01BC0184E595E021E030E00E946226D4
:108A20000F5F1F4F24E030E0E20EF31E023011050D
:108A300009F0A8CFE8EAF5E0949108C08091C00061
:108A400085FFFCCF9093C600319694919923B1F79E
:108A5000809140080E94315DBC0184E595E04AE0C8
:108A600050E00E948F25E3EAF5E0949108C08091E0
:108A7000C00085FFFCCF9093C60031969491992356
:108A8000B1F78FEF9FEF0E94315DBC0184E595E067
:108A90004AE050E00E948F25EDE8F2E007C08091A7
:108AA000C00085FFFCCF31969093C600908199233A
:108AB000B1F78091C00085FFFCCF8AE08093C600AB
:108AC0000C9485558DE690E00E94063A882311F0BB
:108AD0000C945E5588E995E00E9458E01092700D64
:108AE00083E50E94AB39882399F00E94FD392091DB
:108AF0004008022F10E0000F111F055F154F0F9463
:108B00004302F8017183608381E08093B20316C051
:108B100082E50E94AB39882389F00E94FD392091BB
:108B20004008022F10E0000F111F055F154F0F9432
:108B30004302F801718360831092B20383E50E94BF
:108B4000AB39882351F00E94FD396093EB03709399
:108B5000EC038093ED039093EE0382E40E94AB3923
:108B6000882351F00E94FD396093E7037093E80376
:108B70008093E9039093EA0386E40E94AB3988234B
:108B800069F00E94FD396093EF037093F0038093C6
:108B9000F1039093F20381E08093700D0E94EC5DED
:108BA0000E944CFA4B015C0120914008022F10E01A
:108BB00010923708000F111FF801E55FF54F608133
:108BC0007181882777FD8095982F0F947602000F8A
:108BD000111F0B5E154FF8012081318142815381B5
:108BE0000F94E20318161CF481E080933708CC241C
:108BF000CA94DC2C7601E5E9F5E05490E1E9F5E072
:108C00006490EDE8F5E074907AE0472E3DC1952D33
:108C1000E5E9F5E008C08091C00085FFFCCF9093A6
:108C2000C600319694919923B1F7E0914008F0E0A5
:108C3000EE0FFF1FEE0FFF1FEB5EF54F40815181DE
:108C40006281738184E595E021E030E00E94622634
:108C5000962DE1E9F5E008C08091C00085FFFCCFCA
:108C60009093C600319694919923B1F76091400892
:108C700084E595E070E04AE050E00E948F25972D52
:108C8000EDE8F5E008C08091C00085FFFCCF90932F
:108C9000C600319694919923B1F7F7FE03C0EEE830
:108CA000F2E02CC00E944CFA6C197D098E099F09D4
:108CB0000F9474029B01AC0160E070E08AEF93E4D2
:108CC0000F94FA0020E030E04AE754E40F94DB010F
:108CD0000F944802AB01BC0184E595E02AE030E046
:108CE0000E9440258091C00085FFFCCF0EC080917E
:108CF000C00085FFFCCF31969093C60090819923E8
:108D0000B1F78091C00085FFFCCF4092C6000E9461
:108D10004CFA4B015C010E9437630E940A360E94A4
:108D200035E1FFEFCF16FFEFDF06FFEFEF06FFEFB6
:108D3000FF0609F052C080913708E091400888236F
:108D400031F1F0E08F01000F111F000F111F0B5EBA
:108D5000154FEE0FFF1FE55FF54F6081718188278A
:108D600077FD8095982F0F94760220E030E040E266
:108D700051E40F94FA009B01AC01F801608171810C
:108D8000828193810F94E20387FF58C05EC0F0E0B8
:108D90008F01000F111F000F111F0B5E154FEE0FFB
:108DA000FF1FE55FF54F60817181882777FD809512
:108DB000982F0F94760220E030E040E251E40F94C7
:108DC000FB009B01AC01F80160817181828193817C
:108DD0000F94D401181694F538C0F7FC36C0E09112
:108DE0004008F0E08F01000F111F000F111F0B5EF4
:108DF000154FEE0FFF1FE55FF54F608171818827EA
:108E000077FD8095982F0F9476029B01AC01F801B5
:108E100060817181828193810F94FA000F944302E3
:108E200097FF07C090958095709561957F4F8F4F04
:108E30009F4F6B307105810591053CF00E944CFA03
:108E4000AC01CB01DA016C017D01FFEFCF16FFEF22
:108E5000DF06FFEFEF06FFEFFF06B1F0F7FE02C0FF
:108E60000C9461550E944CFA6C197D0980E090E0E9
:108E70000F94740220E030E04AEF53E40F94D401E1
:108E8000882314F00C9461550E944CFA68197909F2
:108E90008A099B09695E73408040904008F0B7CE14
:108EA0003ACF82E795E00E9458E083E50E94AB3913
:108EB000882361F00E94FD390F9443027093100AD9
:108EC00060930F0A81E08093B2030FC082E50E9495
:108ED000AB39882351F00E94FD390F9443027093FF
:108EE000100A60930F0A1092B2030E944CFA7B01A1
:108EF0008C011092370860910F0A7091100A882730
:108F000077FD8095982F0F94760220911F0A30915B
:108F1000200A4091210A5091220A0F94E203181668
:108F20000CF082C081E0809337087EC00E944CFA2A
:108F30006E197F09800B910B695E734080409040F1
:108F400008F46BC0E0912808F0E0EE0FFF1FEE0F71
:108F5000FF1FEB5EF54F40815181628173819B2D34
:108F6000EFE6F5E008C08091C00085FFFCCF90934C
:108F7000C600319694919923B1F784E595E022E0FB
:108F800030E00E9462269C2DEBE6F5E008C080915F
:108F9000C00085FFFCCF9093C60031969491992331
:108FA000B1F76091280884E595E070E04AE050E070
:108FB0000E948F259D2DE7E6F5E008C08091C00056
:108FC00085FFFCCF9093C600319694919923B1F719
:108FD00040911F0A5091200A6091210A7091220A43
:108FE00084E595E021E030E00E946226EDE8F2E0C1
:108FF00007C08091C00085FFFCCF31969093C600DA
:1090000090819923B1F78091C00085FFFCCFA09299
:10901000C6000E944CFA7B018C010E9437630E94BB
:109020000A360E9435E10BC0EFE6F5E0B490EBE6BE
:10903000F5E0C490E7E6F5E0D490BAE0AB2E80917D
:10904000370820910F0A3091100A8823A9F0B9013E
:10905000882777FD8095982F0F94760220911F0A1C
:109060003091200A4091210A5091220A0F94E20384
:1090700018160CF45BCF18C0B901882777FD8095CE
:10908000982F0F94760220911F0A3091200A409168
:10909000210A5091220A0F94D40188232CF4809144
:1090A000B203882309F442CF8DE595E00E9458E091
:1090B0000E944CFA6093490870934A0880934B08C9
:1090C00090934C080C945E551092290880E50E94FC
:1090D000AB398823F1F00E94FD3920E030E040E018
:1090E00050E00F94D401882314F460E010C00E9473
:1090F000FD3920E030E040E85FE30F94E20318160A
:1091000014F461E004C00E94FD390F94480260939A
:10911000290880912908882389F583E50E94AB39C5
:10912000882321F10E94FD3920E030E040E050E04A
:109130000F94D40188231CF460E070E011C00E94F9
:10914000FD3920E030E04FE753E40F94E2031816B6
:109150001CF46FEF70E004C00E94FD390F944302CD
:1091600070932B0860932A080C945E558FEF90E063
:1091700090932B0880932A080C945E55813011F04F
:109180000C945E5583E50E94AB39882321F10E943F
:10919000FD3920E030E040E050E00F94D401882316
:1091A0001CF460E070E011C00E94FD3920E030E066
:1091B0004FE753E40F94E20318161CF46FEF70E0CE
:1091C00004C00E94FD390F94430270932D086093F0
:1091D0002C080C945E558FEF90E090932D088093AF
:1091E0002C080C945E551092290810922B081092AE
:1091F0002A0810922D0810922C080C945E559D9A06
:10920000A59881E08093B10389E495E00E9458E03D
:109210000E9435E10C945E550E94ED5D0E94776DD1
:10922000149A139A0E94856D10922B0810922A08A6
:1092300068EE73E080E090E00E945AFA9D9AA59A49
:109240001092B10387E395E00E9458E00E9435E157
:109250000C945E551092E6070C945E5581E0809365
:10926000E6070C945E5583E50E94AB398823A1F094
:109270000E94FD3920E030E04AE754E40F94B40442
:109280000F9448026093B3037093B4038093B503C3
:109290009093B6030C945E5588E50E94AB39882301
:1092A00011F00C947A5589E50E94AB39882311F0AE
:1092B0000C947A558AE50E94AB39882311F00C94FE
:1092C0007A5585E40E94AB39882311F00C947A55C5
:1092D0000E94776D149A139A0E94856D0C945E55C6
:1092E000179A1092110889E50E94AB39882319F06A
:1092F000169A109212088AE50E94AB39882319F059
:10930000159A1092130885E40E94AB39882311F452
:109310000C945E55149A139A0C945E5583E50E9442
:10932000AB390E94FD3920E030E04AE754E40F9465
:10933000B4040F94480260934D0870934E088093D4
:109340004F08909350080C945E55A0E16A2EADE052
:109350007A2EF0E02F2EFDE03F2EE0E54E2EEDE0E0
:109360005E2E88249924F401E25EFB4F80810E94E6
:10937000AB39882309F45DC043E0841609F052C07C
:109380000E94FD395B016C0120E030E040EA51E4CD
:109390000F94D40188230CF03FC0F30160817181E8
:1093A00082819381A60195010F94DB017B018C01E1
:1093B0006091480D7091490D80914A0D90914B0D2F
:1093C000A80197010F94B4046093480D7093490D60
:1093D00080934A0D90934B0DF101608171818281E0
:1093E0009381A80197010F94B404F1016083718304
:1093F00082839383F20160817181828193810F94D2
:109400007402A80197010F94B4040F944802F2016A
:109410006083718382839383F301A082B182C282CD
:10942000D38207C00E94FD39F30160837183828378
:1094300093830894811C911C24E030E0620E731E1B
:10944000220E331E420E531E34E08316910409F09F
:109450008ACF0C945E55ECE6F4E0949108C08091BC
:10946000C00085FFFCCF9093C6003196949199235C
:10947000B1F70C945E5580917C0890917D0805961B
:109480006AE270E00E945121FC01009711F03197CF
:10949000108280917C0890917D0805960E947AE068
:1094A0000C945E55E9E6F4E0949108C08091C00008
:1094B00085FFFCCF9093C600319694919923B1F724
:1094C0004091E9075091EA076091EB077091EC0732
:1094D00084E595E022E030E00E946226E6E6F4E0D2
:1094E000949108C08091C00085FFFCCF9093C60086
:1094F000319694919923B1F74091ED075091EE0781
:109500006091EF077091F00784E595E022E030E08C
:109510000E946226E3E6F4E0949108C08091C000C6
:1095200085FFFCCF9093C600319694919923B1F7B3
:109530004091F1075091F2076091F3077091F407A1
:1095400084E595E022E030E00E946226E0E6F4E067
:10955000949108C08091C00085FFFCCF9093C60015
:10956000319694919923B1F74091F5075091F60700
:109570006091F7077091F80784E595E022E030E00C
:109580000E946226E5E5F4E0949108C08091C00055
:1095900085FFFCCF9093C600319694919923B1F743
:1095A00080E00E94456B0F9476022091100D30915F
:1095B000110D4091120D5091130D0F94DB01AB0171
:1095C000BC0184E595E022E030E00E946226E2E5FD
:1095D000F4E0949108C08091C00085FFFCCF909387
:1095E000C600319694919923B1F781E00E94456BB2
:1095F0000F9476022091140D3091150D4091160DA7
:109600005091170D0F94DB01AB01BC0184E595E08F
:1096100022E030E00E946226EFE4F4E0949108C07A
:109620008091C00085FFFCCF9093C6003196949145
:109630009923B1F782E00E94456B0F947602209146
:10964000180D3091190D40911A0D50911B0D0F946A
:10965000DB01AB01BC0184E595E022E030E00E9433
:109660006226EDE8F2E007C08091C00085FFFCCFE4
:1096700031969093C60090819923B1F78091C000F4
:1096800085FFFCCF8AE08093C6000C945E5580E095
:109690000E94F16A0C945E5581E00E94F16A0C947C
:1096A0005E558091C00085FFFCCF31969093C60037
:1096B00090819923B1F78091C00085FFFCCF8AE0AB
:1096C0008093C600E7E4F4E0949108C08091C00064
:1096D00085FFFCCF9093C600319694919923B1F702
:1096E0001E9B03C0E0E9F2E00AC0E5E9F2E007C032
:1096F0008091C00085FFFCCF31969093C600908189
:109700009923B1F78091C00085FFFCCF8AE0809358
:10971000C600EFE3F4E0949108C08091C00085FF9B
:10972000FCCF9093C600319694919923B1F71D9B7D
:1097300003C0E0E9F2E00AC0E5E9F2E007C0809189
:10974000C00085FFFCCF31969093C600908199238D
:10975000B1F78091C00085FFFCCF8AE08093C600FE
:10976000E7E3F4E0949108C08091C00085FFFCCF4E
:109770009093C600319694919923B1F71C9B03C036
:10978000E0E9F2E00AC0E5E9F2E007C08091C0003C
:1097900085FFFCCF31969093C60090819923B1F755
:1097A0008091C00085FFFCCF8AE08093C6000C94B6
:1097B0005E5584E40E94AB39882311F40C945E5505
:1097C0000E94FD3920E030E040E05FE30F94B404F4
:1097D0007B018C0120E030E040E050E00F94D401A8
:1097E000882359F40F2EF0E0CF2EF0E0DF2EF0E8C2
:1097F000EF2EFFE3FF2EF02D11C0C801B701A80125
:1098000097010F94B4049B01AC01CA012BED3FE01A
:1098100049E450E40F94B4046B017C018091280862
:109820008093400884E50E94AB398823A1F10E940F
:10983000FD390F944802262F609340086230D8F01B
:10984000ECE2F3E0949108C08091C00085FFFCCF6A
:109850009093C600319694919923B1F7EFE9F2E025
:1098600007C08091C00085FFFCCF31969093C60061
:1098700090819923B1F784E595E0622F40E050E0B4
:109880000E944B258091C00085FFFCCF8AE0809329
:10989000C6000C945E5580914008082F10E0000F20
:1098A000111F000F111F03561C4F60E070E080E88D
:1098B0009FE3A70196010F94DB01F8016083718398
:1098C000828393830C945E550EE114E064E2E62EED
:1098D0006DE0F62EF80180810E94AB39882349F0B3
:1098E0000E94FD390F944802F701608371838283DF
:1098F00093830F5F1F4F24E030E0E20EF31E34E04D
:109900000232130739F70E94398A0C945E550EE132
:1099100014E050E0E52E5DE0F52EF80180810E9414
:10992000AB39882339F00E94FD39F70160837183D8
:10993000828393830F5F1F4F24E030E0E20EF31E1B
:1099400034E00232130749F70C945E5583E50E9418
:10995000AB39882351F00E94FD396093380D709324
:10996000390D80933A0D90933B0D84E50E94AB39FD
:10997000882311F40C945E550E94FD3960933C0DD0
:1099800070933D0D80933E0D90933F0D0C945E556A
:1099900083E50E94AB39882351F00E94FD39609322
:1099A000340D7093350D8093360D9093370D84E50B
:1099B0000E94AB39882351F00E94FD3960934C0D11
:1099C00070934D0D80934E0D90934F0D82E40E9445
:1099D000AB39882361F00E94FD390F9448026093EF
:1099E000FC0C7093FD0C8093FE0C9093FF0C88E5AB
:1099F0000E94AB39882351F00E94FD396093400DDD
:109A00007093410D8093420D9093430D8AE50E941F
:109A1000AB39882351F00E94FD396093440D709357
:109A2000450D8093460D9093470D85E40E94AB3918
:109A3000882311F40C945E550E94FD396093480D03
:109A40007093490D80934A0D90934B0D0C945E5585
:109A50000EE114E049EFE42E47E0F42EF801808196
:109A60000E94AB39882339F00E94FD39F7016083E9
:109A70007183828393830F5F1F4F24E030E0E20EF7
:109A8000F31E34E00132130749F70C945E558AED5A
:109A900090E00E94063A882311F00C945E5588E508
:109AA0000E94AB39882389F080914008082F10E08C
:109AB0000E94FD39000F111F000F111F085E174F84
:109AC000F801608371838283938389E50E94AB39B7
:109AD000882389F080914008082F10E00E94FD390A
:109AE000000F111F000F111F005E174FF801608358
:109AF000718382839383ECE2F3E0949108C08091B8
:109B0000C00085FFFCCF9093C600319694919923B5
:109B1000B1F7E7E2F4E0949108C08091C00085FFBE
:109B2000FCCF9093C600319694919923B1F710928F
:109B3000400840C08091C00085FFFCCF11969093F3
:109B4000C6009C919923B1F7F0E0EE0FFF1FEE0FD6
:109B5000FF1FE85EF74F408151816281738184E588
:109B600095E022E030E00E946226E6EBF2E007C0DA
:109B70008091C00085FFFCCF31969093C600908104
:109B80009923B1F7E0914008F0E0EE0FFF1FEE0FD0
:109B9000FF1FE05EF74F408151816281738184E550
:109BA00095E022E030E00E946226809140088F5FBD
:109BB00080934008E0914008E23018F0EDE8F2E0D0
:109BC0000AC0A8EBB2E0BDCF8091C00085FFFCCFFA
:109BD00031969093C60090819923B1F78091C0008F
:109BE00085FFFCCF8AE08093C60068C783E50E94AA
:109BF000AB39882309F462C70E94FD390F944302F0
:109C000070939A036093990359C783E50E94AB3917
:109C1000882309F453C70E94FD390F9443027093BF
:109C20009C0360939B034AC780E50E94AB3988235D
:109C300009F444C70E94FD390F9443027B0183E578
:109C40000E94AB39882319F40FEF1FEF05C00E9463
:109C5000FD390F9443028B01C8010196039708F068
:109C60002DC7E2E2F4E0808191818E159F0509F411
:109C700025C7329624E0E23AF207A9F7F7FC1EC79F
:109C80000E94776DDE2C8E2D60E00E94F3FB0115A3
:109C9000110541F00130110579F03FEF0F3F130737
:109CA000A1F403C000E010E010C08E2D0E94D8FC8B
:109CB00000E010E0892B49F401E010E006C00E94AA
:109CC00037630E940A360E9435E18D2D0E94D8FC30
:109CD00080179107A1F7F2C683E50E94AB3988236C
:109CE00021F41EE6C12ED12C05C00E94FD390F942F
:109CF00043026B0180E50E94AB39882319F468EEBA
:109D000073E004C00E94FD390F9443027B010027D9
:109D1000F7FC0095102F1C141D0484F48FE4B60189
:109D200020E030E040E050E00E940CFEC801B701A6
:109D30000E945AFA8FE40E9498FDC0C6C801B7017C
:109D40000E945AFABBC680E50E94AB39882351F0C5
:109D50000E94FD396093BC037093BD038093BE03E2
:109D60009093BF0389E40E94AB39882361F00E947D
:109D7000FD390E94115E6093C0037093C10380930C
:109D8000C2039093C30384E40E94AB39882361F03B
:109D90000E94FD390E941D5E6093C4037093C50349
:109DA0008093C6039093C70383E40E94AB39882352
:109DB00051F00E94FD396093C8037093C9038093EA
:109DC000CA039093CB030E94F85CEAEBF2E007C071
:109DD0008091C00085FFFCCF31969093C6009081A2
:109DE0009923B1F7EDEBF2E007C08091C00085FF49
:109DF000FCCF31969093C60090819923B1F74091A2
:109E0000BC035091BD036091BE037091BF0384E514
:109E100095E022E030E00E946226E1ECF2E007C02B
:109E20008091C00085FFFCCF31969093C600908151
:109E30009923B1F76091C0037091C1038091C2036F
:109E40009091C3030E94175EAB01BC0184E595E0CD
:109E500022E030E00E946226E5ECF2E007C080914B
:109E6000C00085FFFCCF31969093C6009081992366
:109E7000B1F76091C4037091C5038091C6039091BE
:109E8000C7030E94235EAB01BC0184E595E022E09C
:109E900030E00E946226E9ECF2E007C08091C00049
:109EA00085FFFCCF31969093C60090819923B1F73E
:109EB0004091C8035091C9036091CA037091CB03CC
:109EC00084E595E022E030E00E946226EDE8F2E0D1
:109ED00007C08091C00085FFFCCF31969093C600EB
:109EE00090819923B1F78091C00085FFFCCF8AE073
:109EF0008093C600E3C580E50E94AB39882351F00A
:109F00000E94FD396093CC037093CD038093CE0300
:109F10009093CF0389E40E94AB39882361F00E94BB
:109F2000FD390E94115E6093D0037093D10380933A
:109F3000D2039093D30384E40E94AB39882361F069
:109F40000E94FD390E941D5E6093D4037093D50377
:109F50008093D6039093D7030E94F85CEAEBF2E07B
:109F600007C08091C00085FFFCCF31969093C6005A
:109F700090819923B1F7EDEBF2E007C08091C0002A
:109F800085FFFCCF31969093C60090819923B1F75D
:109F90004091CC035091CD036091CE037091CF03DB
:109FA00084E595E022E030E00E946226E1ECF2E0F8
:109FB00007C08091C00085FFFCCF31969093C6000A
:109FC00090819923B1F76091D0037091D103809172
:109FD000D2039091D3030E94175EAB01BC0184E5CC
:109FE00095E022E030E00E946226E5ECF2E007C056
:109FF0008091C00085FFFCCF31969093C600908180
:10A000009923B1F76091D4037091D5038091D60361
:10A010009091D7030E94235EAB01BC0184E595E0DB
:10A0200022E030E00E946226EDE8F2E007C0809175
:10A03000C00085FFFCCF31969093C6009081992394
:10A04000B1F78091C00085FFFCCF8AE08093C60005
:10A0500035C583E40E94AB39882349F00E94FD395D
:10A060000F944302DC01CB018F730E944DE0E2E1CB
:10A07000F4E0949108C08091C00085FFFCCF9093DC
:10A08000C600319694919923B1F76091B9147091FB
:10A09000BA1484E595E04AE050E00E948F25EDE88F
:10A0A000F2E007C08091C00085FFFCCF319690930D
:10A0B000C60090819923B1F78091C00085FFFCCF45
:10A0C0008AE08093C600FAC483E50E94AB398823F6
:10A0D00029F460E070E080E090E002C00E94FD3969
:10A0E0000E94308AEBC485E40E94AB39882319F4BE
:10A0F000CC24DD2412C00E94FD390F9443026B0171
:10A1000077FF0BC00F2EF0E0EF2EF0E0FF2EFCE803
:10A110000F2FF2E41F2FF02D0AC00F2EF0E0EF2ECC
:10A12000F0E0FF2EF6E10F2FF3E41F2FF02D83E573
:10A130000E94AB39882321F00E94FD397B018C01FC
:10A1400083E40E94AB39882319F425E030E005C090
:10A150000E94FD390F9443029B01C801B701A6017B
:10A160000E944166ABC40E94776DA8C40E9460E75C
:10A17000A5C40E944EEFA2C40E9433EA9FC40E946D
:10A180000CEC9CC4A090E907B090EA07C090EB07E4
:10A19000D090EC07A982BA82CB82DC82E090ED07F6
:10A1A000F090EE070091EF071091F007ED82FE822C
:10A1B0000F8318872091F1073091F2074091F30740
:10A1C0005091F40729873A874B875C878091F50780
:10A1D0009091F607A091F707B091F8078D879E87B9
:10A1E000AF87B88BA98ABA8ACB8ADC8AED8AFE8AC5
:10A1F0000F8B188F298F3A8F4B8F5C8F8D8F9E8F8F
:10A20000AF8FB8A385E40E94AB39882369F0ED8451
:10A21000FE840F8518890E94FD399B01AC01C8019D
:10A22000B7010F94FB000AC06D857E858F859889E4
:10A2300020E030E040E050E40F94FA006D877E8724
:10A240008F87988B6091B7037091B8038091B903A1
:10A250009091BA0320E030E040E752E40F94DB0134
:10A260007B018C01CE010196BE016B5F7F4FAE0179
:10A27000475F5F4F9E01235F3F4FB8E2CB2EB8E0B0
:10A28000DB2E0E94F38F8AE50E94AB39882359F0B8
:10A29000E984FA840B851C850E94FD399B01AC0181
:10A2A000C801B70108C069857A858B859C8520E047
:10A2B00030E040E251E40F94FB0069877A878B8796
:10A2C0009C876091B7037091B8038091B903909116
:10A2D000BA0320E030E040E752E40F94DB017B0159
:10A2E0008C01CE010196BE016B5F7F4FAE01475FCF
:10A2F0005F4F9E01235F3F4FA8E2CA2EA8E0DA2EEF
:10A300000E94F38F88E50E94AB39882389F0E980A9
:10A31000FA800B811C810E94FD399B01AC01C801B0
:10A32000B7010F94FB0069837A838B839C8308C0F9
:10A3300080E090E0A0E4B0E489839A83AB83BC839F
:10A3400089E50E94AB39882339F00E94FD396D837D
:10A350007E838F83988708C080E090E0A0E4B0E41B
:10A360008D839E83AF83B8876091B7037091B803E4
:10A370008091B9039091BA0320E030E040E752E4C5
:10A380000F94DB017B018C01CE010196BE016B5F56
:10A390007F4FAE01475F5F4F9E01235F3F4FF8E263
:10A3A000CF2EF8E0DF2E0E94F38F8CE40E94AB39B1
:10A3B000882369F0ED84FE840F8518890E94FD3999
:10A3C0009B01AC01C801B7010F94FB000AC06D8569
:10A3D0007E858F85988920E030E048EC52E40F9428
:10A3E000FA006D877E878F87988B6091B703709195
:10A3F000B8038091B9039091BA0320E030E040E7C0
:10A4000052E40F94DB017B018C01CE010196BE0169
:10A410006B5F7F4FAE01475F5F4F9E01235F3F4FF2
:10A42000E8E2CE2EE8E0DE2E0E94F38F0E94776DE8
:10A43000149A139A64E670E080E090E00E945AFA61
:10A4400082E094E00E9467E010E018C01F5F0E9465
:10A4500037630E940A360E9435E1112379F46E9A1F
:10A46000769A63E070E080E090E00E945AFA769875
:10A4700063E070E080E090E00E945AFA0E94959CB0
:10A48000882321F38CE40E94AB39882369F0ED84A2
:10A49000FE840F8518890E94FD399B01AC01C8011B
:10A4A000B7010F94FA000AC06D857E858F85988963
:10A4B00020E030E048EC52E40F94FB006D877E878B
:10A4C0008F87988B8D859E85AF85B8898093F5079A
:10A4D0009093F607A093F707B093F80785EF97E0FE
:10A4E0000E94648AB9E04B2E512C4C0E5D1EADE0EB
:10A4F0006A2E712C6C0E7D1E6091B7037091B803AB
:10A500008091B9039091BA0320E030E040E752E433
:10A510000F94DB017B018C01CE010196BE016B5FC4
:10A520007F4FA2019301F8E2CF2EF8E0DF2E0E94C8
:10A53000F38FE1E1AE2EB12CAC0EBD1E75E1872E7E
:10A54000912C8C0E9D1E6091B7037091B803809181
:10A55000B9039091BA0320E030E040E752E40F9451
:10A56000DB017B018C01C501B401A20193010E94B2
:10A57000F38F69E1462E512C4C0E5D1E6091B7039E
:10A580007091B8038091B9039091BA0320E030E054
:10A5900040E752E40F94DB017B018C01C501B4015B
:10A5A000A20193010E94F38F6091B7037091B803E9
:10A5B0008091B9039091BA0320E030E040E752E483
:10A5C0000F94DB017B018C01C501B401A2019E0146
:10A5D000235E3F4F0E94F38F71C200E010E0F8014C
:10A5E000E25EFB4F80810E94AB39882351F00E94CC
:10A5F000FD390F9443029B01AC01802FB9010E94E9
:10A60000C96C0F5F1F4F0430110549F782E40E94A7
:10A61000AB39882351F00E94FD390F9443029B010E
:10A62000AC0184E0B9010E94C96C83E50E94AB399A
:10A63000882309F443C210E00E94FD390F944302BD
:10A640009B01AC01812FB9010E94C96C1F5F1530BD
:10A6500099F734C280E50E94AB39882329F00E9423
:10A66000FD390F944802162F83E50E94AB398823E9
:10A6700021F00E94FD390F944802812F90E070E094
:10A680000E94B06C1BC283E50E94AB39882319F489
:10A6900000E010E00FC010E00E94FD390F94480266
:10A6A0009B01AC01812F622F0E94946C1F5F1530BB
:10A6B00099F7EECFF801E25EFB4F80810E94AB3943
:10A6C000882351F00E94FD390F9448029B01AC0190
:10A6D000802F622F0E94946C0F5F1F4F0430110572
:10A6E00049F782E40E94AB39882351F00E94FD397A
:10A6F0000F9448029B01AC0184E0622F0E94946C8D
:10A700000E947A6BDBC183E50E94AB39882309F490
:10A710005FC00E94FD390F9443026130710529F03A
:10A720006230710509F054C029C000E010E0F80162
:10A73000E25EFB4F80810E94AB39882359F00E9472
:10A74000FD390F9443029B01AC01802F622F4FEF24
:10A750000E94566C0F5F1F4F0430110541F782E4D1
:10A760000E94AB398823A1F10E94FD390F94430266
:10A770009B01AC0184E0622F4FEF28C000E010E0A5
:10A78000F801E25EFB4F80810E94AB39882359F0CB
:10A790000E94FD390F9443029B01AC01802F6FEFA3
:10A7A000422F0E94566C0F5F1F4F0430110541F776
:10A7B00082E40E94AB39882359F00E94FD390F943E
:10A7C00043029B01AC0184E06FEF422F0E94566C64
:10A7D0000E947A6B73C1109236080E94929C8091FD
:10A7E000450890914608A0914708B0914808809389
:10A7F000410890934208A0934308B09344080E94F4
:10A80000F0375CC184E50E94AB39882309F40BC1A1
:10A810000E94FD390F944802262F60934008623051
:10A82000B8F1ECE2F3E0949108C08091C00085FF9C
:10A83000FCCF9093C600319694919923B1F7EDEC3B
:10A84000F2E007C08091C00085FFFCCF3196909365
:10A85000C60090819923B1F784E595E0622F40E02E
:10A8600050E00E944B25EFECF2E007C08091C00061
:10A8700085FFFCCF31969093C60090819923B1F764
:10A880008091C00085FFFCCF8AE08093C60016C18E
:10A8900086E40E94AB39882311F4EE241EC00E9486
:10A8A000FD397B018C0160936E0870936F08809373
:10A8B00070089093710820E030E040E050E00F9481
:10A8C000E203181644F4E092B703F092B803009341
:10A8D000B9031093BA03EE24E39490914008809159
:10A8E0002808981709F473C0ADE5B8E0E9EEF7E081
:10A8F00080E101900D928150E1F720912808C22E4D
:10A90000DD24CC0CDD1CCC0CDD1CF601E85EF74F21
:10A910006091E9077091EA078091EB079091EC074D
:10A9200020813181428153810F94FA00F0904008D8
:10A930000F2D10E0000F111F000F111FF801E85E2E
:10A94000F74F20813181428153810F94FB00609346
:10A95000E9077093EA078093EB079093EC0740E2D6
:10A9600058E0C40ED51E6091ED077091EE078091FE
:10A97000EF079091F007F6012081318142815381E8
:10A980000F94FA00005E174FF80120813181428157
:10A9900053810F94FB006093ED077093EE07809353
:10A9A000EF079093F007F092280889EE97E06DEE9C
:10A9B00077E041EF57E025EF37E00E94948AEE20E0
:10A9C00031F080913608882311F40E942F37ECE291
:10A9D000F3E0949108C08091C00085FFFCCF909374
:10A9E000C600319694919923B1F7E0EEF2E007C0EA
:10A9F0008091C00085FFFCCF31969093C600908176
:10AA00009923B1F76091280884E595E070E04AE069
:10AA100050E00E948F258091C00085FFFCCF8AE026
:10AA20008093C6004BC0ECE2F3E0949108C08091A3
:10AA3000C00085FFFCCF9093C60031969491992376
:10AA4000B1F7EFEEF3E0949108C08091C00085FF6C
:10AA5000FCCF9093C600319694919923B1F7209141
:10AA600072083091730880E690E0289FF001299FDA
:10AA7000F00D389FF00D1124E258F74F07C0809178
:10AA8000C00085FFFCCF31969093C600908199233A
:10AA9000B1F7EDEEF3E0949108C08091C00085FF1E
:10AAA000FCCF9093C600319694919923B1F7809191
:10AAB000C00085FFFCCF8AE08093C6000E948635E7
:10AAC00024C08FE795E00E9458E00E944CFA609302
:10AAD0002E0870932F0880933008909331080E94BD
:10AAE0004CFA6093490870934A0880934B089093FE
:10AAF0004C08E4CF0E94776D88E50E94AB3988232B
:10AB000011F00C9470490C947349EE960FB6F894BA
:10AB1000DEBF0FBECDBFCF91DF911F910F91FF9090
:10AB2000EF90DF90CF90BF90AF909F908F907F90ED
:10AB30006F905F904F903F902F9008952F923F928B
:10AB40004F925F926F927F928F929F92AF92BF923D
:10AB5000CF92DF92EF92FF920F931F93DF93CF93E9
:10AB6000CDB7DEB76E970FB6F894DEBF0FBECDBF80
:10AB700080E6A82EB12CE3E9F6E084900AE0702E7E
:10AB8000E9E0F7E094906624639413C22D3071F0ED
:10AB90002A3321F48091FF09882341F08091000A33
:10ABA0009091010A8F3591050CF4DFC1E091000A04
:10ABB000F091010A309709F404C3A091020AB09100
:10ABC000030AAA9D7001AB9DF00CBA9DF00C1124F4
:10ABD000EE0DFF1DE258F74F10828091FF09882388
:10ABE00009F0BEC11092FF09AC58B74F1C92870103
:10ABF0000258174FC8016EE470E00E9451219C0179
:10AC0000009709F4F7C090937D0880937C082F5F2C
:10AC10003F4F201B310B2E0D3F1DC9018258974F0E
:10AC200060E070E04AE050E00E94B01F6093040AC8
:10AC30007093050A8093060A9093070AC090410812
:10AC4000D0904208E0904308F0904408A701960194
:10AC50002F5F3F4F4F4F5F4F621773078407950772
:10AC600009F457C38091020A9091030A9C012A9D1E
:10AC7000C0012B9D900D3A9D900D11248258974F45
:10AC800062EB77E00E941621892B09F042C3E2E3D0
:10AC9000F3E0949108C08091C00085FFFCCF9093B1
:10ACA000C600319694919923B1F7EFE7F7E09491BC
:10ACB00008C08091C00085FFFCCF9093C6003196FC
:10ACC00094919923B1F784E595E0B701A6012AE0B4
:10ACD00030E00E945C258091C00085FFFCCF73C0EE
:10ACE000FE264F5FFC01E40FF11DE258F74FE081B3
:10ACF000EA32B1F730937D0820937C08C9010196B0
:10AD000060E070E00E94531E0F9443022F2D30E04C
:10AD10002617370709F45DC0E2E3F3E0949108C019
:10AD20008091C00085FFFCCF9093C600319694912E
:10AD30009923B1F7E0E6F7E0949108C08091C00054
:10AD400085FFFCCF9093C600319694919923B1F77B
:10AD50004091410850914208609143087091440825
:10AD600084E595E02AE030E00E945C258091C000F7
:10AD700085FFFCCF28C0E2E3F3E0949108C0809106
:10AD8000C00085FFFCCF9093C60031969491992323
:10AD9000B1F7E6E3F7E0949108C08091C00085FF29
:10ADA000FCCF9093C600319694919923B1F784E536
:10ADB00095E0B701A6012AE030E00E945C25809171
:10ADC000C00085FFFCCF8AE08093C6000E94F03768
:10ADD0004AC08091040A9091050AA091060AB09198
:10ADE000070A8093410890934208A0934308B093C8
:10ADF00044083EC0C8016AE270E00E9451210097F9
:10AE000009F436C0E2E3F3E0949108C08091C000F9
:10AE100085FFFCCF9093C600319694919923B1F7AA
:10AE2000ECE0F7E0949108C08091C00085FFFCCF72
:10AE30009093C600319694919923B1F740914108BF
:10AE400050914208609143087091440884E595E070
:10AE50002AE030E00E945C258091C00085FFFCCF95
:10AE60008AE08093C6001092010A1092000A70C214
:10AE70008091020A9091030A8A9D70018B9DF00CCB
:10AE80009A9DF00C112487010258174FC80167E4FE
:10AE900070E00E9451219C01009709F44BC09093EF
:10AEA0007D0880937C082F5F3F4F201B310B2E0DB8
:10AEB0003F1DC9018258974F60E070E00E94531E09
:10AEC0000F94430264307105A8F5809136088823F9
:10AED000C9F480915505882369F5992DE9E0F7E0DB
:10AEE00008C08091C00085FFFCCF9093C6003196CA
:10AEF00094919923B1F78091C00085FFFCCF7092A7
:10AF0000C60018C0982DE3E9F6E008C08091C000A3
:10AF100085FFFCCF9093C600319694919923B1F7A9
:10AF20008091C00085FFFCCF7092C60089E896E052
:10AF30000E9458E08091020A9091030A019664E011
:10AF400070E00F94B9059093030A8093020A8091F0
:10AF5000080A9091090A01969093090A8093080AB9
:10AF60001092010A1092000A24C02B3311F460924F
:10AF7000FF098091FF098823E1F42091000A3091B4
:10AF8000010A8091020A9091030A8A9DF0018B9D2B
:10AF9000F00D9A9DF00D1124E20FF31FE258F74FC8
:10AFA0008091FE0980832F5F3F4F3093010A2093E9
:10AFB000000A8091500590915105209152053091E1
:10AFC0005305821B930B8F779070892B09F4BBC1BB
:10AFD0008091080A9091090A04970CF0B4C184E5A5
:10AFE00095E00E948024282F8093FE098A3009F082
:10AFF000CDCDDCCD8091000A9091010A892B09F01A
:10B00000A7C18091080A9091090A892B09F02FC1E4
:10B0100010920A0A2CC14D3099F0433211F04A3394
:10B0200021F48091FF09882359F08091000A9091C2
:10B03000010A8F35910524F42F5F3F4F09F0F2C0CC
:10B040002091D8073091D9074091DA075091DB075A
:10B050008091D0079091D107A091D207B091D307EA
:10B06000281739074A075B0708F49EC0932DE6E7C7
:10B07000F6E008C08091C00085FFFCCF9093C60029
:10B08000319694919923B1F78091C00085FFFCCF50
:10B090002092C6000E944CFA6093320870933308E5
:10B0A000809334089093350820912E0830912F0812
:10B0B0004091300850913108621B730B840B950B43
:10B0C00028EE33E040E050E00F94CC05F22EE32E62
:10B0D000D42EC52EEDB7FEB738970FB6F894FEBF45
:10B0E0000FBEEDBF0DB71EB70F5F1F4FB282A1821B
:10B0F000F80153824282622F732F842F952F20E113
:10B100003EE040E050E00F94CC05F8013583248305
:10B110006F2D7E2D8D2D9C2D2CE330E040E050E0F6
:10B120000F94CC05CA01B9012CE330E040E050E0B7
:10B130000F94CC05F801778366830E948021982DB7
:10B14000ECE2F3E02DB73EB7285F3F4F0FB6F8941F
:10B150003EBF0FBE2DBF08C08091C00085FFFCCF51
:10B160009093C600319694919923B1F7F50107C0E9
:10B170008091C00085FFFCCF31969093C6009081EE
:10B180009923B1F78091C00085FFFCCF2092C600C3
:10B19000C5010E947AE085E595E00E94B92D85E51C
:10B1A00095E061E00E941E2F8091FE09833211F428
:10B1B00090920A0A2091000A3091010A2115310566
:10B1C00019F41092FF09C4C08091020A9091030AF9
:10B1D000869DF001879DF00D969DF00D1124E20FE4
:10B1E000F31FE258F74F1082FC01EC58F74F9082A2
:10B1F0002091080A3091090A2F5F3F4F3093090AC6
:10B200002093080A019664E070E00F94B9059093CA
:10B21000030A8093020A1092FF091092010A109209
:10B22000000A3AC04B3311F49092FF098091FF0954
:10B23000882391F52091000A3091010A8091020A39
:10B240009091030A869DF001879DF00D969DF00D6B
:10B250001124E20FF31FE258F74F8091FE0980831B
:10B260002F5F3F4F3093010A2093000A15C010E66C
:10B27000612E712C99249394E6E7F6E03490BAE0BD
:10B280002B2E5E010894A11CB11CA2E64A2EA6E05A
:10B290005A2EECE2F3E084902091D8073091D90740
:10B2A0004091DA075091DB078091D0079091D10748
:10B2B000A091D207B091D307281739074A075B0737
:10B2C00008F046C08091080A9091090A04970CF092
:10B2D0003FC080910A0A8823D9F580912B0790916D
:10B2E0002C07A0912D07B0912E078093D80790933B
:10B2F000D907A093DA07B093DB0783E297E00E94B7
:10B30000C2839C01482F8093FE098A3009F083CEC6
:10B3100097CE8091020A9091030A8A9D80018B9DAD
:10B32000100D9A9D100D1124C8018258974F6AE2A2
:10B3300070E00E9451219C01009709F41CCDFF246C
:10B3400040E0C801CFCC80915705882309F052CE48
:10B350006E960FB6F894DEBF0FBECDBFCF91DF91D2
:10B360001F910F91FF90EF90DF90CF90BF90AF9023
:10B370009F908F907F906F905F904F903F902F9015
:10B380000895CF93DF938091080A9091090A03975B
:10B390000CF4D4DB85E595E060E00E941E2F8091DF
:10B3A000080A9091090A892B09F46AC08091550511
:10B3B000882309F44DC0209172083091730880E60B
:10B3C00090E0289FE001299FD00D389FD00D1124D7
:10B3D000C258D74FCE016CEC77E00E941621892B22
:10B3E000E1F485E595E0BE010E94B4278091560501
:10B3F000882371F5E9ECF7E0949108C08091C000D2
:10B4000085FFFCCF9093C600319694919923B1F7B4
:10B410008091C00085FFFCCF17C085E595E060E016
:10B420000E949B27E7EBF7E0949108C08091C00051
:10B4300085FFFCCF9093C600319694919923B1F784
:10B440008091C00085FFFCCF8AE08093C60002C0D7
:10B450000E94373B8091080A9091090A01979093C6
:10B46000090A8093080A80917208909173080196E6
:10B4700064E070E00F94B9059093730880937208AC
:10B480000E9437630E940A360E943A740E9435E196
:10B49000DF91CF910895DF93CF930F920F92CDB7A5
:10B4A000DEB70E9446359D9AA59884E595E040E078
:10B4B00052EC61E070E00E944824E7EBF8E09491E0
:10B4C00008C08091C00085FFFCCF9093C6003196E4
:10B4D00094919923B1F78091C00085FFFCCF8AE059
:10B4E0008093C6004CE253E0FA01949108C0809129
:10B4F000C00085FFFCCF9093C600319694919923AC
:10B50000B1F784B7282F80FF15C0EFEAF8E09491D7
:10B5100008C08091C00085FFFCCF9093C600319693
:10B5200094919923B1F78091C00085FFFCCF8AE008
:10B530008093C60021FF15C0EFE9F8E0949108C0A0
:10B540008091C00085FFFCCF9093C6003196949106
:10B550009923B1F78091C00085FFFCCF8AE08093EA
:10B56000C60022FF15C0EEE8F8E0949108C0809173
:10B57000C00085FFFCCF9093C6003196949199232B
:10B58000B1F78091C00085FFFCCF8AE08093C600B0
:10B5900023FF15C0EEE7F8E0949108C08091C00049
:10B5A00085FFFCCF9093C600319694919923B1F713
:10B5B0008091C00085FFFCCF8AE08093C60025FF04
:10B5C00015C0EEE6F8E0949108C08091C00085FFB8
:10B5D000FCCF9093C600319694919923B1F7809156
:10B5E000C00085FFFCCF8AE08093C60014BEE6E66B
:10B5F000F8E0949108C08091C00085FFFCCF909343
:10B60000C600319694919923B1F7E0E6F8E0949161
:10B6100008C08091C00085FFFCCF9093C600319692
:10B6200094919923B1F78091C00085FFFCCF8AE007
:10B630008093C600FA019491ECE2F3E008C0809197
:10B64000C00085FFFCCF9093C6003196949199235A
:10B65000B1F7E0E5F8E0949108C08091C00085FF63
:10B66000FCCF9093C600319694919923B1F7EBE308
:10B67000F8E0949108C08091C00085FFFCCF9093C2
:10B68000C600319694919923B1F7EFE2F8E09491D6
:10B6900008C08091C00085FFFCCF9093C600319612
:10B6A00094919923B1F7EDE0F8E0949108C080916E
:10B6B000C00085FFFCCF9093C600319694919923EA
:10B6C000B1F78091C00085FFFCCF8AE08093C6006F
:10B6D000E2E0F8E0949108C08091C00085FFFCCFC3
:10B6E0009093C600319694919923B1F7E6EFF7E075
:10B6F000949108C08091C00085FFFCCF9093C60054
:10B70000319694919923B1F78091C00085FFFCCFC9
:10B710008AE08093C600FA019491ECE2F3E008C05D
:10B720008091C00085FFFCCF9093C6003196949124
:10B730009923B1F7E7EEF7E0949108C08091C0003B
:10B7400085FFFCCF9093C600319694919923B1F771
:10B750002091251630912616CE010196211531052E
:10B7600019F48B52964102C0821B930B9A838983F2
:10B7700069817A8184E595E04AE050E00E948F2556
:10B78000E0EDF7E0949108C08091C00085FFFCCF08
:10B790009093C600319694919923B1F784E595E092
:10B7A00060E175E04AE050E00E948F258091C00082
:10B7B00085FFFCCF8AE08093C60010927408109237
:10B7C000750810927608109277080E944EEFD2D535
:10B7D0000E94368D0E94116D0E943DE280E197E249
:10B7E00020E931E0F9013197F1F70197D9F76C9A27
:10B7F00082E062E80E94A6FC82E062E870E00E94BB
:10B8000015FB0F900F90CF91DF910895BC018091AF
:10B81000080A9091090A04970CF070C02091020A5E
:10B820003091030A80E690E0AC01249FC001259F7F
:10B83000900D349F900D11248258974F0E94DF2065
:10B84000ECE2F3E0949108C08091C00085FFFCCF4A
:10B850009093C600319694919923B1F7EFEBF8E0FD
:10B86000949108C08091C00085FFFCCF9093C600E2
:10B87000319694919923B1F72091020A3091030AED
:10B8800080E690E0289FF001299FF00D389FF00D91
:10B890001124E258F74F07C08091C00085FFFCCF0C
:10B8A00031969093C60090819923B1F7EDEBF8E0C3
:10B8B000949108C08091C00085FFFCCF9093C60092
:10B8C000319694919923B1F78091C00085FFFCCF08
:10B8D0008AE08093C600C901019664E070E00F948D
:10B8E000B9059093030A8093020A8091080A909107
:10B8F000090A01969093090A8093080A0895BC01E9
:10B900008091080A9091090A04970CF070C0209168
:10B91000020A3091030A80E690E0AC01249FC00146
:10B92000259F900D349F900D11248258974F0E94AF
:10B930005C21ECE2F3E0949108C08091C00085FFA7
:10B94000FCCF9093C600319694919923B1F7ECEC1B
:10B95000F8E0949108C08091C00085FFFCCF9093DF
:10B96000C600319694919923B1F72091020A309143
:10B97000030A80E690E0289FF001299FF00D389F90
:10B98000F00D1124E258F74F07C08091C00085FFE9
:10B99000FCCF31969093C60090819923B1F7EAECE1
:10B9A000F8E0949108C08091C00085FFFCCF90938F
:10B9B000C600319694919923B1F78091C00085FF1C
:10B9C000FCCF8AE08093C600C901019664E070E074
:10B9D0000F94B9059093030A8093020A8091080A94
:10B9E0009091090A01969093090A8093080A089594
:10B9F00060E070E08CE593E42091C0033091C103D6
:10BA00004091C2035091C3030F94DB01DC019B0101
:10BA1000AC012093490A30934A0A40934B0A509351
:10BA20004C0ACB0180934D0A90934E0AA0934F0A83
:10BA3000B093500A60E070E08CE593E42091D0036D
:10BA40003091D1034091D2035091D3030F94DB0185
:10BA50006093550A7093560A8093570A9093580A38
:10BA60000895FC0197FF03C08091230A03C0EC5D99
:10BA7000F54F808190E008952F923F924F925F9210
:10BA80006F927F928F929F92AF92BF92CF92DF92EE
:10BA9000EF92FF920F931F93CF93DF93EC0121E07E
:10BAA00030E0A901440F551F440F551FFA01E65419
:10BAB000F64F85919491C817D9070CF059C0B90178
:10BAC00061507040660F771F660F771FCB0184545B
:10BAD000964FFC01059114916654764FFB01C59079
:10BAE000D490FA01E454F64FE590F490FA01E6544C
:10BAF000F64FA590B490B801882777FD8095982FD0
:10BB00000F9476021B012C01CC19DD09BE01882798
:10BB100077FD8095982F0F9476023B014C01E01A37
:10BB2000F10A0027F7FC0095102FC801B7010F9408
:10BB300076029B01AC01C401B3010F94B4047B01F4
:10BB40008C01AC18BD08CC24B7FCC094DC2CC60119
:10BB5000B5010F9476029B01AC01C801B7010F94A7
:10BB6000DB019B01AC01C201B1010F94FB0019C0C4
:10BB7000822F8F5F2F5F3F4F2A33310509F091CF1E
:10BB80008A3329F0E0E070E080E060E00CC0E0EA99
:10BB9000FAE065917491882777FD8095982F0F942E
:10BBA0007602E62F692F2E2F372F482F562FB901F7
:10BBB000CA01DF91CF911F910F91FF90EF90DF901D
:10BBC000CF90BF90AF909F908F907F906F905F903D
:10BBD0004F903F902F900895089510920C0A109264
:10BBE0000B0A1092240A9FB7F894E2E0F1E08081FA
:10BBF0008F7B80839FBF10920E0A10920D0A1092C5
:10BC0000250A9FB7F894E2E0F1E080818F7E80837F
:10BC10009FBF1092100A10920F0A1092230A759873
:10BC200008952DEB37E346E05EE30D94B4042DEB6D
:10BC300037E346E05EE30D94DB012DEB37E346E0AE
:10BC40005EE30D94DB012DEB37E346E05EE30D94FC
:10BC5000B40475980E946234882339F5E7EDF8E062
:10BC6000949108C08091C00085FFFCCF9093C600DE
:10BC7000319694919923B1F7EFEEF8E0949108C0D2
:10BC80008091C00085FFFCCF9093C60031969491BF
:10BC90009923B1F78091C00085FFFCCF8AE08093A3
:10BCA000C6008EED98E00E9467E00C9404351F9367
:10BCB000182F93DF0E946234882309F036C0E7ED25
:10BCC000F8E0949108C08091C00085FFFCCF90936C
:10BCD000C600319694919923B1F784E595E0612FE0
:10BCE00070E04AE050E00E948F258091C00085FFFF
:10BCF000FCCF8AE08093C600E6E3F9E0949108C0A7
:10BD00008091C00085FFFCCF9093C600319694913E
:10BD10009923B1F78091C00085FFFCCF8AE0809322
:10BD2000C60089E299E00E9467E00E9404351F91F5
:10BD300008951F93182F51DF0E946234882309F061
:10BD400036C0E7EDF8E0949108C08091C00085FF0F
:10BD5000FCCF9093C600319694919923B1F784E576
:10BD600095E0612F70E04AE050E00E948F258091BD
:10BD7000C00085FFFCCF8AE08093C600E0E7F9E0D1
:10BD8000949108C08091C00085FFFCCF9093C600BD
:10BD9000319694919923B1F78091C00085FFFCCF33
:10BDA0008AE08093C60083E699E00E9467E00E94E3
:10BDB00004351F9108951F920F920FB60F920BB684
:10BDC0000F9211242F933F934F935F936F937F9321
:10BDD0008F939F93AF93BF93EF93FF932091DC03D7
:10BDE000222389F58091240A80932F0A882331F039
:10BDF0009FB7F89480910201806405C09FB7F894C2
:10BE0000809102018F7B809302019FBF8091250A60
:10BE100080932E0A882331F09FB7F8948091020115
:10BE2000806105C09FB7F894809102018F7E809356
:10BE300002019FBF8091230A80932D0A882311F06D
:10BE4000759A01C0759880912F0A821740F49FB7A8
:10BE5000F894809102018F7B809302019FBF8091B3
:10BE60002E0A821740F49FB7F894809102018F7ECA
:10BE7000809302019FBF80912D0A821708F4759864
:10BE80002F5F2F772093DC038091DD03843009F44A
:10BE90006FC0853050F4813019F1813098F08230D4
:10BEA000E9F1833009F09CC047C0863009F48AC0AC
:10BEB000863008F46BC0873009F488C0883009F0F8
:10BEC0008FC08CC010927B0080E480937C008091B6
:10BED0007A00806480937A000E94DD9F81E01BC01D
:10BEE0008091780090917900A0E0B0E020913C0A28
:10BEF00030913D0A40913E0A50913F0A280F391F68
:10BF00004A1F5B1F20933C0A30933D0A40933E0A30
:10BF100050933F0A82E08093DD0362C010927B0061
:10BF200082E480937C0080917A00806480937A0020
:10BF30000E94DD9F83E0EFCF80917800909179009F
:10BF4000A0E0B0E02091300A3091310A4091320AED
:10BF50005091330A280F391F4A1F5B1F2093300A64
:10BF60003093310A4093320A5093330A84E0D3CF9E
:10BF700010927B0081E480937C0080917A00806441
:10BF800080937A000E94DD9F85E0C5CF8091780084
:10BF900090917900A0E0B0E02091380A3091390A00
:10BFA00040913A0A50913B0A280F391F4A1F5B1FE4
:10BFB0002093380A3093390A40933A0A50933B0A47
:10BFC00086E0A9CF0E94DD9F87E0A5CF1092DD0318
:10BFD0008091400A8F5F8093400A02C01092DD0377
:10BFE0008091400A803108F485C08091260A882318
:10BFF000C1F480913C0A90913D0A9093120A80937B
:10C00000110A8091380A9091390A9093140A80930A
:10C01000130A8091300A9091310A90931E0A8093FE
:10C020001D0A81E08093260A1092400A10923C0A71
:10C0300010923D0A10923E0A10923F0A1092380A5E
:10C040001092390A10923A0A10923B0A1092340A5E
:10C050001092350A1092360A1092370A1092300A5E
:10C060001092310A1092320A1092330A2091110A6A
:10C070003091120A8091270A9091280A821793071B
:10C0800014F080E056DE2091110A3091120A80915E
:10C09000D8039091D9032817390714F080E007DE00
:10C0A0002091130A3091140A8091290A90912A0A4A
:10C0B0008217930714F081E03CDE2091130A30913F
:10C0C000140A8091DA039091DB032817390714F0E2
:10C0D00081E0EDDD20911D0A30911E0A80912B0A2E
:10C0E00090912C0A821793072CF01092100A10924C
:10C0F0000F0AAFDDFF91EF91BF91AF919F918F91AB
:10C100007F916F915F914F913F912F910F900BBE57
:10C110000F900FBE0F901F9018952F926F927F92E5
:10C120008F929F92AF92BF92CF92DF92EF92FF9247
:10C130000F931F93DF93CF93CDB7DEB729970FB639
:10C14000F894DEBF0FBECDBF8C01E62E61E06E1508
:10C1500068F5E7EDF8E0949108C08091C00085FF94
:10C16000FCCF9093C600319694919923B1F784E562
:10C1700095E06E2D70E04AE050E00E948F25EDE9D9
:10C18000F9E0949108C08091C00085FFFCCF9093A6
:10C19000C600319694919923B1F78091C00085FF34
:10C1A000FCCF8AE08093C6000E944C35AE2DB0E0F3
:10C1B000FD01EE0FFF1FEE59FB4F808191819987A2
:10C1C0008887892B09F49FC0AA59BB4F9C919B83F8
:10C1D0002224239479C0222D30E0A901440F551F59
:10C1E000440F551FE885F985E40FF51F859194915B
:10C1F000081719070CF067C0C9010197880F991F2C
:10C20000880F991FFC013296A885B985EA0FFB1F9C
:10C21000C590D4908A0F9B1FFC01659174917A831D
:10C220006983FA013296EA0FFB1FE590F490FD0155
:10C23000E40FF51FA590B490B601882777FD80958F
:10C24000982F0F9476026C837D838E839F838981E0
:10C250009A81081B190BB801882777FD8095982FC4
:10C260000F9476023B014C01EC18FD080027F7FC07
:10C270000095102FC801B7010F9476029B01AC0105
:10C28000C401B3010F94B4047B018C01A981BA816C
:10C29000AA1ABB0ACC24B7FCC094DC2CC601B50199
:10C2A0000F9476029B01AC01C801B7010F94DB012A
:10C2B0009B01AC016C817D818E819F810F94FB007D
:10C2C000E62F692F09C02394BB812B1608F483CF76
:10C2D000E0E070E080E060E0FB812F1679F5E22D70
:10C2E000F0E0EE0FFF1FEE0FFF1F32976885798594
:10C2F000E60FF71F65917491882777FD8095982F39
:10C300000F94760219C0B801882777FD8095982F81
:10C310000F94760220E030E04AEF5EE30F94B4041D
:10C3200020E030E040E85DE30F94B40420E030E02A
:10C3300040E050E00F94FB00E62F692F2E2F372F9F
:10C34000482F562FB901CA0129960FB6F894DEBFBF
:10C350000FBECDBFCF91DF911F910F91FF90EF9056
:10C36000DF90CF90BF90AF909F908F907F906F9015
:10C370002F9008958F929F92AF92BF92CF92DF92AB
:10C38000EF92FF920F931F93CF93DF9360E070E0E3
:10C390008CE593E42091C0033091C1034091C20326
:10C3A0005091C3030F94DB017B018C0160E070E0CE
:10C3B0008CE593E42091D0033091D1034091D203D6
:10C3C0005091D3030F94DB01E091DE03F091DF0382
:10C3D0000F2EF0E0AF2EF0E0BF2EF0E0CF2EF0E019
:10C3E000DF2EF02DA092410AB092420AC092430A79
:10C3F000D092440A9701402F512F2093490A30933D
:10C400004A0A40934B0A50934C0AF093E103E0939D
:10C41000E003A092450AB092460AC092470AD09221
:10C42000480A20934D0A30934E0A40934F0A509386
:10C43000500AAC01CB01DA018093550A9093560A59
:10C44000A093570AB093580AA092510AB092520A88
:10C45000C092530AD092540A809101018064809363
:10C460000101809101018061809301016D9A8091A9
:10C4700001018860809301018091010180628093B5
:10C48000010186E061E070E00E94653488E061E0CF
:10C4900070E00E94653487ED80937A0010927E00F0
:10C4A00010927D0080917E00816080937E0080915B
:10C4B0007E00826080937E0080917E008460809305
:10C4C0007E0080E888BD80916E00846080936E005D
:10C4D0006AEF70E080E090E00E945AFA85E090E018
:10C4E00090935A0A8093590A09C08091D803909179
:10C4F000D90340979093D9038093D8038091D803B0
:10C500009091D90360E009DE20E030E040EA50E499
:10C510000F94D40187FDE9CF81E391E09093DF038D
:10C520008093DE0309C08091270A9091280A4096E3
:10C530009093280A8093270A8091270A9091280ACD
:10C5400060E0EBDD20E030E848E953E40F94E203DB
:10C5500018164CF385E090E090935C0A80935B0A98
:10C5600009C08091DA039091DB0340979093DB033D
:10C570008093DA038091DA039091DB0361E0CDDDF3
:10C5800020E030E040EA50E40F94D40187FDE9CF89
:10C5900081E391E09093E1038093E00309C08091EF
:10C5A000290A90912A0A409690932A0A8093290A90
:10C5B0008091290A90912A0A61E0AFDD20E030E8FD
:10C5C00048E953E40F94E20318164CF3C0912B0A88
:10C5D000D0912C0AEC2EAD2ECE014EDA609620E0E2
:10C5E00030E046E153E40F94E20318169CF3E09226
:10C5F0002B0AA0922C0ADF91CF911F910F91FF90EF
:10C60000EF90DF90CF90BF90AF909F908F90089564
:10C610008091110A9091120A60E07FDD6093150A03
:10C620007093160A8093170A9093180A8091130A40
:10C630009091140A61E071DD6093190A70931A0AEF
:10C6400080931B0A90931C0A80911D0A90911E0AE8
:10C6500013DA60931F0A7093200A8093210A909343
:10C66000220A8FB7F8941092260A8FBF08952F924E
:10C670003F924F925F926F927F928F929F92AF9272
:10C68000BF92CF92DF92EF92FF920F931F93DF93AF
:10C69000CF93CDB7DEB76A970FB6F894DEBF0FBE63
:10C6A000CDBF8091260A882309F4D2C2B1DF8091E0
:10C6B000BC039091BD03A091BE03B091BF038D8BCD
:10C6C0009E8BAF8BB88F8091C0039091C103A091D6
:10C6D000C203B091C303898B9A8BAB8BBC8B8091C7
:10C6E000C4039091C503A091C603B091C7038D8781
:10C6F0009E87AF87B88BA4E2BAE0BA87A987EFE735
:10C70000FAE0F887EF8385E69AE09E838D83A7E6BB
:10C71000BAE0BC83AB83E7E8FAE0FA83E9831A8ED8
:10C72000198E1C861B86E98DFA8DEB5EF54F6080B5
:10C73000718082809380EB85FC85E55FF54FC0803A
:10C74000D180B601882777FD8095982F0F947602C7
:10C75000A40193010F94FA007B018C01E98DFA8DFD
:10C76000E35AF54F608371838283938320E030E046
:10C7700040E851E40F94E20318167CF4E1E0AD8147
:10C78000BE81EC930F2EF0E0EF2EF0E0FF2EFCE5E3
:10C790000F2FF3E41F2FF02DE1C0C801B70120E0F7
:10C7A00030E040E851EC0F94D40187FD02C0CD2861
:10C7B00029F4E1E0AD81BE81EC93B1C0AD81BE81D1
:10C7C0008C91882369F080E090E0A0E0B0E0EB81FC
:10C7D000FC8180839183A283B383AD81BE811C924F
:10C7E0006D897E898F89988DA80197010F94B40473
:10C7F0001B012C01E98DFA8DE159F54F608371839E
:10C8000082839383C801B701EB81FC812081318150
:10C81000428153810F94FB005B016C01E98DFA8D1D
:10C82000EF5BF54FE080F18002811381A801970151
:10C830000F94D40187FD12C0E98DFA8DE75BF54FA7
:10C84000E080F18002811381C601B501A801970142
:10C850000F94E203181614F086017501AB81BC81B8
:10C86000ED92FD920D931C93139769897A898B89B8
:10C870009C89A80197010F94B4045B016C01E98DB8
:10C88000FA8DE958F54F6083718382839383C401E5
:10C89000B301EF81F88520813181428153810F946A
:10C8A000FA009B01AC016D857E858F8598890F9478
:10C8B000B40420E137ED43E25DE30F94B4047B015F
:10C8C0008C01A981BA816D917D918D919C912FE808
:10C8D00032EC45E75FE30F94B4049B01AC01C8015F
:10C8E000B7010F94FB007B018C01E981FA81608321
:10C8F000718382839383C201B101A60195010F94D4
:10C90000FB00A80197010F94FA007B018C0120E045
:10C9100030E040E050E00F94D40188235CF40F2E07
:10C92000F0E0EF2EF0E0FF2EF0E00F2FF0E01F2FF1
:10C93000F02D14C0C801B70120E030E041E653E417
:10C940000F94E203181654F40F2EF0E0EF2EF0E0EF
:10C95000FF2EF1E60F2FF3E41F2FF02DAF81B885E6
:10C960006D927D928D929C921397EB85FC85E75A90
:10C97000F54F60817181882777FD8095982F0F94FE
:10C9800076029B01AC01C401B3010F94E2031816B7
:10C99000F4F4EB85FC85E252FC4F608171818827BD
:10C9A00077FD8095982F0F9476029B01AC01C4010E
:10C9B000B3010F94D401882354F4C801B7010F9434
:10C9C000430275956795E985FA85608303C0A9855B
:10C9D000BA851C92E98DFA8D3496FA8FE98F8B8592
:10C9E0009C8502969C878B87A985BA851196BA8704
:10C9F000A987EF81F8853496F887EF838D819E8132
:10CA000001969E838D83AB81BC811496BC83AB83DE
:10CA1000E981FA813496FA83E983898D9A8D0897A2
:10CA200009F081CE60901F0A7090200A8090210A40
:10CA30009090220A60910F0A7091100A882777FD62
:10CA40008095982F0F947602A40193010F94FA0019
:10CA50007B018C0160938F0A7093900A8093910AF6
:10CA60009093920A2091CC033091CD034091CE0354
:10CA70005091CF030F94B4041B012C016093930ACF
:10CA80007093940A8093950A9093960AC801B7010F
:10CA90002091970A3091980A4091990A50919A0AE8
:10CAA0000F94FB005B016C01E090510AF090520A78
:10CAB0000091530A1091540AA80197010F94D401D0
:10CAC00087FD12C0E090550AF090560A0091570A6F
:10CAD0001091580AC601B501A80197010F94E2030D
:10CAE000181614F086017501E092970AF092980AE0
:10CAF0000093990A10939A0AC801B7012091D003B4
:10CB00003091D1034091D2035091D3030F94B404D8
:10CB10005B016C0160939B0A70939C0A80939D0A51
:10CB200090939E0AC401B30120919F0A3091A00AFC
:10CB30004091A10A5091A20A0F94FA002091D403C7
:10CB40003091D5034091D6035091D7030F94B4048C
:10CB500020E137ED43E25DE30F94B4047B018C01E7
:10CB60006091A30A7091A40A8091A50A9091A60AE7
:10CB70002FE832EC45E75FE30F94B4049B01AC016E
:10CB8000C801B7010F94FB007B018C016093A30ADD
:10CB90007093A40A8093A50A9093A60A60929F0AB4
:10CBA0007092A00A8092A10A9092A20AC201B101D9
:10CBB000A60195010F94FB00A80197010F94FA00BC
:10CBC0007B018C0120E030E040E050E00F94D40184
:10CBD00088235CF40F2EF0E0EF2EF0E0FF2EF0E063
:10CBE0000F2FF0E01F2FF02D14C0C801B70120E077
:10CBF00030E04EE453E40F94E203181654F40F2E81
:10CC0000F0E0EF2EF0E0FF2EFEE40F2FF3E41F2FF5
:10CC1000F02DC401B30120E030E040EA50E40F946D
:10CC2000E20318169CF4C401B30120E030E046E1B1
:10CC300053E40F94D40188234CF4C801B7010F9436
:10CC40004302759567956093230A02C01092230AE8
:10CC50006A960FB6F894DEBF0FBECDBFCF91DF91BD
:10CC60001F910F91FF90EF90DF90CF90BF90AF900A
:10CC70009F908F907F906F905F904F903F902F90FC
:10CC800008952F923F924F925F926F927F928F9270
:10CC90009F92AF92BF92CF92DF92EF92FF920F934B
:10CCA0001F93DF93CF93CDB7DEB7E6970FB6F89417
:10CCB000DEBF0FBECDBF6C8F7D8F8E8F9F8F5EAB23
:10CCC0004DAB39A328A30E944CFA698B7A8B8B8BCE
:10CCD0009C8B2DA93EA9233031051CF4E2EFF2E034
:10CCE00019C0E5E0F3E007C08091C00085FFFCCFEC
:10CCF00031969093C60090819923B1F78091C0003E
:10CD000085FFFCCF48C48091C00085FFFCCF3196E1
:10CD10009093C60090819923B1F78091C00085FF60
:10CD2000FCCF8AE08093C6000E94ED5D4DA95EA90C
:10CD300057FF74C087E68093230A87E6A82EB12C9C
:10CD4000C12CD12C07E6202E312C412C512C898965
:10CD50009A89AB89BC898D879E87AF87B88B898775
:10CD60009A87AB87BC871D821E821F82188620E0AF
:10CD700030E040E050E029833A834B835C830F2E00
:10CD8000F0E06F2EF0E47F2EFCE18F2EF6E49F2E74
:10CD9000F02D19AA1AAA1BAA1CAA1F8A1E8A31E002
:10CDA0003D8B4DA95EA94C5D554F5BA34AA3E3E8BB
:10CDB000FBE054915CA3EEE7FBE084918DA3E7E7F1
:10CDC000FBE094919EA3E0E7FBE0A491AFA3EAE629
:10CDD000FBE0B491B8A7E4E6FBE0249129A7E7E5DE
:10CDE000FBE034913AA7E1E5FBE044914BA7EBE48B
:10CDF000FBE054915CA7E5E4FBE084918DA7ADA92D
:10CE0000BEA9AA0FBB1FAA0FBB1FAB5EB54FBFA722
:10CE1000AEA7EBE0FBE0B491B8AB11C0EDA9FEA961
:10CE2000EC5DF54F80E78083B0E7AB2EB12CC12CD1
:10CE3000D12CA0E72A2E312C412C512C88CF809167
:10CE4000260A882309F4CDC2E3DBEDA9FEA9F7FF8A
:10CE50000DC0F0911F0AF9AB2091200A2AAB309146
:10CE6000210A3BAB4091220A4CAB11C0AEA5BFA535
:10CE7000BC91B9ABEEA5FFA5F181FAABAEA5BFA5FC
:10CE80001296BC91BBABEEA5FFA5F381FCAB69810B
:10CE90007A818B819C8129A93AA94BA95CA90F941D
:10CEA000E203181644F089A99AA9ABA9BCA9898301
:10CEB0009A83AB83BC83C401B30129A93AA94BA9C6
:10CEC0005CA90F94D40187FD06C089A99AA9ABA9D2
:10CED000BCA93C014D012D89222309F451C069A947
:10CEE0007AA98BA99CA92C8D3D8D4E8D5F8D0F94B9
:10CEF000E20318160CF075C20E944CFA29853A8597
:10CF00004B855C85621B730B840B950B69587341D1
:10CF10008040904008F465C2D601C501821993098A
:10CF2000A409B5094DA95EA957FF07C0B595A795F6
:10CF3000979587958093230A07C0B595A7959795F0
:10CF40008795EAA1FBA180830E944CFA6D877E87BA
:10CF50008F87988B9B01AC0189859A85AB85BC85B1
:10CF6000281B390B4A0B5B0B2D833E834F8358875D
:10CF70002C8D3D8D4E8D5F8D29833A834B835C8351
:10CF800069A97AA98BA99CA92C8D3D8D4E8D5F8DA9
:10CF90000F94D40188230CF023C20E944CFA2D85F3
:10CFA0003E854F855889621B730B840B950B69581E
:10CFB00073418040904008F413C20E944CFA698784
:10CFC0007A878B879C874E895F89452B09F4E3C15B
:10CFD000DC01CB012D853E854F855889821B930B43
:10CFE000A40BB50B2D813E814F815885280F391F29
:10CFF0004A1F5B1F288F398F4A8F5B8F2D813E819F
:10D000004F815885281B390B4A0B5B0BCA01B901AC
:10D01000A20191010F948605288D398D4A8D5B8D73
:10D020000F94EE05A20EB31EC41ED51E34E1A31646
:10D03000B104C104D10434F14DA95EA957FD05C066
:10D040008DEC90E0A0E0B0E004C08AEB90E0A0E0BE
:10D05000B0E08A159B05AC05BD05CCF48DA99EA951
:10D0600097FD0AC020EE30E040E050E07DECA72EB6
:10D07000B12CC12CD12C2DC06AEBA62EB12CC12C09
:10D08000D12C0EC054E1A52EB12CC12CD12CADA9B0
:10D09000BEA9B7FD05C080E790E0A0E0B0E004C005
:10D0A00087E690E0A0E0B0E08A159B05AC05BD05E1
:10D0B0001CF01501260113C0EDA9FEA9F7FD05C05E
:10D0C00020EE30E040E050E004C02DEC30E040E0E5
:10D0D00050E019012A012A183B084C085D089CA160
:10D0E000E3E8FBE008C08091C00085FFFCCF90938F
:10D0F000C600319694919923B1F784E595E0B60185
:10D10000A5012AE030E00E945C259DA1EEE7FBE04E
:10D1100008C08091C00085FFFCCF9093C600319677
:10D1200094919923B1F784E595E0B201A1012AE039
:10D1300030E00E945C259EA1E7E7FBE008C08091FB
:10D14000C00085FFFCCF9093C6003196949199233F
:10D15000B1F784E595E0B401A30122E030E00E943C
:10D1600062269FA1E0E7FBE008C08091C00085FF38
:10D17000FCCF9093C600319694919923B1F784E542
:10D1800095E049815A816B817C8122E030E00E94E8
:10D1900062268091C00085FFFCCF8AE08093C600A4
:10D1A0002E893F89233031050CF4F5C0C201B1014D
:10D1B0000F94760220E030E040E850E40F94B4048D
:10D1C0007B018C0169817A818B819C81A40193010F
:10D1D0000F94FA0020ED3FE049E450E40F94B404CA
:10D1E00020E030E040E05FE30F94B4049B01AC0129
:10D1F000C801B7010F94DB017B018C01688D798D2B
:10D200008A8D9B8D0F94760220E030E04AE754E44B
:10D210000F94DB013B014C0198A5EAE6FBE008C056
:10D220008091C00085FFFCCF9093C6003196949109
:10D230009923B1F784E595E0B801A70122E030E039
:10D240000E94622699A5E4E6FBE008C08091C00038
:10D2500085FFFCCF9093C600319694919923B1F746
:10D2600084E595E0B401A30122E030E00E9462264B
:10D270008091C00085FFFCCF8AE08093C600C80182
:10D28000B7012AE939E949E15FE30F94B4047B016E
:10D290008C019AA5E7E5FBE008C08091C00085FFFE
:10D2A000FCCF9093C600319694919923B1F7809169
:10D2B000C00085FFFCCF8AE08093C6009BA5E1E516
:10D2C000FBE008C08091C00085FFFCCF9093C600B2
:10D2D000319694919923B1F784E595E0B801A701BF
:10D2E00022E030E00E9462268091C00085FFFCCFE2
:10D2F0008AE08093C6009CA5EBE4FBE008C0809127
:10D30000C00085FFFCCF9093C6003196949199237D
:10D31000B1F7C801B701A80197010F94FB00A40160
:10D3200093010F94DB01AB01BC0184E595E022E0A1
:10D3300030E00E9462268091C00085FFFCCF8AE029
:10D340008093C6009DA5E5E4FBE008C08091C00085
:10D3500085FFFCCF9093C600319694919923B1F745
:10D36000C801B701A40193010F94B40420E030E098
:10D3700040E05EE30F94B404AB01BC0184E595E0AA
:10D3800022E030E00E9462268091C00085FFFCCF41
:10D390008AE08093C600D201C1018A0D9B1DAC1D9D
:10D3A000BD1D4DA95EA957FF07C0B595A7959795D7
:10D3B00087958093230A07C0B595A795979587957C
:10D3C000EAA1FBA180832E893F892F5F3F4F3F8BCE
:10D3D0002E8B6C8C7D8C8E8C9F8C31E03D8B01C0B4
:10D3E0001D8A6C8D7D8D8E8D9F8D20E030E040EA12
:10D3F00051E40F94FB009B01AC0169A97AA98BA9A8
:10D400009CA90F94E20318169CF4EBE1FBE09491C5
:10D4100008C08091C00085FFFCCF9093C600319674
:10D4200094919923B1F78091C00085FFFCCFB3C0E0
:10D430000E944CFA29893A894B895C89621B730BDB
:10D44000840B950B615D77408040904008F454C098
:10D450004DA95EA957FF11C06091230AE5E1FBE0E9
:10D46000949108C08091C00085FFFCCF9093C600C6
:10D47000319694919923B1F711C0AAA1BBA16C91E7
:10D48000EFE0FBE0949108C08091C00085FFFCCFE5
:10D490009093C600319694919923B1F7162F84E5A5
:10D4A00095E049A95AA96BA97CA922E030E00E9425
:10D4B000622698A9EBE0FBE008C08091C00085FFE0
:10D4C000FCCF9093C600319694919923B1F784E5EF
:10D4D00095E0612F70E04AE050E00E948F25809136
:10D4E000C00085FFFCCF8AE08093C6000E944CFA02
:10D4F000698B7A8B8B8B9C8B0E944CFA7B018C0105
:10D500000E944CFA2D853E854F855889E21AF30A10
:10D51000040B150B29853A854B855C85E21AF30AC5
:10D52000040B150BE60EF71E081F191F31E8E31652
:10D530003FE4F30632E1030730E0130798F0EEEE24
:10D54000FAE0949108C08091C00085FFFCCF9093D1
:10D55000C600319694919923B1F78091C00085FF60
:10D56000FCCF19C04E895F8988A199A184179507BE
:10D5700074F5E2EAFAE0949108C08091C00085FF5A
:10D58000FCCF9093C600319694919923B1F7809186
:10D59000C00085FFFCCF8AE08093C600E6960FB6F8
:10D5A000F894DEBF0FBECDBFCF91DF911F910F91D9
:10D5B000FF90EF90DF90CF90BF90AF909F908F90B3
:10D5C0007F906F905F904F903F902F9008950E94B2
:10D5D00035E135CC1092DB0A1092DD0A1092DF0A99
:10D5E00008958093E6030895EFE6F0E0808182607D
:10D5F000808308951F93FC011FB7F8948081918167
:10D60000A281B3818093B50A9093B60AA093B70A1A
:10D61000B093B80AFB0180819181A281B38180938C
:10D62000B90A9093BA0AA093BB0AB093BC0AFA0154
:10D6300080819181A281B3818093BD0A9093BE0ABB
:10D64000A093BF0AB093C00AF90180819181A281A1
:10D65000B3818093C10A9093C20AA093C30AB09386
:10D66000C40A1FBF1F910895FC012FB7F894808151
:10D670009181A281B3818093C10A9093C20AA09341
:10D68000C30AB093C40A2FBF0895E82F8FB7F89448
:10D69000F0E0EE0FFF1FEE0FFF1FEB54F54F208160
:10D6A0003181428153818FBFB901CA0108958091B0
:10D6B0006F008D7F80936F0006C0809182128F5F14
:10D6C0008F708093821290918112809182129817AC
:10D6D00051F41092A80A1092A70A80916F008260FC
:10D6E00080936F0008959091811280918212981713
:10D6F00051F3E3CFE1E2FCE0949108C08091C000D7
:10D7000085FFFCCF9093C600319694919923B1F791
:10D71000EDE1FCE0949108C08091C00085FFFCCF52
:10D720009093C600319694919923B1F788E20E94B4
:10D73000D8FCBC0184E595E04AE050E00E948F25CA
:10D7400089E20E94D8FCBC0184E595E04AE050E003
:10D750000E948F258091C00085FFFCCF8AE08093D6
:10D76000C600E9E1FCE0949108C08091C00085FF0B
:10D77000FCCF9093C600319694919923B1F785E43C
:10D780000E94D8FCBC0184E595E04AE050E00E948C
:10D790008F2587E20E94D8FCBC0184E595E04AE031
:10D7A00050E00E948F258091C00085FFFCCF8AE069
:10D7B0008093C600E5E1FCE0949108C08091C00030
:10D7C00085FFFCCF9093C600319694919923B1F7D1
:10D7D00084E40E94D8FCBC0184E595E04AE050E076
:10D7E0000E948F2583E40E94D8FCBC0184E595E06B
:10D7F0004AE050E00E948F258091C00085FFFCCF59
:10D800008AE08093C600E0E1FCE0949108C080913A
:10D81000C00085FFFCCF9093C60031969491992368
:10D82000B1F781E40E94D8FCBC0184E595E04AE0B0
:10D8300050E00E948F2582E40E94D8FCBC0184E560
:10D8400095E04AE050E00E948F258091C00085FF5E
:10D85000FCCF8AE08093C600EBE0FCE0949108C026
:10D860008091C00085FFFCCF9093C60031969491C3
:10D870009923B1F78FE30E94D8FCBC0184E595E0C1
:10D880004AE050E00E948F2580E40E94D8FCBC0151
:10D8900084E595E04AE050E00E948F258091C00029
:10D8A00085FFFCCF8AE08093C60008950F931F93F5
:10D8B000182F042F67FD19C0823081F0833028F4BF
:10D8C000882341F0813089F407C0833049F08430E7
:10D8D00061F408C088E207C085E405C084E403C0A1
:10D8E00081E401C08FE30E94A6FC07FD1AC012303C
:10D8F00081F0133028F4112341F0113091F407C066
:10D90000133049F0143069F408C089E207C087E297
:10D9100005C083E403C082E401C080E4602F0E945C
:10D92000A6FC1F910F910895643089F0653028F4AA
:10D93000613041F0623099F407C0683051F06031D5
:10D9400071F40AC060E001C061E040E004C060E042
:10D9500001C061E041E0AACF61E041E0A7CF0895B6
:10D960000F931F93182F062F86E260E00E94A6FCFB
:10D970001EBD0DB407FEFDCF8EB50EBD0DB407FE66
:10D98000FDCF8EB586E261E00E94A6FC1F910F914B
:10D990000895EDE6F4E0E80FF11D808190E0E0CF1E
:10D9A000CF93DF9389E261E00E94F3FB87E261E0BD
:10D9B0000E94F3FB83E461E00E94F3FB82E461E0F8
:10D9C0000E94F3FB80E461E00E94F3FBC0E0D0E042
:10D9D000FE01E859FB4F8C2F6081A6DF2196C530F0
:10D9E000D105B1F7DF91CF910895CF93DF930E94D6
:10D9F000F2F986E261E00E94F3FBC0E0D0E0FE01B4
:10DA0000E359FB4FDE01AE58BB4F6C91808190E033
:10DA100070E0A6DF2196C530D10589F7DF91CF915F
:10DA20000895E3DFBDDFEAE0F1E08081826080837A
:10DA30008081816080838081846080838081806434
:10DA400080838081806880830F9A179A0E9A169A35
:10DA50000D9A159A0C9A149A0B9A139A26982E9A44
:10DA600025982D9A24982C9A389A4098179A1092B3
:10DA70001108399A4198169A109212083A9A4298C7
:10DA8000159A109213083B9A4398149A3C9A44981A
:10DA9000139AA1E8B0E08C918F7E8C938C91886072
:10DAA0008C93E0E8F0E080818D7F808380818E7FA1
:10DAB000808380818F73808380818F7C80838C9131
:10DAC000887F82608C9380E090E4909389008093BB
:10DAD00088001092850010928400EFE6F0E08081CB
:10DAE0008260808381E08093E6037894089590912A
:10DAF000811280918212981739F00E9437630E9438
:10DB00000A360E9435E1F3CF0895F1DF179A10929B
:10DB10001108169A10921208159A10921308149A66
:10DB2000139A08951F920F920FB60F920BB60F9291
:10DB30001124AF92BF92CF92DF92EF92FF920F9398
:10DB40001F932F933F934F935F936F937F938F9385
:10DB50009F93AF93BF93CF93DF93EF93FF93809106
:10DB6000A70A9091A80A892B09F097C19091811278
:10DB700080918212981719F4E0E0F0E014C08091CF
:10DB8000821290E021E530E0829FF001839FF00D4A
:10DB9000929FF00D1124EF58F24FE05BFF4F81E0B0
:10DBA0008083E055F040F093A80AE093A70A3097ED
:10DBB00009F46DC1E05BFF4F81E08083E055F040E8
:10DBC0001092E70A1092E80A1092E90A1092EA0A03
:10DBD00060AD71AD2CE96134720718F060E47CE946
:10DBE00004C03EE46132730730F076956795769510
:10DBF000679584E007C047E26131740730F076959D
:10DC0000679582E08093E00A07C08093E00A603263
:10DC1000710510F460E270E06052704058E06030CE
:10DC20007507E8F0472F50E0440F551F440F551F6C
:10DC3000415D534F9A012E5F3F4FF90185919491B9
:10DC40009C01AA27639FC001629F810D9A1F0694C1
:10DC50008A1F9A1F1124FA01459154911EC0CB01CD
:10DC6000969587958C7F815D9F4EFC0145915491DF
:10DC7000FC01329625913491862F90E08770907048
:10DC8000FC012E9FC0012F9F900D3E9F900D1124EF
:10DC9000B3E096958795BA95E1F7481B590B443642
:10DCA0005105A8F4EFE2F3E007C08091C00085FFC2
:10DCB000FCCF31969093C60090819923B1F784E50B
:10DCC00095E04AE050E00E94B62544E650E05093CB
:10DCD000EC0A4093EB0A8091E00A992787FD909522
:10DCE0009093EE0A8093ED0AE091A70AF091A80ABA
:10DCF00064AD75AD7093E60A6093E50AFCE96134A2
:10DD00007F0718F060E47CE904C02EE461327207FA
:10DD100030F0769567957695679584E007C037E291
:10DD20006131730730F07695679582E08093E00A61
:10DD300008C081E08093E00A6032710510F460E26F
:10DD400070E06052704048E060307407E8F0472FA0
:10DD500050E0440F551F440F551F415D534F9A012A
:10DD60002E5F3F4FF901859194919C01AA27639FF3
:10DD7000C001629F810D9A1F06948A1F9A1F112469
:10DD8000FA01459154911EC0CB01969587958C7FE1
:10DD9000815D9F4EFC0145915491FC013296259185
:10DDA0003491862F90E087709070FC012E9FC00107
:10DDB0002F9F900D3E9F900D112433E096958795EF
:10DDC0003A95E1F7481B590B44365105A8F4EFE2A8
:10DDD000F3E007C08091C00085FFFCCF319690939F
:10DDE000C60090819923B1F784E595E04AE050E0C0
:10DDF0000E94B62544E650E0CA01A0E0B0E080935E
:10DE0000E10A9093E20AA093E30AB093E40A5093E4
:10DE1000890040938800E091A70AF091A80A8089C0
:10DE20009189A289B389B695A79597958795B0955D
:10DE3000A095909581959F4FAF4FBF4F8093C50A96
:10DE40009093C60AA093C70AB093C80A8093C90AE0
:10DE50009093CA0AA093CB0AB093CC0A8093CD0AC0
:10DE60009093CE0AA093CF0AB093D00A8093D10AA0
:10DE70009093D20AA093D30AB093D40A1092D50AF1
:10DE80001092D60A1092D70A1092D80A06C080EDD6
:10DE900097E09093890080938800C091A70AD09161
:10DEA000A80A209709F4C9C488A18093D90A80FFE1
:10DEB0000AC08FB7F89490910B019D7F90930B014E
:10DEC0008FBF8FEF09C08FB7F89490910B019260CC
:10DED00090930B018FBF81E08093E2038091D90A78
:10DEE00081FF0AC08FB7F89490910B0191609093D5
:10DEF0000B018FBF8FEF09C08FB7F89490910B0182
:10DF00009E7F90930B018FBF81E08093E30380910C
:10DF1000D90A80FF3CC08091E6038823C1F183B118
:10DF200082958695869583708095282F217080FF35
:10DF30002CC08091DA0A882341F188819981AA81D5
:10DF4000BB81181619061A061B06FCF48091B50A47
:10DF50009091B60AA091B70AB091B80A8093A90A25
:10DF60009093AA0AA093AB0AB093AC0A81E0809385
:10DF7000DB0A88899989AA89BB898093D50A9093FD
:10DF8000D60AA093D70AB093D80A2093DA0A8091D0
:10DF9000D90A81FF3BC08091E6038823B9F183B1A0
:10DFA0008295869587708095282F217080FF2CC0E0
:10DFB0008091DC0A882341F18C819D81AE81BF81F3
:10DFC000181619061A061B06FCF48091B90A9091DE
:10DFD000BA0AA091BB0AB091BC0A8093AD0A909393
:10DFE000AE0AA093AF0AB093B00A81E08093DD0A35
:10DFF00088899989AA89BB898093D50A9093D60A82
:10E00000A093D70AB093D80A2093DC0A8091D90A4A
:10E0100082FF47C09FB7F89480910B018B7F80935C
:10E020000B019FBF8FEF8093E4038091E603882369
:10E0300009F442C083B182958F708095282F21709A
:10E0400080FF2CC08091DE0A882341F18885998564
:10E05000AA85BB85181619061A061B06FCF48091C2
:10E06000BD0A9091BE0AA091BF0AB091C00A8093E8
:10E07000B10A9093B20AA093B30AB093B40A81E0B4
:10E080008093DF0A88899989AA89BB898093D50AF8
:10E090009093D60AA093D70AB093D80A2093DE0AA9
:10E0A0000BC08FB7F89490910B01946090930B0183
:10E0B0008FBF81E08093E4038091D90A99A183FF07
:10E0C00012C0913031F49FB7F89480910B018068B1
:10E0D00005C09FB7F89480910B01806480930B0179
:10E0E0009FBF8FEF11C0913031F49FB7F8948091AA
:10E0F0000B018F7705C09FB7F89480910B018F7B40
:10E1000080930B019FBF81E08093E50360E074C1C1
:10E110008091C00087FF19C04091C600E091500572
:10E12000F091510531969F012F7730703197809192
:10E130005205909153052817390739F0E053FB4FEA
:10E1400040833093510520935005288139814A81BD
:10E150005B818091C50A9091C60AA091C70AB091CF
:10E16000C80A280F391F4A1F5B1F2093C50A309326
:10E17000C60A4093C70A5093C80A1216130614061B
:10E1800015066CF5409A88899989AA89BB89281B4C
:10E19000390B4A0B5B0B2093C50A3093C60A409398
:10E1A000C70A5093C80A2091B50A3091B60A409127
:10E1B000B70A5091B80A8091E203992787FD90959C
:10E1C000A92FB92F820F931FA41FB51F8093B50AE3
:10E1D0009093B60AA093B70AB093B80A40982C81DE
:10E1E0003D814E815F818091C90A9091CA0AA091B8
:10E1F000CB0AB091CC0A280F391F4A1F5B1F20930E
:10E20000C90A3093CA0A4093CB0A5093CC0A12161B
:10E210001306140615066CF5419A88899989AA890E
:10E22000BB89281B390B4A0B5B0B2093C90A30931F
:10E23000CA0A4093CB0A5093CC0A2091B90A309174
:10E24000BA0A4091BB0A5091BC0A8091E303992716
:10E2500087FD9095A92FB92F820F931FA41FB51F7B
:10E260008093B90A9093BA0AA093BB0AB093BC0AF0
:10E270004198288539854A855B858091CD0A9091A2
:10E28000CE0AA091CF0AB091D00A280F391F4A1F99
:10E290005B1F2093CD0A3093CE0A4093CF0A509350
:10E2A000D00A12161306140615066CF5429A8889D0
:10E2B0009989AA89BB89281B390B4A0B5B0B2093D0
:10E2C000CD0A3093CE0A4093CF0A5093D00A2091C2
:10E2D000BD0A3091BE0A4091BF0A5091C00A809198
:10E2E000E403992787FD9095A92FB92F820F931FDB
:10E2F000A41FB51F8093BD0A9093BE0AA093BF0AC6
:10E30000B093C00A42982C853D854E855F858091EB
:10E31000D10A9091D20AA091D30AB091D40A280FC1
:10E32000391F4A1F5B1F2093D10A3093D20A4093B2
:10E33000D30A5093D40A1216130614061506BCF518
:10E3400089A1813011F4449A01C0439A888999893E
:10E35000AA89BB89281B390B4A0B5B0B2093D10A76
:10E360003093D20A4093D30A5093D40A2091C10A21
:10E370003091C20A4091C30A5091C40A8091E503CA
:10E38000992787FD9095A92FB92F820F931FA41F5E
:10E39000B51F8093C10A9093C20AA093C30AB09399
:10E3A000C40A89A1813011F4449801C04398809136
:10E3B000D50A9091D60AA091D70AB091D80A0196B1
:10E3C000A11DB11D8093D50A9093D60AA093D70AB8
:10E3D000B093D80A2091D50A3091D60A4091D70A35
:10E3E0005091D80A88899989AA89BB892817390741
:10E3F0004A075B0730F46F5F8091E00A68170CF4FE
:10E4000087CE2091D50A3091D60A4091D70A5091F3
:10E41000D80A8C899D89AE89BF8982179307A40782
:10E42000B50708F4E3C0E090E10AF090E20A009139
:10E43000E30A1091E40AAC8CBD8CCE8CDF8CA80171
:10E440009701C601B501AA27279FB12D389FF0017A
:10E45000489FF00D479FE00DF11D289FB00DE11D75
:10E46000FA1F379FB00DE11DFA1F469FB00DE11D49
:10E47000FA1F369FB10DEA1FFA1FB695EA1FFA1F61
:10E4800011248CAD9DAD8E0F9F1F9093E60A809353
:10E49000E50A28AD39AD4AAD5BADA0E0B0E0281784
:10E4A00039074A075B0720F43093E60A2093E50A10
:10E4B0006091E50A7091E60A8CE96134780718F0FA
:10E4C00060E47CE904C09EE46132790730F076951F
:10E4D00067957695679584E007C0E7E261317E072E
:10E4E00030F07695679582E08093E00A08C081E07D
:10E4F0008093E00A6032710510F460E270E06052CF
:10E500007040F8E060307F07E8F0472F50E0440F9C
:10E51000551F440F551F415D534F9A012E5F3F4FCA
:10E52000F901859194919C01AA27639FC001629F84
:10E53000810D9A1F06948A1F9A1F1124FA01459192
:10E5400054911EC0CB01969587958C7F815D9F4E1F
:10E55000FC0145915491FC01329625913491862F0E
:10E5600090E087709070FC012E9FC0012F9F900D4E
:10E570003E9F900D1124B3E096958795BA95E1F7EB
:10E58000481B590B44365105A8F4EFE2F3E007C0ED
:10E590008091C00085FFFCCF31969093C60090819A
:10E5A0009923B1F784E595E04AE050E00E94B62552
:10E5B00044E650E050938900409388009A0140E07F
:10E5C00050E08091E10A9091E20AA091E30AB091B3
:10E5D000E40A820F931FA41FB51F8093E10A909352
:10E5E000E20AA093E30AB093E40A02C12091D50A9B
:10E5F0003091D60A4091D70A5091D80A888D998DCA
:10E60000AA8DBB8D82179307A407B50708F0E4C055
:10E610006091E70A7091E80A8091E90A9091EA0A0C
:10E620002C8D3D8D4E8D5F8DAA27639FB12D749FDC
:10E63000F001849FF00D839FE00DF11D649FB00DEC
:10E64000E11DFA1F739FB00DE11DFA1F829FB00DEF
:10E65000E11DFA1F729FB10DEA1FFA1FB695EA1F5E
:10E66000FA1F11248091E50A9091E60A8E179F0700
:10E6700038F4C05CDF4F68817981C054D04003C05A
:10E68000BC016E1B7F0BC05CDF4F288139814A8142
:10E690005B81CB01A0E0B0E082179307A407B50728
:10E6A00008F4B901FCE961347F0718F060E47CE903
:10E6B00004C02EE46132720730F076956795769546
:10E6C000679584E007C037E26131730730F07695D3
:10E6D000679582E08093E00A08C081E08093E00AB9
:10E6E0006032710510F460E270E06052704048E002
:10E6F00060307407E8F0472F50E0440F551F440F77
:10E70000551F415D534F9A012E5F3F4FF90185918F
:10E7100094919C01AA27639FC001629F810D9A1F5B
:10E7200006948A1F9A1F1124FA01459154911EC024
:10E73000CB01969587958C7F815D9F4EFC0145911D
:10E740005491FC01329625913491862F90E0877088
:10E750009070FC012E9FC0012F9F900D3E9F900D49
:10E76000112423E0969587952A95E1F7481B590BCC
:10E7700044365105A8F4EFE2F3E007C08091C000F1
:10E7800085FFFCCF31969093C60090819923B1F715
:10E7900084E595E04AE050E00E94B62544E650E06A
:10E7A00050938900409388009A0140E050E08091A6
:10E7B000E70A9091E80AA091E90AB091EA0A820F6B
:10E7C000931FA41FB51F8093E70A9093E80AA093B4
:10E7D000E90AB093EA0A0CC08091EB0A9091EC0A26
:10E7E00090938900809388008091ED0A8093E00ADD
:10E7F0002091D50A3091D60A4091D70A5091D80A73
:10E80000E091A70AF091A80A80899189A289B38929
:10E81000281739074A075B0780F01092A80A109260
:10E82000A70A9091811280918212981731F08091FD
:10E8300082128F5F8F7080938212FF91EF91DF9130
:10E84000CF91BF91AF919F918F917F916F915F9188
:10E850004F913F912F911F910F91FF90EF90DF907B
:10E86000CF90BF90AF900F900BBE0F900FBE0F9048
:10E870001F9018958091DB0A882349F48091DD0A66
:10E88000882329F48091DF0A882309F49CC0EFE2F1
:10E89000F4E1949108C08091C00085FFFCCF909373
:10E8A000C600319694919923B1F7E1E7F4E1949190
:10E8B00008C08091C00085FFFCCF9093C6003196C0
:10E8C00094919923B1F78091DB0A8823F1F060914C
:10E8D000A90A7091AA0A8091AB0A9091AC0A0F9490
:10E8E00076022091100D3091110D4091120D509132
:10E8F000130D0F94DB01AB01BC018DE694E10E9486
:10E90000CC398DE594E10E9458E08091DD0A88239E
:10E91000F1F06091AD0A7091AE0A8091AF0A9091CA
:10E92000B00A0F9476022091140D3091150D40918C
:10E93000160D5091170D0F94DB01AB01BC0189E559
:10E9400094E10E94CC3989E494E10E9458E08091DE
:10E95000DF0A8823F1F06091B10A7091B20A8091C8
:10E96000B30A9091B40A0F9476022091180D309159
:10E97000190D40911A0D50911B0D0F94DB01AB0145
:10E98000BC0185E494E10E94CC3985E394E10E94C6
:10E9900058E0E3E4F3E007C08091C00085FFFCCFBE
:10E9A00031969093C60090819923B1F78091C00071
:10E9B00085FFFCCF8AE08093C6001092DB0A10929C
:10E9C000DD0A1092DF0A08952F923F924F925F92D4
:10E9D0006F927F928F929F92AF92BF92CF92DF926F
:10E9E000EF92FF920F931F93DF93CF93CDB7DEB7D4
:10E9F000CD55D0400FB6F894DEBF0FBECDBF2F96D9
:10EA00009FAF8EAF2F9761967FAF6EAF61972A0150
:10EA100062962FAF629763960FAF63976496EFAEDF
:10EA200064976896ACAEBDAECEAEDFAE6897E22E10
:10EA3000FF24EE0CFF1CEE0CFF1C9A012E0D3F1D57
:10EA40002D963FAF2EAF2D97D9016D907D908D9073
:10EA50009C90FC01EE0DFF1DC401B30120813181AA
:10EA6000428153810F94FB0069AF7AAF8BAF9CAFAB
:10EA700010E0000F111F000F111FF201E00FF11F36
:10EA80002B96FFAFEEAF2B97A080B180C280D380D2
:10EA90002F96EEADFFAD2F97E00FF11FC601B50128
:10EAA00020813181428153810F94FB006DAB7EAB9D
:10EAB0008FAB98AF64962FAD6497E22FF0E0EE0F26
:10EAC000FF1FEE0FFF1F2F96AEADBFAD2F97AE0FFE
:10EAD000BF1F4D915D916D917C9129964CAF5DAFBB
:10EAE0006EAF7FAF299761966EAD7FAD6197E60FF0
:10EAF000F71F608171818281938129962CAD3DAD94
:10EB00004EAD5FAD29970F94FA0069AB7AAB8BAB32
:10EB10009CAB6196AEADBFAD61971C968D919D91FA
:10EB20000D90BC91A02D25968CAF9DAFAEAFBFAF21
:10EB300025972F96AEADBFAD2F971C962D913D9189
:10EB40004D915C911F9721962CAF3DAF4EAF5FAFBB
:10EB50002197A401930150582DA73EA74FA758AB6A
:10EB6000B601A501705849A75AA76BA77CA7619663
:10EB70006EAD7FAD6197E60EF71ED7016D917D9169
:10EB80008D919C9129AD3AAD4BAD5CAD0F94FA00DF
:10EB90003B014C016196EEADFFAD61970E0F1F1F5B
:10EBA000D8016D917D918D919C912DA93EA94FA980
:10EBB00058AD0F94FA005B016C016DA57EA58FA581
:10EBC00098A9A60195010F94B4047B018C0169A555
:10EBD0007AA58BA59CA5A40193010F94B4049B0175
:10EBE000AC01C801B7010F94FA001B012C016DA5FF
:10EBF0007EA58FA598A9A40193010F94B4047B016D
:10EC00008C0169A57AA58BA59CA5A60195010F94F9
:10EC1000B4049B01AC01C801B7010F94FB009B0138
:10EC2000AC01C201B1010F946E015B016C0120E0E7
:10EC300030E040E050E00F94D401882354F4C60142
:10EC4000B5012BED3FE049EC50E40F94FB005B0174
:10EC50006C01E8968FADE897882351F0C601B501A5
:10EC60002BED3FE049EC50E40F94FA005B016C019E
:10EC7000C601B501E7962CAD3DAD4EAD5FADE79752
:10EC80000F94B40429A93AA94BA95CA95F770F9402
:10EC9000EF037B018C012FE632E143E85AE30F9446
:10ECA000D40187FDF6C1C801B7010F94B1020F94DA
:10ECB000480278A76FA3672B21F4E1E0F0E0F8A702
:10ECC000EFA32FA138A5B90180E090E00F94740262
:10ECD0007B018C01C601B501A80197010F94DB01EE
:10ECE0006BA37CA38DA39EA369A97AA98BA99CA9D8
:10ECF000A80197010F94DB016F8F78A389A39AA3D2
:10ED000025966CAD7DAD8EAD9FAD259721962CAD32
:10ED10003DAD4EAD5FAD21970F94FA00A80197016C
:10ED20000F94DB016B8F7C8F8D8F9E8F6BA17CA1ED
:10ED30008DA19EA120E030E040E05FEB0F94B40491
:10ED40002BA13CA14DA15EA10F94B40420E030E0C2
:10ED500040E85FE30F94FB006F8B788F898F9A8F69
:10ED600064963FAD6497E32FF0E0EE0FFF1FEE0FC8
:10ED7000FF1F9E012F5F3F4FE20FF31F29964CADFF
:10ED80005DAD6EAD7FAD2997408351836283738300
:10ED90002F96AEADBFAD2F971C964D915D916D91A5
:10EDA0007C911F974D875E876F87788B41E050E09D
:10EDB0005A8B498B662462967FAD6297672F70E00D
:10EDC000660F771F660F771FC901860F971F6A9618
:10EDD0009FAF8EAF6A976396BFAD6397AB2FB0E0DE
:10EDE000AA0FBB1FAA0FBB1F21E030E02C0F3D1F55
:10EDF0002A0F3B1F6C963FAF2EAF6C976E96FFAFFE
:10EE0000EEAF6E971AC138E136150CF446C06DA509
:10EE10007EA58FA598A92BA13CA14DA15EA10F9421
:10EE2000B4047B018C0169A57AA58BA59CA52F89CB
:10EE3000388D498D5A8D0F94B4049B01AC01C801E3
:10EE4000B7010F94FB007B018C016DA57EA58FA5FA
:10EE500098A92F89388D498D5A8D0F94B4045B0180
:10EE60006C0169A57AA58BA59CA52BA13CA14DA100
:10EE70005EA10F94B4049B01AC01C601B5010F94CF
:10EE8000FA006DA77EA78FA798AB6394C701D8013E
:10EE900089A79AA7ABA7BCA765C049895A89BA01B7
:10EEA00080E090E00F9474022BA13CA14DA15EA1E3
:10EEB0000F94B4047B018C01C8010F94D8016B8BB3
:10EEC0007C8B8D8B9E8BB701C8010F9417053B017E
:10EED0004C012D96AEADBFAD2D97ED90FD900D91EF
:10EEE0001C9117FB109517F910952B96EEADFFAD01
:10EEF0002B972080318042805380C801B7012B8935
:10EF00003C894D895E890F94B4045B016C01C20198
:10EF1000B101A40193010F94B4049B01AC01C6019B
:10EF2000B5010F94FB006DA77EA78FA798ABC80112
:10EF3000B701A40193010F94B4047B018C01C201B9
:10EF4000B1012B893C894D895E890F94B4049B01E2
:10EF5000AC01C801B7010F94FA0069A77AA78BA783
:10EF60009CA7662469AD7AAD8BAD9CAD2DA53EA561
:10EF70004FA558A90F94FB006A96AEADBFAD6A9736
:10EF80006D937D938D939C9313976DA97EA98FA903
:10EF900098AD29A53AA54BA55CA50F94FB006C96EE
:10EFA000EEADFFAD6C9760837183828393836E9621
:10EFB000AEADBFAD6E976D917D918D919C912F8D72
:10EFC00038A149A15AA10F94FB006E96EEADFFAD9A
:10EFD0006E9760837183828393836D857E858F8531
:10EFE00098892B8D3C8D4D8D5E8D0F94FB006D8728
:10EFF0007E878F87988BCE0101960E94D033CE01F9
:10F000000196BE016B5F7F4FAE01475F5F4F9E0170
:10F01000235F3F4F6896ECACFDAC0EAD1FAD68971B
:10F02000F8E7CF2ED12CCC0EDD1E0E94F38F29895C
:10F030003A892F5F3F4F3A8B298B49895A896FA1B3
:10F0400078A54617570708F4DECE61964EAD5FAD42
:10F050006197485F5F4F61962EAD3FAD6197245F2A
:10F060003F4F61968EAD9FAD6197DC01149661961E
:10F07000BFAFAEAF6197BD016896ECACFDAC0EAD15
:10F080001FAD6897E8E7CE2ED12CCC0EDD1E0E9476
:10F09000F38FC35ADF4F0FB6F894DEBF0FBECDBF5C
:10F0A000CF91DF911F910F91FF90EF90DF90CF9064
:10F0B000BF90AF909F908F907F906F905F904F9098
:10F0C0003F902F900895FF920F931F93CF93DF935C
:10F0D0008B010E944CFAEB01FF24FA9409C00E94B4
:10F0E0004CFA6C1B7D0B6017710710F080E008C0B4
:10F0F000FEBC0DB407FEFDCF8EB58F3F81F781E0DA
:10F10000DF91CF911F910F91FF900895FC014281F3
:10F11000242F30E0C9019595879580658CBD40FF0F
:10F1200002C080E004C080E0463009F081E08DBD7F
:10F13000808160E00C94A6FCDF92EF92FF920F9327
:10F140001F93CF93DF93EC01D62E79018A01DEDF86
:10F15000CE016CE271E0B7DF8D2D80648EBD0DB401
:10F1600007FEFDCF28E130E0D801C701022E04C020
:10F17000B695A795979587950A94D2F78EBD0DB44D
:10F1800007FEFDCF285030408FEF283F380761F74A
:10F19000DD2011F485E906C088E0D81611F487E86F
:10F1A00001C08FEF8EBD0DB407FEFDCF8CE0D816E9
:10F1B00031F48FEF8EBD0DB407FEFDCF8EB59FEFFE
:10F1C0002FEF2EBD0DB407FEFDCF8EB587FF04C017
:10F1D000992311F09150F5CF8B83DF91CF911F913F
:10F1E0000F91FF90EF90DF900895FC01808161E026
:10F1F0000C94A6FCDC016EBDFA0120E030E00DB4F9
:10F2000007FEFDCF80818EBD0DB407FEFDCF81814D
:10F210008EBD2E5F3F4F329682E02030380779F75F
:10F220000DB407FEFDCF8FEF8EBD0DB407FEFDCFF1
:10F230008FEF8EBD0DB407FEFDCF8FEF8EBD0DB4E9
:10F2400007FEFDCF8EB513968C9313978F71853083
:10F2500011F481E0089583E111968C931197CD010B
:10F26000C4DF80E00895CF92DF92EF92FF920F9378
:10F270001F93CF93DF93EC017A018B0169018C819D
:10F28000833039F059E0EE0CFF1C001F111F5A9516
:10F29000D1F7CE0168E1A80197014EDF882311F074
:10F2A00086E020C0CE016EEFA601A4DF8823D9F04E
:10F2B000CE0168E572E007DF882311F487E112C010
:10F2C000CE016DE020E030E040E050E035DF882303
:10F2D00041F48FEF8EBD0DB407FEFDCF8EB58823B0
:10F2E00071F086E18983CE0180DF80E0DF91CF91EC
:10F2F0001F910F91FF90EF90DF90CF900895CE0176
:10F3000074DF81E0F3CFBF92CF92DF92EF92FF9252
:10F310000F931F93CF93DF93EC016B017A010E944F
:10F320004CFA8B01BB24BA9409C00E944CFA601BB2
:10F33000710B6D52714010F081E10BC0BEBC0DB479
:10F3400007FEFDCF8EB58B838F3F79F38E3F31F073
:10F350008FE08983CE0149DF80E02EC0D70111976D
:10F36000EF28D9F08FEF8EBD20E030E09FEF0BC08B
:10F370000DB407FEFDCF8EB5F601E20FF31F8083BB
:10F380009EBD2F5F3F4F2A173B0790F30DB407FE3A
:10F39000FDCF8EB5AC0DBD1D8C938FEF8EBD0DB422
:10F3A00007FEFDCF8EB58FEF8EBD0DB407FEFDCFEE
:10F3B0008EB5CE011ADF81E0DF91CF911F910F91C1
:10F3C000FF90EF90DF90CF90BF900895CF92DF92A3
:10F3D000EF92FF920F931F93CF93DF93EC017A018B
:10F3E0008B0169018C81833039F0A9E0EE0CFF1CA0
:10F3F000001F111FAA95D1F7CE0161E1A801970165
:10F400009BDE882331F084E08983CE01EEDE80E04C
:10F4100005C0CE01B60140E052E075DFDF91CF912B
:10F420001F910F91FF90EF90DF90CF900895BF92C2
:10F43000CF92DF92EF92FF920F931F93CF93DF93C0
:10F44000EC01B62E1C82198248830E944CFA6B0193
:10F45000888161E00E94F3FBCE01C7DE82E360E0B9
:10F460000E94F3FB83E361E00E94F3FB84E361E02D
:10F470000E94F3FB85E361E00E94F3FB85E361E01A
:10F480000E94A6FC85E08A8382E58CBD1DBC80E0DD
:10F490009FEF9EBD0DB407FEFDCF8F5F8A30C9F789
:10F4A00009C00E944CFA6C197D09615D774010F02B
:10F4B00081E059C0CE0160E020E030E040E050E063
:10F4C0003BDE182F8B83813061F7CE0168E02AEA9A
:10F4D00031E040E050E030DE82FF02C01C8311C00A
:10F4E00080E02FEF2EBD0DB407FEFDCF9EB58F5FE0
:10F4F0008430C1F79B839A3A11F082E034C082E0F5
:10F500008C838C81823021F0EE24FF2487010FC090
:10F51000E12CF12C012D00E4102F09C00E944CFABF
:10F520006C197D09615D774010F08AE01CC0CE0146
:10F5300067E320E030E040E050E0FEDDCE0169E22C
:10F54000A8019701F9DD8B83882341F78C818230F4
:10F5500019F5CE016AE320E030E040E050E0ECDD58
:10F56000882329F088E08983CE013FDE20C08FEF19
:10F570008EBD0DB407FEFDCF8EB5807C803C11F4AE
:10F5800083E08C8380E09FEF9EBD0DB407FEFDCF2E
:10F590002EB58F5F8330C1F7CE0127DE86E08B1555
:10F5A00018F488E1898303C0BA8281E001C080E059
:10F5B000DF91CF911F910F91FF90EF90DF90CF904F
:10F5C000BF9008958091F50C882389F14091EF0A4E
:10F5D0005091F00A6091F10A7091F20A8091F30C57
:10F5E0009091F40C23EF3AE03EDE882311F1409134
:10F5F000F60C5091F70C6091F80C7091F90C4115D4
:10F6000051056105710589F08091F30C9091F40C1E
:10F6100023EF3AE028DE882361F01092F60C109276
:10F62000F70C1092F80C1092F90C1092F50C81E086
:10F63000089580E00895DF92EF92FF920F931F9359
:10F640007B018C01D42E8091EF0A9091F00AA09159
:10F65000F10AB091F20A8E159F05A007B107B1F02B
:10F66000B1DF8823D9F08091F30C9091F40CB801AC
:10F67000A70123EF3AE0AADE882381F0E092EF0AA7
:10F68000F092F00A0093F10A1093F20ADD2011F4CF
:10F6900081E005C081E08093F50C01C080E01F91FE
:10F6A0000F91FF90EF90DF9008958F929F92AF920D
:10F6B000BF92CF92DF92EF92FF920F931F93CF935F
:10F6C000DF936C01142F7093F40C6093F30CFC0126
:10F6D000178A82E090E0A0E0B0E080839183A2836B
:10F6E000B3831092F50C1092F60C1092F70C109256
:10F6F000F80C1092F90C8FEF9FEFAFEFBFEF8093F4
:10F70000EF0A9093F00AA093F10AB093F20A44230F
:10F7100021F48824992454013FC0453008F01CC1CD
:10F7200060E070E080E090E040E085DF882309F44D
:10F7300013C1C12FD0E02197FE0174E0EE0FFF1F2F
:10F740007A95E1F7ED50F54FE254FE4F8081EE5B84
:10F75000F14090E08F779070892B09F0FDC0E6535F
:10F76000FE4F80819181A281B38184369105A105EC
:10F77000B10508F4F1C064E0CC0FDD1F6A95E1F734
:10F78000C754D34F88809980AA80BB80811491048C
:10F79000A104B10409F4E0C0C501B40140E04BDFAD
:10F7A000882309F4D9C08091FE0A9091FF0A805005
:10F7B000924009F0D1C02091030B222309F4CCC060
:10F7C0008091010B9091020B892B09F4C5C08091A7
:10F7D000000B882309F4C0C0F601228B8091000B36
:10F7E0008483158661E070E007C04F5FF6014587AE
:10F7F0004150483008F0B0C0F6014585848190E062
:10F800009B01042E02C0220F331F0A94E2F78217D5
:10F81000930759F72091090B30910A0B21153105F7
:10F8200019F040E050E008C02091170B3091180B00
:10F830004091190B50911A0BF601258336834783AB
:10F840005087E090010BF090020B00E010E0E80C14
:10F85000F91C0A1D1B1DE38AF48A058B168B809107
:10F86000040B9091050B918F808F6091030B70E0DA
:10F8700080E090E00F9486056E0D7F1D801F911F24
:10F88000F601628F738F848F958F2091040B3091D6
:10F89000050B55E0220F331F5A95E1F721503E4FDB
:10F8A000232F3327269540E050E0260F371F481FAF
:10F8B000591F26873787408B518B8091060B90917B
:10F8C000070B009719F0A0E0B0E008C08091130B7F
:10F8D0009091140BA091150BB091160B850174013A
:10F8E000E21AF30A040B150BA8019701280F391F20
:10F8F0004A1F5B1FF601058404C05695479537954E
:10F9000027950A94D2F72187328743875487253F6A
:10F91000FFE03F07F0E04F07F0E05F0720F48CE0E6
:10F92000F601878B19C0255F3F4F4040504018F4C7
:10F9300080E1F6010EC080911F0B9091200BA091E9
:10F94000210BB091220BF601828F938FA48FB58F7C
:10F9500080E2878B81E001C080E0DF91CF911F9131
:10F960000F91FF90EF90DF90CF90BF90AF909F905E
:10F970008F9008956F927F928F929F92AF92BF92D5
:10F98000CF92DF92EF92FF920F931F93CF93DF936B
:10F99000EC015A016B013801490142305105610502
:10F9A000710508F45DC089859A85AB85BC85019693
:10F9B000A11DB11D84179507A607B70708F450C00D
:10F9C0008F89803129F4E52EF62E072F11270CC0E0
:10F9D000803209F045C07A018B0187E016950795C2
:10F9E000F794E7948A95D1F78B899C89AD89BE8974
:10F9F000E80EF91E0A1F1B1FC801B70141E01BDEFC
:10FA0000882371F18F89803149F4F501F070EE0F90
:10FA1000FF1FED50F54F718260820DC0F501EF7749
:10FA2000F070EE0FFF1FEE0FFF1FED50F54F6082DD
:10FA30007182828293828A89823080F08D819E8158
:10FA4000AF81B885E80EF91E0A1F1B1FE092F60C65
:10FA5000F092F70C0093F80C1093F90C81E001C0C0
:10FA600080E0DF91CF911F910F91FF90EF90DF9099
:10FA7000CF90BF90AF909F908F907F906F900895A0
:10FA8000CF92DF92EF92FF920F931F93CF93DF936A
:10FA9000EC017A018B01690189859A85AB85BC856A
:10FAA0000196A11DB11D84179507A607B70708F495
:10FAB00052C08F89803129F45527412F302F2F2DA7
:10FAC0000CC0803209F047C09A01AB0167E056953F
:10FAD0004795379527956A95D1F78B899C89AD898C
:10FAE000BE89280F391F4A1F5B1F8091EF0A909132
:10FAF000F00AA091F10AB091F20A281739074A07D3
:10FB00005B0731F0CA01B90140E095DD882319F1A6
:10FB10008F89803159F4F701F070EE0FFF1FED501F
:10FB2000F54F80819181A0E0B0E00EC0F701EF7742
:10FB3000F070EE0FFF1FEE0FFF1FED50F54F8081AD
:10FB40009181A281B381BF70F60180839183A283EA
:10FB5000B38381E001C080E0DF91CF911F910F91CD
:10FB6000FF90EF90DF90CF900895AF92BF92CF9229
:10FB7000DF92EF92FF920F931F93DF93CF9300D00A
:10FB80000F92CDB7DEB76C017A018B0182E090E075
:10FB9000A0E0B0E0F60180839183A283B3835E018D
:10FBA0000894A11CB11CC601B801A701950168DF2A
:10FBB000882339F1C601B801A70100E010E020E078
:10FBC00030E0D8DE8823E9F0E980FA800B811C81DF
:10FBD000F6018789803151F4F8EFEF16FFEFFF0649
:10FBE000F0E00F07F0E01F07F0F209C088EFE81619
:10FBF0008FEFF8068FEF08078FE01807A0F281E07B
:10FC000001C080E00F900F900F900F90CF91DF9187
:10FC10001F910F91FF90EF90DF90CF90BF90AF902A
:10FC200008954F925F926F927F928F929F92AF92C0
:10FC3000BF92CF92DF92EF92FF920F931F93DF93C9
:10FC4000CF9300D00F92CDB7DEB76C0149835A83B2
:10FC50006B837C833901EE24FF2487012E010894F5
:10FC6000411C511C812CE2E09E2EA12CB12C49811B
:10FC70005A816B817C81C601920102DF882339F1B0
:10FC8000D501C401F601058404C0880F991FAA1F7D
:10FC9000BB1F0A94D2F7E80EF91E0A1F1B1F298109
:10FCA0003A814B815C818789803131F4285F3F4FF5
:10FCB00040405040E0F205C0285F3F4F4F4F5F404B
:10FCC000B0F2F301E082F1820283138381E00F90AE
:10FCD0000F900F900F90CF91DF911F910F91FF9098
:10FCE000EF90DF90CF90BF90AF909F908F907F90DC
:10FCF0006F905F904F9008952F923F924F925F9236
:10FD00006F927F928F929F92AF92BF92CF92DF922B
:10FD1000EF92FF920F931F93DF93CF93CDB7DEB790
:10FD20002F970FB6F894DEBF0FBECDBF1C014A87D8
:10FD30005B876C877D873F872E87DC0119968D91C5
:10FD40009D910D90BC91A02D0196A11DB11D8E839A
:10FD50009F83A887B987F9010081118122813381AE
:10FD6000011511052105310549F048015901089493
:10FD7000811C911CA11CB11C1D8210C0D1018D9051
:10FD80009D90AD90BC901D828A859B85AC85BD857C
:10FD90000197A105B10511F491E09D8375016401FE
:10FDA0004424552432018E010F5F1F4FF1018185DC
:10FDB0009285A385B485481659066A067B0608F025
:10FDC0008CC08E819F81A885B9858C159D05AE0557
:10FDD000BF0550F4A2E08A2E912CA12CB12CF2E0A8
:10FDE000CF2ED12CE12CF12CC101B701A601980135
:10FDF00047DE882309F471C089819A81AB81BC8177
:10FE0000A70196012F5F3F4F4F4F5F4F0097A1050E
:10FE1000B10519F049015A010DC0281939094A09DB
:10FE20005B098A859B85AC85BD85281739074A07FC
:10FE30005B0759F00894411C511C611C711C08940B
:10FE4000C11CD11CE11CF11CB1CFC101A601B7013D
:10FE50000FEF1FEF2FEF3FE08DDD882391F43DC0C2
:10FE60002601370108944108510861087108C10151
:10FE7000B301A201970186017DDD882371F1730131
:10FE800062018C149D04AE04BF0450F3AE85BF859F
:10FE90004D915D916D917C91411551056105710503
:10FEA00031F0C1019501840165DD8823B1F0EE8553
:10FEB000FF8580829182A282B382FD81FF2359F067
:10FEC0000894811C911CA11CB11CD1018D929D92A2
:10FED000AD92BC92139781E001C080E02F960FB6DF
:10FEE000F894DEBF0FBECDBFCF91DF911F910F9170
:10FEF000FF90EF90DF90CF90BF90AF909F908F904A
:10FF00007F906F905F904F903F902F900895DB010E
:10FF10000D900020E9F71197A61BB70B0496AD01D1
:10FF200081C5DF93CF930F92CDB7DEB76983049677
:10FF3000BE016F5F7F4F41E050E074D50F90CF91CD
:10FF4000DF910895CF93DF93EB01DC0190E020E097
:10FF50003EE28C91803269F0283029F4FE01E90FED
:10FF6000F11D30839F5FFE01E90FF11D8C918083AD
:10FF70009F5F2F5F11962B3061F7C90FD11D18823B
:10FF8000DF91CF9108950F931F93CF93DF93DC01FF
:10FF9000EB018A0180E090E020E2FE01E80FF91F0A
:10FFA000208301968B309105C1F757E040E024C0D3
:10FFB000622F2E3219F080E894E107C05A3051F1D7
:10FFC0005AE048E018C0321729F1FC01019634913B
:10FFD0003323C9F75417F0F02132E0F02F37D0F473
:10FFE000822F81568A3110F4622F6052FE01E40F95
:10FFF000F11D60834F5F11962C91222311F02F3257
:020000021000EC
:10000000B9F6F801B183A08390E08881803219F0BD
:1000100091E001C090E0892FDF91CF911F910F9166
:1000200008956F927F928F929F92AF92BF92CF92DC
:10003000DF92EF92FF920F931F93CF93DF93EC0128
:100040007A018B012B81222309F47FC089899A8947
:10005000AB89BC8984179507A607B70708F475C054
:1000600084C0E114F1040105110551F41C821D82C4
:100070001E821F82188619861A861B8681E066C03A
:10008000288539854A855B85E98DFA8D858590E0DF
:100090000996215030404040504039014A01082E15
:1000A00004C096948794779467940A94D2F72F5F4C
:1000B0003F4F4F4F5F4F0894E108F10801091109C4
:1000C0005701680104C0D694C794B794A7948A9541
:1000D000D2F70894E11CF11C011D111DA614B704F0
:1000E000C804D90428F0211531054105510549F40A
:1000F0008D899E89AF89B88D8C839D83AE83BF83A4
:1001000015C0A618B708C808D90810C04C815D8171
:100110006E817F81898D9A8D9401B2DC0894A1084B
:10012000B108C108D108882331F40FC084E0882EBB
:10013000912C8C0E9D1EA114B104C104D10431F781
:10014000E886F9860A871B8799CF80E0DF91CF91F7
:100150001F910F91FF90EF90DF90CF90BF90AF90E5
:100160009F908F907F906F900895223009F079CF03
:10017000E7CFCF93DF93EC018C859D85AE85BF855E
:1001800040E0611141E0BC01CD0155DA882319F44A
:1001900020E030E00AC08889282F30E095E0220F67
:1001A000331F9A95E1F72D50354FC901DF91CF915B
:1001B00008950F931F93CF93DF938C01FC018381EC
:1001C0008823D1F1818187FF35C0C80161E0D1DF8B
:1001D000EC01009789F18881853E71F1F8018381F6
:1001E000823040F481899289A389B4898C8F9D8F54
:1001F000AE8FBF8FF80185899689A789B08D9B8FB7
:100200008A8FCD01AA27BB279D8B8C8BE091FA0C9E
:10021000F091FB0C309751F0BE016A5E7F4FCE012A
:1002200048961995888D998D9B8B8A8BF8018181D1
:100230008F778183C7D904C081E0F801808380E093
:10024000DF91CF911F910F9108950F931F938C0110
:10025000B0DFF80113821F910F910895FC01838193
:10026000882311F0CF01F1CF0895CF93DF93FC01E4
:10027000EB018381882381F08250823020F48FE269
:100280008883198207C0CF0160E073DF009721F0F7
:10029000BE0158DE81E001C080E0DF91CF9108957A
:1002A0006F927F928F929F92AF92BF92CF92DF9286
:1002B000EF92FF920F931F93DF93CF9300D00F9293
:1002C000CDB7DEB77C015A016B01DC0113968C912E
:1002D0001397813009F08AC011968C9181FF86C0F6
:1002E00099C00097A105B10511F481E080C0F70124
:1002F0006084718482849384C701B601A50191DE74
:10030000882309F473C0D70159968D919C915A970F
:10031000A114B104C104D10481F455964D915D91AD
:100320006D917C91589721DC882309F45FC0F70117
:10033000158A168A178A108E41C0D70114964D91DE
:100340005D916D917C9117979E012F5F3F4F98DBD8
:10035000882309F44BC0D7015996ED91FC915A9727
:1003600049815A816B817C818789803149F4483F7A
:10037000BFEF5B07B0E06B07B0E07B0748F01EC043
:10038000483F8FEF58078FEF68078FE07807B0F48A
:10039000CF01EBDB882351F1D70114964D915D918C
:1003A0006D917C91179759968D919C915A970FEF6B
:1003B0001FEF2FEF3FE0DEDA8823C1F0F701A18ABB
:1003C000B28AC38AD48A818180688183C701F1DEC1
:1003D000882361F0B601A5016A147B048C049D0496
:1003E00010F4B401A301C7011CDE01C080E00F902E
:1003F0000F900F900F90CF91DF911F910F91FF9071
:10040000EF90DF90CF90BF90AF909F908F907F90B4
:100410006F900895F70181899289A389B48984171F
:100420009507A607B70708F05CCFE0CFCF93DF931F
:10043000EC0140E050E060E070E032DF882359F0EA
:10044000CE0161E096DEFC01009729F085EE808305
:100450001B82B8D801C080E0DF91CF9108952F9220
:100460003F924F925F926F927F928F929F92AF9244
:10047000BF92CF92DF92EF92FF920F931F93CF9391
:10048000DF93EC012A018B81882309F4B5C08981AF
:1004900080FFB2C0C7C025014E185F083B0174E061
:1004A000272E312C2C0E3D1E4201A0C028853985F7
:1004B0004A855B856FEFA62E61E0B62EA222B3229D
:1004C0008B8179018A0199E016950795F794E79455
:1004D0009A95D1F7E98DFA8D823049F4428D538D8A
:1004E000648D758D4E0D5F1D601F711F3EC0D480E1
:1004F000DA94DE20A114B104D1F4DD20C1F4211579
:1005000031054105510549F48D899E89AF89B88D22
:100510008C839D83AE83BF830AC04C815D816E81D5
:100520007F81CF019101ACDA882309F465C0E98DA0
:10053000FA8D4C815D816E817F81425050406040D8
:100540007040058404C0440F551F661F771F0A942E
:10055000D2F786859785A089B189480F591F6A1FF0
:100560007B1F4D0D511D611D711D80E092E08A19A8
:100570009B0984018815990508F48C0182E00030FC
:10058000180709F067C08091EF0A9091F00AA091D6
:10059000F10AB091F20A481759076A077B0709F474
:1005A00059C08091F30C9091F40C93010E94E6796C
:1005B000882349F421C095012D50354FC301B9015D
:1005C000A8010E943D21600E711E980140E050E09C
:1005D00088859985AA85BB85820F931FA41FB51FA7
:1005E00088879987AA87BB87801A910A811491040A
:1005F00009F05CCFA20102C04FEF5FEFCA01DF91AB
:10060000CF911F910F91FF90EF90DF90CF90BF900F
:10061000AF909F908F907F906F905F904F903F90A2
:100620002F900895A988BA88CB88DC88E884F9845B
:100630000A851B859A0140E050E0D601C5018E195C
:100640009F09A00BB10B281739074A075B0708F071
:1006500022CF24CFCB01BA0140E00E941B7B88232C
:1006600009F0A9CFC9CFCF92DF92EF92FF920F93FB
:100670001F93CF93DF937C01EB018A01FC018381FF
:10068000823008F46EC080859185A285B3858F7114
:100690009070A070B0700097A105B10509F061C01D
:1006A0006CC0F8011082EDE0CE2ED12CC701BE0146
:1006B00040E250E0D4DE9C018032910521F00097A9
:1006C00009F04FC050C04881442309F44CC0453E56
:1006D00069F34E3259F38B858F738F30E9F501152D
:1006E0001105D1F18A8D9B8D892BB1F5842F90E076
:1006F0008F719070009781F1833091056CF58C9D1E
:1007000090018D9D300D9C9D300D11242D50304059
:10071000F801E20FF31F898180838B8181838D81B2
:1007200082838F818383898584838E85858388896D
:1007300086838A8987838C8980878E898187888D43
:1007400082878C8D83878E8D8487888186FF04C005
:10075000F801E20FF31F15868B8583FDA7CF822F4B
:1007600003C08FEF01C080E0DF91CF911F910F9107
:10077000FF90EF90DF90CF9008954115510509F05B
:1007800090CF91CFDF93CF930F92CDB7DEB7BE015D
:100790006F5F7F4F41E050E062DE019719F02FEF6D
:1007A0003FEF03C08981282F30E0C9010F90CF911E
:1007B000DF910895EF92FF920F931F93CF93DF93F2
:1007C000EC018B81823030F1E884F9840A851B8545
:1007D000CE01D8DF97FD1EC088859985AA85BB8587
:1007E0004F96A11DB11D88879987AA87BB87A5E071
:1007F00016950795F794E794AA95D1F72E2D30E03A
:100800002F703070F5E0220F331FFA95E1F72D506D
:10081000354F02C020E030E0C901DF91CF911F9138
:100820000F91FF90EF9008950F931F93CF93DF9355
:10083000EC018B018B81882309F03FC0FB01878984
:10084000803109F040C082E08B831D8A1E8A1F8A96
:10085000188E808D918DA0E0B0E045E0880F991F43
:10086000AA1FBB1F4A95D1F7898B9A8BAB8BBC8B88
:1008700012C083E08B83F801428D538D648D758D9A
:100880004D8B5E8B6F8B788F9E012F5E3F4FC80123
:10089000C8D9882391F01A8F098F81E089831C823F
:1008A0001D821E821F82188619861A861B861C8648
:1008B0001D861E861F86188A01C080E0DF91CF91B9
:1008C0001F910F9108958032C1F7D3CF1F93CF931B
:1008D000DF93EC01142F262F30E0F90175E0EE0FC5
:1008E000FF1F7A95E1F7ED50F54F8385817121F077
:1008F000842F827109F066C08091EF0A9091F00A0E
:10090000A091F10AB091F20A8C879D87AE87BF87CC
:10091000688BF90165E0EE0FFF1F6A95E1F7ED5076
:10092000F54F84899589A0E0B0E0DC0199278827FC
:100930008D8B9E8BAF8BB88F228D338DA90160E09C
:1009400070E0482B592B6A2B7B2B4D8B5E8B6F8B6A
:10095000788F838590E088719070009751F4848D32
:10096000958DA68DB78D898B9A8BAB8BBC8B81E0D7
:100970000BC0409739F59E012F5E3F4F898D9A8DB0
:1009800050D98823F9F084E08B83812F8F7089837D
:100990001C821D821E821F82188619861A861B865B
:1009A00014FF16C0CE0140E050E060E070E078DC5B
:1009B000882371F409C049895A896B897C89CE01E1
:1009C00030DB02C01B8280E0DF91CF911F91089540
:1009D00015FDF1CF81E0F8CFCF93DF93EC019C01BF
:1009E0002C5F3F4F898D9A8D41E050E060E070E0D0
:1009F00083D98823A1F08D899E89AF89B88D00970E
:100A0000A105B10559F48C819D81AE81BF818D8B8B
:100A10009E8BAF8BB88F89818068898381E0DF915D
:100A2000CF9108952F923F924F925F927F928F9233
:100A30009F92AF92BF92CF92DF92EF92FF920F936D
:100A40001F93DF93CF9300D000D0CDB7DEB76C01FA
:100A5000162F072F5E834D83DC0113968C9113971D
:100A6000813009F06CC111968C9181FF68C185C1FC
:100A7000F601418952896389748980859185A285AF
:100A8000B38584179507A607B70729F0C601C9DA09
:100A9000882309F454C1812F902F9C0119014D80A6
:100AA0005E8012C1D6015996ED91FC915A97DA01F8
:100AB000C90149E0B695A795979587954A95D1F7CD
:100AC00074807A9478228FEF882E81E0982E82228B
:100AD0009322772009F052C08114910409F04EC08E
:100AE000D60114964D915D916D917C9117974115AA
:100AF00051056105710581F455968D919D910D907B
:100B0000BC91A02D0097A105B10561F1F601848388
:100B10009583A683B78332C0CF019E012F5F3F4FDD
:100B20000E94407D882309F40AC129813A814B81C2
:100B30005C81D6015996ED91FC915A978789803155
:100B400049F4283FBFEF3B07B0E04B07B0E05B073D
:100B500070F008C0283FEFEF3E07EFEF4E07EFE0E1
:100B60005E0728F0C60138DF882341F4E8C0D601CB
:100B700014962D933D934D935C93179780E092E0EC
:100B80008819990952018415950508F45C01D6016C
:100B90005996ED91FC915A971496ED90FD900D9118
:100BA0001C9117978EEF9FEFAFEFBFEFE80EF91E86
:100BB0000A1F1B1F058404C0EE0CFF1C001F111F21
:100BC0000A94D2F786859785A089B189E80EF91E27
:100BD0000A1F1B1FE70CF11C011D111D90E0A91637
:100BE00092E0B90639F58091EF0A9091F00AA09150
:100BF000F10AB091F20A8E159F05A007B10771F4B2
:100C00001092F50C8FEF9FEFAFEFBFEF8093EF0ADD
:100C10009093F00AA093F10AB093F20A8091F30C3A
:100C20009091F40CB801A70191010E9433798823B7
:100C3000B9F585C08114910419F5D60118962D9146
:100C40003D914D915C911B9751968D919D910D9089
:100C5000BC91A02D281739074A075B0788F00E942E
:100C6000E27A882309F46BC081E08093F50CE0926E
:100C7000EF0AF092F00A0093F10A1093F20A08C00A
:100C8000C801B70141E00E941B7B882309F457C0CB
:100C900094012D50354FC901B101A5010E943D219C
:100CA000950140E050E0F60180859185A285B385ED
:100CB000820F931FA41FB51F80879187A287B387D8
:100CC0002A0C3B1C4A185B08D60118962D913D91C1
:100CD0004D915C911B974114510409F0E3CE51965C
:100CE0008D919D910D90BC91A02D82179307A40723
:100CF000B50748F4F601218B328B438B548B8181ED
:100D00008068818311C08091FA0C9091FB0C892B33
:100D100059F08D819E81892B39F0D60111968C91E5
:100D20001197806811968C93F601818183FF04C02E
:100D3000C6013FDA882319F04D815E8105C081E04C
:100D4000D6018C934FEF5FEFCA0126960FB6F89449
:100D5000DEBF0FBECDBFCF91DF911F910F91FF90EE
:100D6000EF90DF90CF90BF90AF909F908F907F904B
:100D70005F904F903F902F90089582FD79CE8BCE5B
:100D8000DF92EF92FF920F931F93CF93DF93EC01CB
:100D900089899A89AB89BC89805E9F4FAF41B040F9
:100DA00008F070C0CE0118DE882309F46BC00E94E1
:100DB000E27A882309F466C0E98DFA8DEC80FD8023
:100DC0000E811F818EEF9FEFAFEFBFEFE80EF91E90
:100DD0000A1F1B1F058404C0EE0CFF1C001F111FFF
:100DE0000A94D2F786859785A089B189E80EF91E05
:100DF0000A1F1B1F81E08093F50CE092EF0AF0922E
:100E0000F00A0093F10A1093F20A80E092E0E3EF17
:100E1000FAE0DF019C011D9221503040E1F7DD2412
:100E2000D39411C0B801A7014D0D511D611D711D55
:100E30008091F30C9091F40C23EF3AE00E94337907
:100E4000882301F1D394E98DFA8D8481D81650F36B
:100E500020E032E040E050E0058404C0220F331F60
:100E6000441F551F0A94D2F789899A89AB89BC8996
:100E7000820F931FA41FB51F898B9A8BAB8BBC8BE2
:100E800081E001C080E0DF91CF911F910F91FF9031
:100E9000EF90DF9008958F929F92AF92BF92CF9282
:100EA000DF92EF92FF920F931F93CF93DF936C012A
:100EB000EB01942E852EA22E898D9A8DD6015A96FD
:100EC0009C938E935997CB0140E050E060E070E036
:100ED000A8D8BB2437C0CE016DDCFC01009709F413
:100EE00090C055E016950795F794E7945A95D1F779
:100EF0001E2D1F708081882311F0853EC9F4BB2010
:100F000099F42091EF0A3091F00A4091F10A509142
:100F1000F20AD6011C962D933D934D935C931F9737
:100F200050961C93BB24B3948081882359F418C035
:100F3000892D982DBF014BE050E00E943021009791
:100F400009F46DC0E884F9840A851B8589899A892A
:100F5000AB89BC89E816F9060A071B0708F4BBCF62
:100F6000A6FE4FC0A1FE4DC0BB2049F0F60110897E
:100F7000C60161E0FED8EC01009761F442C08B81AC
:100F8000823009F43EC0CE01FBDE8823D1F110E0AF
:100F9000C3EFDAE080E2DE011D928A95E9F7DE0117
:100FA000292D382DC901FC018BE001900D92815053
:100FB000E1F7E091FA0CF091FB0C309739F0BE01AB
:100FC000625F7F4FCE014096199508C081E298E29A
:100FD000998B888B80E098E09F878E878889998994
:100FE0009B8B8A8B998F888F8E859F859F8B8E8B0D
:100FF0000E94E27A882329F0C601612F4A2D66DC1F
:1010000001C080E0DF91CF911F910F91FF90EF9091
:10101000DF90CF90BF90AF909F908F900895A7FEE4
:10102000EBCFEFCF2F923F924F925F926F927F92D2
:101030008F929F92AF92BF92CF92DF92EF92FF92E8
:101040000F931F93DF93CF93CDB7DEB7C654D04035
:101050000FB6F894DEBF0FBECDBF3C016B01DE01C1
:10106000AE5BBF4F11965C934E9325962FAF25979D
:101070001C861F861FA21AA66115710509F47CC083
:10108000FC018381882309F077C0FA0180818F32C7
:10109000F1F08601ECE0EE2EF12CEC0EFD1E72E478
:1010A000A72EB12CAC0EBD1E4E010894811C911CC4
:1010B0002796FFAEEEAE279767E2262E312C2C0E38
:1010C0003D1E270123C01196B183A08301C0FD01FD
:1010D000A081B1818C918F32B1F3D60113968C919E
:1010E000139782508230A8F28E01095D1F4F5996E6
:1010F0006D917C915A97C80197DB882359F63CC0C3
:10110000342D252D8701832F922F7C01F5018081BD
:101110009181B401A5010E94C37F882329F42CC0CA
:101120003196D501ED93FC93D501ED91FC91808131
:101130008F32B1F38823B9F0C701B801A40121E0CF
:10114000AADE8823C9F00C151D0511F0C8017DD851
:101150002796EEADFFAD2797EE16FF0689F6C10183
:10116000322D292FCFCFC301B801A40125962FAD71
:10117000259791DE182F01C010E0CE0187966ED81A
:10118000CE010C966BD8812FCA5BDF4F0FB6F89457
:10119000DEBF0FBECDBFCF91DF911F910F91FF90AA
:1011A000EF90DF90CF90BF90AF909F908F907F9007
:1011B0006F905F904F903F902F9008950F931F93E3
:1011C000DF93CF93CDB7DEB76B970FB6F894DEBF42
:1011D0000FBECDBF9C01AB0119821C828E010F5F37
:1011E0001F4FC801B90122E01DDF882311F410E070
:1011F00003C0C8011BD9182FCE0101962FD8812F0B
:101200006B960FB6F894DEBF0FBECDBFCF91DF91C6
:101210001F910F9108953F924F925F926F927F922C
:101220008F929F92AF92BF92CF92DF92EF92FF92F6
:101230000F931F93CF93DF938091700D882309F450
:10124000F6C08090EB039090EC03A090ED03B0907B
:10125000EE0360910B0A70910C0A882777FD809548
:10126000982F0F94760220E030E040E050E40F9495
:10127000FB00A50194010F94D40187FDD8C03090E4
:1012800082120F2EF0E04F2EF0E05F2EF0E06F2E76
:10129000F0E07F2EF02DC1E5D0E058C0232D30E0E6
:1012A0002C9FF0012D9FF00D3C9FF00D1124EF5865
:1012B000F24F80819181A281B3810097A105B10590
:1012C00081F484819581A681B7810097A105B1053C
:1012D00041F480859185A285B3850097A105B1056C
:1012E00091F12C9F60012D9FD00C3C9FD00C1124BC
:1012F00081E79DE0C80ED91EF60164857585868557
:1013000097850F9476027B018C01F60160897189C3
:10131000828993890F9474029B01AC01C801B701C3
:101320000F94DB01F60122A133A144A155A10F9432
:10133000B4047B018C01A30192010F94E2031816FF
:1013400014F4270138013394FFE03F228091811289
:10135000381609F0A3CFC301B2012091EF033091F9
:10136000F0034091F1035091F2030F94B4049B01F8
:10137000AC01C501B4010F94FB007B018C01A501F8
:1013800094010F94D40187FD02C0470158011091C8
:10139000E7030091E803F090E903E090EA03C50158
:1013A000B401212F302F4F2D5E2D0F94E20318161C
:1013B00034F4812F902FAF2DBE2D4C015D01409054
:1013C0009B1250909C1260909D1270909E12C301CF
:1013D000B201A50194010F94E2031816C4F4C501EB
:1013E000B40120E037ED43EA5CE30F94B4047B01E1
:1013F0008C01C301B20128E431EE4AE75FE30F94A8
:10140000B404A80197010F94FB004B015C0180928A
:101410009B1290929C12A0929D12B0929E12C501B6
:10142000B4010F94430270930C0A60930B0ADF918E
:10143000CF911F910F91FF90EF90DF90CF90BF90D1
:10144000AF909F908F907F906F905F904F903F9064
:1014500008958091811290918212891B8F70089556
:101460006093F3037093F4038093F5039093F60372
:1014700008950F931F93CF93DF93C0E0D0E08E01C8
:10148000005B124FFE01EC5DF24F60817181828141
:1014900093810F947402FE01E05FF24F208131814D
:1014A000428153810F94B4040F944802F801608381
:1014B0007183828393832496C031D10501F7DF9134
:1014C000CF911F910F910895FC01809128088823E6
:1014D00069F4608171818281938120911C0D30912A
:1014E0001D0D40911E0D50911F0D0EC08130C1F495
:1014F00060817181828193812091200D3091210D35
:101500004091220D5091230D0F94B4040F94840444
:1015100060936C0D70936D0D80936E0D90936F0DB5
:101520008CE69DE00C94346BCF92DF92EF92FF92A9
:101530000F931F93CF93DF93FC018B017A01690115
:1015400060817181828193812091100D3091110D04
:101550004091120D5091130D0F94B4040F94840414
:10156000C0E6DDE06093600D7093610D8093620DC5
:101570009093630DF8016081718182819381209144
:10158000140D3091150D4091160D5091170D0F94BB
:10159000B4040F948404FE0134966093640D718347
:1015A00082839383F701608171818281938120918D
:1015B000180D3091190D40911A0D50911B0D0F947B
:1015C000B4040F948404FE0138966093680D71830F
:1015D0008283938380912808882371F4F6016081C7
:1015E00071818281938120911C0D30911D0D40915C
:1015F0001E0D50911F0D0FC08130C1F4F6016081A6
:101600007181828193812091200D3091210D409133
:10161000220D5091230D0F94B4040F948404FE0105
:101620003C9660936C0D71838283938380E69DE08A
:1016300064E67DE048E65DE02CE63DE00E94FA6A63
:1016400080E090E0A0E0B0E0809383129093841259
:10165000A0938512B093861280938712909388127C
:10166000A0938912B0938A1280938B1290938C125C
:10167000A0938D12B0938E1280938F12909390123C
:10168000A0939112B093921280939312909394121C
:10169000A0939512B0939612DF91CF911F910F9165
:1016A000FF90EF90DF90CF9008958F929F92AF922E
:1016B000BF92CF92DF92EF92FF920F931F93CF933F
:1016C000DF93EC016B01009709F45CC08FA98823BC
:1016D00009F058C0EEA0FFA008A519A5FB01B6A00F
:1016E000A7A090A481A4C801B7012B2D3A2D492DA4
:1016F000582D0F94D40188230CF044C0C801B701C1
:10170000A80197010F94B4047B018C016AA97BA9FD
:101710008CA99DA9905820E030E040E050EC0F9457
:10172000B4042EA53FA548A959A90F94B4049B0160
:10173000AC01C801B7010F94FB000F9421057B0198
:101740008C016B2D7A2D892D982D9701A8010F946E
:10175000D401882324F4EB2CFA2C092D182D6B2DA1
:101760007A2D892D982D9701A8010F94D4018823F3
:1017700049F0C701D801F60186A397A3A0A7B1A796
:1017800081E086ABDF91CF911F910F91FF90EF9099
:10179000DF90CF90BF90AF909F908F900895EF9281
:1017A000FF920F931F93CF93DF93F090821200E08C
:1017B00010E020E030E081E5E82E11C0FE9CE00161
:1017C0001124CF58D24FC901B801AE016EDF8F2D61
:1017D0008F5F803109F480E0F82E98018E018091AE
:1017E0008112F81659F7C901B80140E050E05DDFF9
:1017F000DF91CF911F910F91FF90EF900895AF92DD
:10180000BF92CF92DF92EF92FF920F931F93CF93ED
:10181000DF93EB018A016115710509F466C041157A
:10182000510509F462C0DAA4CBA4BCA4ADA46EA196
:101830007FA188A599A52D2D3C2D4B2D5A2D0F94B8
:10184000D401882309F451C08FA9882309F043C02B
:10185000F801E6A0F7A000A511A56D2D7C2D8B2D1C
:101860009A2DA80197010F94E2031816A4F5C80158
:10187000B701A80197010F94B4047B018C016AA9F8
:101880007BA98CA99DA9905820E030E040E050EC65
:101890000F94B4042EA53FA548A959A90F94B404E8
:1018A0009B01AC01C801B7010F94FB000F94210507
:1018B0007B018C016D2D7C2D8B2D9A2D9701A8011C
:1018C0000F94D401882324F4ED2CFC2C0B2D1A2D1D
:1018D000C701D80104C08D2D9C2DAB2DBA2D8EA330
:1018E0009FA3A8A7B9A781E08EABDF91CF911F91ED
:1018F0000F91FF90EF90DF90CF90BF90AF90089541
:10190000CF92DF92EF92FF920F93DF93CF930F92DC
:101910000F92CDB7DEB7809181128FB7F894F09017
:1019200082128FBF8091811290E040968F199109A9
:101930008F7090700497FCF00091811203500F702B
:10194000CC24DD2440E050E091E5E92E12C0802F48
:10195000002309F480E1082F01500E9DC0011124DD
:101960008F58924F9A838983B60149DFA601C980B7
:10197000DA800F1561F70F900F90CF91DF910F91E3
:10198000FF90EF90DF90CF900895CF92DF92EF928B
:10199000FF920F931F9320912A0860912C08909139
:1019A000821280918112981711F4D22E1CC040919E
:1019B0008212242F30E081E590E0289FF001299FDA
:1019C000F00D389FF00D1124EF58F24FE85BFF4FF8
:1019D00090813496608102C04F5F4F708091811278
:1019E0004817D1F7D92EC62EDD2031F1E09097129D
:1019F000F09098120091991210919A12E114F1044A
:101A00000105110579F40E944CFA6C597F4F8F4FF4
:101A10009F4F6093971270939812809399129093AE
:101A20009A1207C00E944CFA6E157F058007910735
:101A300058F4DD24DA9408C010929712109298128C
:101A40001092991210929A1286E06D2D70E00E9409
:101A500015FB88E06C2D70E00E9415FBDCDB1F910C
:101A60000F91FF90EF90DF90CF9008951092811228
:101A70001092821280E1E0E6FDE0DF011D928A957E
:101A8000E9F780E090E0A0E0B0E0809387129093C7
:101A90008812A0938912B0938A1280938B1290932C
:101AA0008C12A0938D12B0938E1280938F1290930C
:101AB0009012A0939112B0939212809393129093EC
:101AC0009412A0939512B0939612809383129093E0
:101AD0008412A0938512B093861208952F923F929C
:101AE0004F925F926F927F928F929F92AF92BF922E
:101AF000CF92DF92EF92FF920F931F93DF93CF93DA
:101B0000CDB7DEB766970FB6F894DEBF0FBECDBF78
:101B10009E8B8D8B6A017B0148015901DC01D896AF
:101B20006D917D918D919C91DB970F947402698BDF
:101B30007A8B8B8B9C8BA70196010F94B4040F9426
:101B4000C1010F9448026D837E838F8398876989D2
:101B50007A898B899C89A50194010F94B4040F9410
:101B6000C1010F94480269837A838B839C832D8102
:101B70003E814F815885283731054105510540F494
:101B800048E750E060E070E04D835E836F837887C4
:101B900069817A818B819C81683771058105910506
:101BA00040F488E790E0A0E0B0E089839A83AB83BB
:101BB000BC83AD89BE89AC5BBF4FAD90BD90CD906D
:101BC000DC901397A454B040BE8BAD8B6D817E81A9
:101BD0008F8198850F9474026D877E878F87988B8D
:101BE000C601B5010F9476021B012C0120E030E004
:101BF00040E050E00F94D401882321F4E0E070E04D
:101C000060E028C069897A898B899C899B01AC0135
